:100000000C94161A0C94471A0C94471A0C94471A1D
:100010000C94471A0C94471A0C94471A0C94471ADC
:100020000C94471A0C94471A0C94471A0C94471ACC
:100030000C94471A0C94471A0C94471A0C94471ABC
:100040000C94471A0C9499D10C94471A0C94471AA3
:100050000C94471A0C94471A0C946CBA0C940CA686
:100060000C94471A0C944A520C9440520C94471A20
:100070000C94471A0C94471A0C94471A0C94471A7C
:100080000C94471A0C94471A0C94471A0C94471A6C
:100090000C94471A0C94471A0C94471A0C94471A5C
:1000A0000C94471A0C94471A0C94471A0C94471A4C
:1000B0000C94471A0C94471A0C94471A0C94471A3C
:1000C0000C94471A0C94471A0C94471A0C94113448
:1000D0000C94DB330C94471A0C94471A0C94471A6F
:1000E0000C94471A084AD73B3BCE016E84BCBFFD37
:1000F000C12F3D6C74319ABD56833DDA3D00C77FF8
:1001000011BED9E4BB4C3E916BAAAABE0000008090
:100110003F05A84CCDB2D44EB93836A9020C50B91F
:10012000918688083CA6AAAA2ABE000000803F004B
:100130000C946A410D94A7080C9430F70C94C49E5B
:100140000C943EA30C94E4520D947D040C94E05264
:100150000C946FF90D940F000C9483A20D94A803D6
:100160000C9488520C94FD400C94C6520C94F0529E
:100170000C949E9E0C9479A20D9440050C94A89E1C
:100180000C9497A20C94479F0D94B7080C94EBFB2A
:100190000C9446A20C9444F90C94949E0C946CFD1F
:1001A0000D9404030C94AC9E0C948D9E0C94BA9EFA
:1001B0000C94A49E0D94A4010C948DA20C94C234B2
:1001C0000C94B69E0C94E8520C94BAA30C94D8A24A
:1001D0000C940E530C94A3340D94D8010C94DC525F
:1001E0000C94BAA20D943A030D94AA070C94899E1C
:1001F0000C944BA20C941FA50C94CEA20D949004C9
:100200000C94E23E0C949A9E0D9474020C94739E8E
:100210000C94A7340C947E340C94DAFA0C94B29EAD
:100220000D94510C0C945AF80C945FA20C94D53494
:100230000C94B3340D94CB070C946E9E0C949C34A8
:100240000C94AF340C94B7520C94A6A20C943EA21A
:100250000C94FB520C94CA9F0C94BB340C94F2A4E3
:100260000C948D340D9455010C94353F0C94C99F1A
:100270000D943B040C9471A20D94D1030D94E503ED
:100280000C94F4520D9488010D944A070C9469A2C1
:100290000D9471070C94C4A20C94EC520D94920727
:1002A0000D947A090C94AB340D94B7190C94D55273
:1002B0000C94E0A40D947A070D941C040C9429412D
:1002C0000C94859E0C945BA30C94A2410C94CD34A9
:1002D0000C94919E0C944F340C94C09E0D9477070F
:1002E0000C9406530C9403A40C9455A20D949919E4
:1002F0000D94BE070D9408040C9462A40C9447A4BA
:100300000C94313F0C94B0A20D94A0070C9442A51C
:100310000C94B7344E414E494E495459494E46CD3E
:10032000CCCC3D0AD7233C17B7D13877CC2B3295AC
:1003300095E6241FB14F0A000020410000C842008A
:10034000401C4620BCBE4CCA1B0E5AAEC59D740054
:10035000407A10F35A00A0724E18090010A5D4E894
:100360000000E87648170000E40B54020000CA9A27
:100370003B000000E1F50500008096980000004079
:10038000420F000000A086010000001027000000BE
:1003900000E803000000006400000000000A000004
:1003A0000000000100000000002C76D888DC674FB8
:1003B0000823DFC1DFAE59E1B1B796E5E3E453C6E8
:1003C0003AE651997696E8E6C28426EB898C9B62E0
:1003D000ED407C6FFCEFBC9C9F40F2BAA56FA5F48A
:1003E00090055A2AF75C936B6CF9676DC11BFCE0B2
:1003F000E40D47FEF520E6B500D0ED902E03009405
:100400003577050080841E080000204E0A00000099
:10041000C80C333333330F986E12831141EF8D21A3
:1004200014893BE65516CFFEE6DB18D1844B381B0A
:10043000F77C1D901DA4BBE424203284725E2281CF
:1004400000C9F124ECA1E53D27434F4D4D554E49E0
:10045000434154494F4E0044525952554E00455263
:10046000524F525300494E464F004543484F0045B6
:1004700072726F722077726974696E6720746F2070
:10048000454550524F4D210A0053544F505045445A
:100490002E20005072696E7465722073746F7070D4
:1004A00065642064756520746F206572726F727365
:1004B0002E2046697820746865206572726F7220FC
:1004C000616E6420757365204D39393920746F2051
:1004D000726573746172742E202854656D70657234
:1004E00061747572652069732072657365742E205E
:1004F0005365742069742061667465722072657337
:1005000074617274696E67290A004E6F20436865D2
:10051000636B73756D2077697468206C696E6520F4
:100520006E756D6265722C204C617374204C696E1F
:10053000653A20004E6F20436865636B73756D20CC
:1005400077697468206C696E65206E756D6265727E
:100550002C204C617374204C696E653A20006368EE
:1005600065636B73756D206D69736D617463682C61
:10057000204C617374204C696E653A20004C696EA2
:1005800065204E756D626572206973206E6F7420F0
:100590004C617374204C696E65204E756D62657296
:1005A0002B312C204C617374204C696E653A20000D
:1005B0004D3131300053657269616C207374617420
:1005C0007573206D69736D617463680A0077616982
:1005D000740A0053442072656164206572726F7200
:1005E0000A002121204B494C4C20636175736564DE
:1005F00020627920746F6F206D75636820696E6169
:1006000063746976652074696D65202D2063757249
:1006100072656E7420636F6D6D616E643A20004880
:100620006F74656E642049646C652054696D656FF4
:10063000757400486F74656E642049646C6520545D
:10064000696D656F75740A003D3D6F6E46696C613A
:100650006D656E7452756E6F75743D3D0070617599
:100660007365004D363030002066696C616D656ED3
:10067000745F72756E6F7574200066696C616D656C
:100680006E745F72756E6F757420540046696C618C
:100690006D656E7452756E6F75742054002A2A2A27
:1006A000496E6974696E67206361726420697320A2
:1006B0004F4B2A2A2A004D6564696120496E736593
:1006C00072746564004D656469612052656D6F7672
:1006D0006564004D313030305300627573793A20D3
:1006E00070617573656420666F7220696E707574D1
:1006F0000A00627573793A207061757365642066CB
:100700006F7220757365720A00627573793A207092
:10071000726F63657373696E670A002A2A2A6B69B0
:100720006C6C2A2A2A00706F7765726F6666004BC0
:10073000494C4C45442E20005072696E74657220FD
:1007400068616C7465642E206B696C6C2829206369
:10075000616C6C6564210A006563686F3A004572DC
:10076000726F723A0042696C696E656172204C6505
:1007700076656C696E6720477269643A0A002F2FAC
:10078000616374696F6E3A0070726F6D70745F00B0
:10079000656E640053656E64204D31303820746F8F
:1007A00020726573756D650A00496E7365727420F9
:1007B00066696C616D656E7420616E642073656E30
:1007C00064204D3130380A005265686561742066D6
:1007D000696E69736865642E00526568656174208E
:1007E000446F6E6500526568656174696E672E2E90
:1007F0002E005265686561740048656174657220F9
:1008000054696D656F75740053656E64204D3130A9
:100810003820746F2068656174206E6F7A7A6C6519
:100820000A004E6F7A7A6C65205061726B656400C5
:10083000486F74656E6420746F6F20636F6C640A18
:10084000007061757365640050617573650044697B
:100850007361626C6552756E6F7574005075726766
:10086000654D6F7265005061757365640073686FE4
:100870007700627574746F6E00626567696E004C14
:100880006F61642046696C616D656E74004C6F61C8
:10089000642046696C616D656E74205400496E7306
:1008A0006572742066696C616D656E7420616E643A
:1008B0002073656E64204D3130380A00726573759F
:1008C0006D656400526573756D696E670057616987
:1008D00074696E6720666F72206865617475702E2A
:1008E0000A004C656176696E6720473236003F53D7
:1008F000706563696669656420582C5920636F6F61
:100900007264696E617465206F7574206F66206211
:100910006F756E64732E0A003F28522965706561F9
:10092000742076616C7565206E6F7420706C6175D3
:100930007369626C653B206D75737420626520611C
:1009400074206C6561737420312E0A003F2852298F
:100950006570656174206D757374206265207370B5
:1009600065636966696564207768656E206E6F747B
:10097000207573696E6720616E204C43442E0A0017
:100980003F537065636966696564206E6F7A7A6C3F
:10099000652074656D7065726174757265206E6F27
:1009A0007420706C61757369626C652E0A003F5328
:1009B00070656369666965642066696C616D656E02
:1009C000742073697A65206E6F7420706C61757322
:1009D00069626C652E0A003F5370656369666965DC
:1009E00064207072696D65206C656E677468206E36
:1009F0006F7420706C61757369626C652E0A003FBC
:100A00005072696D65206C656E677468206D7573D2
:100A10007420626520737065636966696564207718
:100A200068656E206E6F74207573696E6720616EE5
:100A3000204C43442E0A003F537065636966696524
:100A400064206E6F7A7A6C652073697A65206E6FA8
:100A50007420706C61757369626C652E0A003F5278
:100A6000657472616374696F6E204D756C74697022
:100A70006C696572206D7573742062652073706592
:100A80006369666965642E0A003F53706563696631
:100A90006965642052657472616374696F6E204D7C
:100AA000756C7469706C696572206E6F7420706CFF
:100AB00061757369626C652E0A003F5370656369E6
:100AC00066696564206C617965722068656967682C
:100AD00074206E6F7420706C61757369626C652E22
:100AE0000A0043292E0A003F5370656369666965F1
:100AF00064206265642074656D70657261747572DE
:100B000065206E6F7420706C61757369626C65200E
:100B10002834302D00473236207374617274696E48
:100B2000672E2E2E0A004F46460A00466164652055
:100B30004865696768742000426564204C65766585
:100B40006C696E6720004661696C656420746F2073
:100B5000656E61626C6520426564204C6576656CEB
:100B6000696E670A00496E76616C6964206D657311
:100B7000682E0A0050726F62696E6720506F696E4E
:100B8000740025532025692F2569002E0A002F00A7
:100B900050726F62696E67206D65736820706F694F
:100BA0006E742000202844525952554E2900473275
:100BB00039204175746F20426564204C6576656C00
:100BC000696E67003F20284C2C522C462C4229206D
:100BD0006F7574206F6620626F756E64732E0A00E5
:100BE0003F2856296572626F7365206C6576656C67
:100BF00020696D706C61757369626C652028302D99
:100C000034292E0A00426164205A2076616C756591
:100C10000A004E6F2062696C696E656172206772AE
:100C200069640A00446576696174696F6E002553D2
:100C30003A2025730046696E6973686564210A006D
:100C40003A207A3A2000206F662000476F696E676D
:100C500020746F3A20580043570A00206469723AA2
:100C60000020616E676C653A005374617274207283
:100C700061646975733A004D343820506F696E7441
:100C80000025533A2025642F256400506F73697442
:100C9000696F6E696E67207468652070726F626537
:100CA0002E2E2E0A003F4C656773206F66206D6FF5
:100CB00076656D656E7420696D706C6175736962BF
:100CC0006C652028302D3135292E0A003F20285808
:100CD0002C5929206F7574206F6620626F756E64C1
:100CE000732E0A0050726F6265206F7574206F66F4
:100CF00020626F756E6473003F53616D706C652088
:100D000073697A65206E6F7420706C6175736962A7
:100D10006C652028342D3530292E0A004D343820BA
:100D20005A2D50726F626520526570656174616200
:100D3000696C69747920546573740A003F285629D8
:100D40006572626F7365206C6576656C20696D7085
:100D50006C61757369626C652028302D34292E0A08
:100D6000005374616E6461726420446576696174D5
:100D7000696F6E3A20002052616E67653A2000204C
:100D80004D61783A2000204D696E3A200020536969
:100D9000676D613A20004D65616E3A2000574152FF
:100DA0004E494E4721204C6F77205A204A65726B7E
:100DB000206D6179206C65616420746F20756E7799
:100DC000616E746564207061757365732E0A004FDF
:100DD0004646004F4E0020204D61783A200020000A
:100DE00020204D696E3A2000536F667420656E6452
:100DF00073746F70733A20003D3D4F6E506F77658E
:100E0000724C6F7373526573756D653D3D004D3265
:100E1000342053256C642054256C64004739322EED
:100E20003920452573004731204625640047393273
:100E30002E39205A2573004731205A30204632304F
:100E40003000473120582573205925732046333010
:100E50003030004D34323020532569205A2573003C
:100E60004D3130362050256920532569004D3230F0
:100E700030204425730047323852305859004739E2
:100E8000322E39204530205A300A47315A25730016
:100E90004D31303920532569004D313930205325EB
:100EA00069004D343230205330205A300020496ED2
:100EB00076616C696420657874727564657220006F
:100EC00047322F47332062616420706172616D6523
:100ED000746572730A00536C6565702E2E2E005A6D
:100EE0002050726F62652050617374204265640AFD
:100EF000005A2050726F6265205061737420426501
:100F000064004732384C30004D3131372050726F19
:100F10006265206661696C65642E0A4732380A0092
:100F200070726F62655F726577697065004732390C
:100F3000205265747279696E670050726F62696ED3
:100F400067204661696C6564004D31313720426528
:100F500064206C6576656C696E67206661696C6596
:100F6000642E0A4730205A31300A4D333030205039
:100F7000323520533838300A4D3330302050353038
:100F80002053300A4D33303020503235205338381A
:100F9000300A4D333030205035302053300A4D3335
:100FA00030302050323520533838300A4D3330300D
:100FB000205035302053300A4734205331007072AE
:100FC0006F62655F6661696C6564004D3131372021
:100FD000426564206C6576656C696E6720646F6E2F
:100FE000652E00205A3A200020593A2000426564BC
:100FF00020583A20004D65736820706F696E742028
:101000006F7574206F662072616E67650A004D30DF
:101010002053746F70004D312053746F7000436F14
:101020006E74696E756500436C69636B20746F2024
:10103000526573756D652E2E2E004E6F204D6F76A6
:10104000652E00456E642066696C65206C6973745A
:101050000A00426567696E2066696C65206C697379
:10106000740A004E6F206D656469610A00526573F1
:10107000756D696E6720534400286E6F2066696C39
:1010800065290043757272656E742066696C653AF5
:1010900020005072696E742074696D653A20000AF0
:1010A00053746174733A2046696C616D656E742087
:1010B000757365643A20002C204C6F6E67657374FD
:1010C000206A6F623A2000546F74616C2074696DFD
:1010D000653A200053746174733A20002C204661F5
:1010E000696C65643A20002C2046696E69736865F6
:1010F000643A20005072696E74733A200053746130
:1011000074733A2000436F6F6C696E672E2E2E0049
:1011100048656174696E672E2E2E004520255300A8
:101120006F6B006F6666006A0465045E04570449CD
:101130000444454255473A004D3131332053004273
:10114000656420436F6F6C696E672E2E2E004265BA
:10115000642048656174696E672E2E2E00444458E1
:10116000203130532050726F204F46462E002F2FD3
:1011700000205200416363656C65726174696F6E33
:101180003A2050004D32303620580046523A002066
:10119000466C6F773A200020643A0020693A0020BC
:1011A000703A00496E76616C696420657874727576
:1011B0006465720A0020643A0020693A0020703A9F
:1011C0000064697300656E0043290A0061626C6502
:1011D0006420286D696E2074656D702000436F6C0B
:1011E000642065787472756465732061726520008F
:1011F000504944204175746F74756E6500504944C0
:10120000204175746F74756E65206661696C6564E4
:101210002120426164206865617465722069640AF6
:101220000046696C616D656E742072756E6F7574C1
:101230002064697374616E636520286D6D293A209E
:101240000046696C616D656E742072756E6F7574A1
:1012500020004D34323120696E636F7272656374A1
:1012600020706172616D6574657220757361676568
:101270000A004D65736820706F696E74206F757415
:10128000206F662072616E67650A004F666673653F
:101290007473204170706C696564004572723A2005
:1012A000546F6F206661722100546F6F2066617207
:1012B0002066726F6D207265666572656E6365206B
:1012C000706F696E740A00454550524F4D204F4B68
:1012D0000A00506F7765722D6C6F737320726563AF
:1012E0006F7665727920004D383400446F6E65204A
:1012F0007072696E74696E672066696C650A004D6C
:101300003737004D3331004361703A004D45415449
:101310005041434B00434F4F4C45525F54454D5055
:1013200045524154555245004348414D4245525F54
:1013300054454D5045524154555245004241425941
:101340005354455050494E470041524353004D4F6E
:1013500054494F4E5F4D4F44455300544845524DFC
:10136000414C5F50524F54454354494F4E004C4FEF
:101370004E475F46494C454E414D45004155544FFF
:101380005245504F52545F53445F53544154555348
:101390000053445F5752495445005245504541540B
:1013A000005344434152440050524F4D50545F53F8
:1013B0005550504F525400454D455247454E4359A4
:1013C0005F50415253455200434153455F4C49479A
:1013D00048545F4252494748544E45535300544F76
:1013E00047474C455F4C494748545300534F465478
:1013F000574152455F504F574552004255494C4462
:101400005F50455243454E54004C4556454C494E5D
:10141000475F44415441005A5F50524F4245005289
:10142000554E4F5554004155544F4C4556454C0070
:101430005052494E545F4A4F420050524F47524516
:101440005353004155544F5245504F52545F5445E9
:101450004D5000564F4C554D45545249430045455B
:1014600050524F4D0042494E4152595F46494C45FA
:101470005F5452414E534645520053455249414CE8
:101480005F584F4E5F584F4646004649524D5741B0
:1014900052455F4E414D453A4D61726C696E203246
:1014A0002E302E375F4457372E3320426F6E6474D0
:1014B0006563682053534D444E422028417072208A
:1014C000323920323032312031313A30333A31370B
:1014D0002920534F555243455F434F44455F555272
:1014E0004C3A68747470733A2F2F67697468756228
:1014F0002E636F6D2F496E73616E697479417574D7
:101500006F6D6174696F6E2F4D61726C696E2F74AF
:101510007265652F437265616C6974794477696E91
:101520005F322E302050524F544F434F4C5F564540
:101530005253494F4E3A312E30204D414348494E87
:10154000455F545950453A44445820313053205057
:10155000726F2045585452554445525F434F554E83
:10156000543A3120555549443A63656465326132D5
:10157000662D343161322D343734382D39623132B1
:101580002D6335356336326633363766660A00506A
:10159000726F6265204F6666736574205A005072E0
:1015A0006F6265204F6666736574205A00290A00D1
:1015B00020746F20003F5A206F7574206F66207270
:1015C000616E6765202800290A0020746F20003FA3
:1015D00059206F7574206F662072616E67652028D0
:1015E0002D00290A0020746F20003F58206F757469
:1015F000206F662072616E676520282D0050726F23
:101600006265204F666673657420580043616E6E94
:101610006F74206F70656E2073756264697220004C
:101620002569730025696D20256973002569682087
:1016300025696D2025697300256964202569682066
:1016400025696D2025697300256979202569642045
:101650002569682025696D20256973003D3D447723
:10166000696E20496E697420436F6D706C65746596
:101670003D3D002A2A2A4E6F7A7A6C6554656D705A
:101680005374617475735B325D203D003D3D486568
:101690006174696E6720446F6E65204368616E6790
:1016A000652046696C616D656E743D3D0020207358
:1016B0007461727470726F677265737320003D3D60
:1016C0007761697477617920353D3D003D3D7761F3
:1016D000697477617920343D3D003D3D77616974DF
:1016E00077617920333D3D003D3D776169747761D5
:1016F0007920313D3D003D3D6F6E5072696E7454EE
:10170000696D657253746F707065643D3D003D3D59
:101710006F6E466163746F727952657365743D3D97
:1017200000270A0A0000272027002027002D006E2E
:101730006F74696669636174696F6E200063616EBE
:1017400063656C005072696E742041626F727465DB
:1017500064004469736D6973730055492041626F79
:101760007274656400726573756D65004D32340086
:101770002A2A2A43506C617920546F6E652A2A2ADE
:10178000003D3D6F6E5072696E7454696D657250A4
:1017900061757365643D3D00486F6D696E672046F5
:1017A00061696C6564006F70656E0054524947470B
:1017B00045524544003A200066696C616D656E745F
:1017C000007A5F6D696E00795F6D696E00785F6D9C
:1017D000696E005265706F7274696E6720656E6421
:1017E00073746F70207374617475730A0020746F62
:1017F0006F206C6F6E6720657874727573696F6E99
:101800002070726576656E7465640A0020636F6C83
:101810006420657874727573696F6E207072657676
:10182000656E7465640A00486F6D652025732573C5
:101830002573204669727374005761726E696E6712
:101840003A20486F6D696E672042756D702044695B
:101850007669736F72203C20310A00020204000096
:101860000000000000000000000000809D43000018
:101870009B430000C84300000041000000410000FD
:1018800000400000000100000001000080005555EC
:1018900055000000400033333300AAAA2A004992C1
:1018A000240000002000C7711C0099991900D1453F
:1018B0001700555515003BB11300244912001111B2
:1018C0001100000010000F0F0F00E3380E004379E5
:1018D0000D00CCCC0C00C3300C00E8A20B0064213E
:1018E0000B00AAAA0A00703D0A009DD80900427B9D
:1018F000090092240900DCD30800888808001042FF
:10190000080000000800F0C1070087870700755035
:101910000700711C07003EEB0600A1BC06006990A1
:10192000060066660600703E06006118060017F4A1
:10193000050074D105005BB00500B290050062722D
:1019400005005555050078390500B81E0500050548
:1019500005004EEC040087D40400A1BD040090A74C
:10196000040049920400C17D0400EE690400C756DA
:101970000400444404005C320400082104004110C7
:101980000400000004003FF00300F8E0030026D24A
:101990000300C3C30300CCB503003AA803000A9BAD
:1019A0000300388E0300C08103009F750300D069D7
:1019B0000300505E03001D53030034480300913DB3
:1019C00003003333030016290300381F0300971563
:1019D0000300300C0300030303000BFA020049F17B
:1019E0000200BAE802005CE002002DD802002DD00F
:1019F000020059C80200B0C0020031B90200DAB1D9
:101A00000200AAAA0200A0A30200BC9C0200FA9550
:101A100002005C8F0200DF88020082820200457CA7
:101A200002002776020027700200436A02007C64ED
:101A30000200D05E02003F590200C8530200FFFDC1
:101A4000FCFAF8F6F4F2F0EEECEAE9E7E5E3E1E0BF
:101A5000DEDCDAD9D7D5D4D2D0CFCDCBCAC8C7C572
:101A6000C3C2C0BFBDBCBAB9B7B6B4B3B2B0AFADF4
:101A7000ACAAA9A8A6A5A4A2A1A09E9D9C9A99984B
:101A80009795949392908F8E8D8B8A898887868480
:101A9000838281807F7E7D7B7A7978777675747397
:101AA0007271706F6E6D6C6B6A696867666564638E
:101AB0006261605F5E5D5C5B5A5958585756555479
:101AC00053525150504F4E4D4C4B4A4A494847464D
:101AD00046454443424241403F3E3E3D3C3B3B3A0B
:101AE00039383837363535343332323130302F2EBD
:101AF0002E2D2C2B2B2A2929282727262525242360
:101B00002322212120201F1E1E1D1C1C1B1B1A19F5
:101B1000191818171616151514131312121111107F
:101B20000F0F0E0E0D0D0C0C0B0A0A090908080701
:101B300007060605050404030302020100003D3DFB
:101B40006F6E5072696E7454696D65725374617210
:101B50007465643D3D0000809D4300009B43000090
:101B6000C8430000000000000000000000003D3DF0
:101B70006F6E53746F726553657474696E67733DED
:101B80003D003D3D6F6E436F6E66696775726174AF
:101B9000696F6E53746F72655772697474656E3DC8
:101BA0003D0053657474696E67732053746F72657A
:101BB00064000A20696E6974207A70726F62655FD2
:101BC0007A6F6666736574203D20003D3D6F6E43FD
:101BD0006F6E66696775726174696F6E53746F7248
:101BE00065526561643D3D00454550524F4D204969
:101BF0006E697469616C697A65640A003B20003A19
:101C00000A0020204D363033200020440020204D93
:101C100034313220530046696C616D656E742072F8
:101C2000756E6F75742073656E736F723A00205510
:101C3000004C0046696C616D656E74206C6F616468
:101C40002F756E6C6F6164206C656E677468733A93
:101C50000020204D3835312058005A2D50726F62C7
:101C600065204F66667365740020204D3431332043
:101C70005300506F7765722D4C6F737320526563FC
:101C80006F766572793A0020440020490020204D8B
:101C900033303420500020440020490020204D33B0
:101CA00030312050005049442073657474696E6768
:101CB000733A00204A00202047323920572049003B
:101CC00020204D3432302053004175746F2042651E
:101CD00064204C6576656C696E673A0020204D3251
:101CE0003036205800486F6D65206F6666736574E6
:101CF0003A0020580020530020204D323035204239
:101D000000416476616E6365643A20423C6D696EA1
:101D10005F7365676D656E745F74696D655F75731C
:101D20003E20533C6D696E5F6665656472617465E3
:101D30003E20543C6D696E5F74726176656C5F66BF
:101D4000656564726174653E20583C6D61785F78AA
:101D50005F6A65726B3E20593C6D61785F795F6A9E
:101D600065726B3E205A3C6D61785F7A5F6A65727E
:101D70006B3E20453C6D61785F655F6A65726B3EC6
:101D80000020540020520020204D323034205000DA
:101D9000416363656C65726174696F6E2028756E4E
:101DA0006974732F7332293A20503C7072696E74D3
:101DB0005F616363656C3E20523C7265747261635F
:101DC000745F616363656C3E20543C747261766538
:101DD0006C5F616363656C3E0020204D32303120C2
:101DE00058004D6178696D756D20416363656C6560
:101DF000726174696F6E2028756E6974732F733207
:101E0000293A0020204D3230332058004D61786946
:101E10006D756D20666565647261746573202875E3
:101E20006E6974732F73293A005374657073207050
:101E3000657220756E69743A0020440020204D328E
:101E400030302053002044697361626C65640A007D
:101E500046696C616D656E742073657474696E6734
:101E6000733A0020286D6D29002020473231202050
:101E700020203B20556E69747320696E206D6D00C3
:101E80003D3D6F6E4C6F616453657474696E67732A
:101E90003D3D000000FA430000FA430000204100ED
:101EA000008C420000A0420000A0420000C8430095
:101EB00080CF43EE020000EE020000640000003C10
:101EC00000000024F4D43050C38E20C2A2401782F8
:101ED0008B7011127A910D816CD90AA861E108C743
:101EE000586607615143061E4B5D05C145A7041A9C
:101EF000411104093D9803713931034036DB026515
:101F0000339102D4305402802E1D02632CEE0175F1
:101F10002AC501B028A001102781018F2564012B5B
:101F2000244B01E0223401AC211F018D200D0180E2
:101F30001FFC00841EED00971DDF00B81CD200E6D8
:101F40001BC600201BBC00641AB200B219A8000A0C
:101F500019A0006A189900D117910040178B00B59D
:101F600016840031167E00B31579003A157300C748
:101F7000146F0058146A00EE13660088136300257E
:101F8000135E00C7125B006C12570015125400C19B
:101F900011510070114F0021114B00D61049008DD6
:101FA0001047004610440002104200C00F4000805D
:101FB0000F3E00420F3C00060F3B00CB0E38009353
:101FC0000E37005C0E3500270E3400F30D3200C1D1
:101FD0000D3100900D3000600D2E00320D2D0005EA
:101FE0000D2C00D90C2B00AE0C2900850C29005CAF
:101FF0000C2700350C27000E0C2600E80B2400C42B
:102000000B2400A00B23007D0B23005A0B21003969
:102010000B2100180B2000F80A1F00D90A1E00BB74
:102020000A1E009D0A1D00800A1D00630A1C00474D
:102030000A1B002C0A1B00110A1A00F7091A00DDFE
:10204000091900C4091900AB091900920917007B8E
:10205000091800630917004C0916003609160020FC
:102060000916000A091500F5081500E0081400CC4F
:10207000081400B8081400A4081400900813007D88
:102080000812006B081300580812004608120034AA
:10209000081100230811001208110001081100F0B6
:1020A000071000E0071000D0071000C0071000B0B4
:1020B000070F00A107100091070E0083070F00749F
:1020C000070F0065070E0057070E0049070E003B7B
:1020D000070D002E070E0020070D0013070D000648
:1020E000070D00F9060C00ED060D00E0060C00D40B
:1020F000060C00C8060C00BC060C00B0060C00A4C0
:10210000060B0099060C008D060B0082060B00776B
:10211000060B006C060B0061060A0057060B004C0C
:10212000060A0042060A0038060A002E060A0024A3
:10213000060A001A060A001006090007060A00FD32
:10214000050900F4050900EB050900E2050900D9BD
:10215000050900D0050900C7050900BE050900B53D
:10216000050800AD050800A50509009C05080094B8
:102170000508008C050800840508007C050800742B
:102180000508006C050700650508005D0507005699
:102190000508004E05070047050700400508003800
:1021A000050700310507002A050700230507001C65
:1021B000050600160507000F0507000805060002C2
:1021C000050700FB040600F5040700EE040600E81E
:1021D000040600E2040700DB040600D5040600CF75
:1021E000040600C9040600C3040600BD040600B7C7
:1021F000040600B1040500AC040600A6040600A015
:102200000405009B04060095040500900406008A5E
:1022100004050085040500800406007A04050075A5
:10222000040500700405006B0405006604050061E8
:102230000405005C04050057040500520405004D28
:1022400004050048040500430405003E0404003A68
:1022500004050035040500300404002C04050027A3
:10226000040400230405001E0404001A04040016DC
:10227000040500110404000D040400090405000411
:1022800004040000040400FC030400F8030400F448
:10229000030400F0030400EC030400E8030400E47A
:1022A000030400E0030400DC030400D8030400D4AA
:1022B000030400D0030400CC030400C8030300C5DA
:1022C00003030024F404D9201BC40C5C0E9804C43E
:1022D000095F0265077101F405F900FB04B30048CA
:1022E000048700C10369005803550003034500BE7D
:1022F000023A008402310053022A00290225000418
:10230000022000E4011C00C8011900AF0117009869
:1023100001140084011300710110006101100051CB
:10232000010E0043010D0036010B002B010B0020B4
:10233000010B00150109000C01090003010800FB55
:10234000000800F3000800EB000700E4000600DED0
:10235000000600D8000600D2000600CC000500C729
:10236000000500C2000500BD000400B9000400B56E
:10237000000400B1000400AD000400A9000400A5A1
:10238000000300A20003009F0004009B00030098CC
:102390000003009500020093000300900003008DED
:1023A0000002008B00030088000200860002008407
:1023B000000300810002007F0002007D0002007B1C
:1023C000000200790002007700010076000200742C
:1023D00000020072000100710002006F0002006D37
:1023E0000001006C0002006A000100690002006741
:1023F0000001006600010065000100640002006247
:1024000000010061000100600001005F0002005D4A
:102410000001005C0001005B0001005A000100594E
:10242000000100580001005700010056000100554E
:10243000000100540001005300000053000100524D
:1024400000010051000100500001004F0001004E4A
:102450000000004E0001004D0001004C0001004B47
:102460000000004B0001004A000100490001004843
:10247000000000480001004700010046000000463F
:102480000001004500000045000100440001004338
:102490000000004300010042000000420001004132
:1024A00000000041000100400001003F0000003F2B
:1024B0000001003E0000003E0001003D0000003D24
:1024C0000001003C0000003C0000003C0001003B1B
:1024D0000000003B0001003A0000003A0001003912
:1024E000000000390001003800000038000000380A
:1024F0000001003700000037000100360000003600
:1025000000000036000100350000003500000035F5
:1025100000010034000000340000003400010033EA
:1025200000000033000000330001003200000032E0
:1025300000000032000100310000003100000031D5
:102540000001003000000030000000300001002FCA
:102550000000002F0000002F0000002F0001002EBF
:102560000000002E0000002E0001002D0000002DB4
:102570000000002D0000002D0001002C0000002CA8
:102580000000002C0000002C0001002B0000002B9C
:102590000000002B0000002B0001002A0000002A90
:1025A0000000002A0000002A000100290000002984
:1025B0000000002900000029000000290001002877
:1025C000000000280000002800000028000000286B
:1025D000000100270000002700000027000000275E
:1025E0000000002700010026000000260000002651
:1025F0000000002600000026000100250000002544
:102600000000002500000025000000250000002536
:102610000001002400000024000000240000002429
:10262000000000240001002300000023000000231C
:10263000000000230000002300000023000000230E
:102640000001002200000022000000220000002201
:1026500000000022000000220001002100000021F3
:1026600000000021000000210000002100000021E6
:1026700000000021000100200000002000000020D8
:1026800000000020000000200000002000000020CA
:10269000000000200001001F0000001F0000001FBC
:1026A0000000001F0000001F0000001F0000001FAE
:1026B0000001001E0000001E0000001E0000001EA1
:1026C000000000393000003325000087190000B0F9
:1026D0000F0000DB080000BD040000740200003F92
:1026E00001000020436F756E7420583A0023646522
:1026F00066696E652044454641554C545F00006252
:102700006564004B6420004B6920004B7020005032
:102710004944204175746F74756E652066696E69F1
:1027200073686564212050757420746865206C613D
:102730007374204B702C204B6920616E64204B64B5
:1027400020636F6E7374616E74732066726F6D2098
:1027500062656C6F7720696E746F20436F6E666977
:102760006775726174696F6E2E680A005049442063
:102770004175746F74756E65206661696C6564215E
:102780002074696D656F75740A0050494420417565
:10279000746F74756E65206661696C656421205480
:1027A000656D706572617475726520746F6F2068F5
:1027B0006967680A00204B643A2000204B693A2080
:1027C00000204B703A200020436C617373696320D2
:1027D000504944200A00204E6F206F76657273685E
:1027E0006F6F740A002054753A2000204B753A2010
:1027F00000206D61783A2000206D696E3A2000203B
:10280000643A200020626961733A200050494420F4
:102810004175746F74756E652073746172740A000B
:10282000504944204175746F74756E652066616906
:102830006C6564212054656D706572617475726594
:1028400020746F6F20686967680A004265640045FC
:102850003100626564002C2073797374656D207398
:10286000746F7070656421204865617465725F499A
:10287000443A200048656174696E67204661696C5E
:1028800065640048656174696E67206661696C659E
:1028900064004D3131322053687574646F776E0077
:1028A0001000C90210012C01400122017001180121
:1028B000B0010E01F00104015002FA00B002F00074
:1028C0003003E600D003DC009004D2007005C8009D
:1028D000A006BE000008B400B009AA00D00BA000FA
:1028E000600E960060118C0000158200201978009F
:1028F000C01D6E00A0226400B0275A00902C50002A
:1029000000314600E0343C0010383200903A280094
:10291000603C1E00A03D1400803E0A00203F0000E5
:10292000544845524D414C2052554E415741590053
:10293000546865726D616C2052756E6177617900C3
:102940004572723A204D415854454D50004D415802
:1029500054454D502074726967676572656400451F
:1029600072723A204D494E54454D50004D494E54D7
:10297000454D502074726967676572656400202F49
:10298000002042403A0020403A0020573A002057A9
:102990003A00496E76616C6964206578747275647A
:1029A00065720A007C3C3E5E2B3D3F2F5B5D3B2CFD
:1029B0002A225C0043616E6E6F74206F70656E201A
:1029C0007375626469722000534420496E697420F3
:1029D0004661696C0053442063617264206F6B0A26
:1029E000006F70656E526F6F74206661696C65640C
:1029F0000A00766F6C756D652E696E69742066616C
:102A0000696C65640A004E6F2053442063617264F0
:102A10000A000A4D3234004D3233202573002E0A4D
:102A2000006F70656E206661696C65642C20466974
:102A30006C653A200046696C652073656C6563744B
:102A400065640A002053697A653A200046696C651E
:102A5000206F70656E65643A2000454E44205355E2
:102A600042524F5554494E450A002220706F730060
:102A70002220706172656E743A2200535542524FA3
:102A80005554494E452043414C4C20746172676552
:102A9000743A220053756263616C6C204F766572E4
:102AA000666C6F77004578636565646564206D6169
:102AB0007820535542524F5554494E452064657015
:102AC00074683A002E0A0044656C6574696F6E2064
:102AD0006661696C65642C2046696C653A20004625
:102AE000696C652064656C657465643A00534420C4
:102AF0007072696E74696E67206279746520004E29
:102B00006F74205344207072696E74696E670A0096
:102B100057726974696E6720746F2066696C653AD4
:102B20002000667265736800646F696E67002066D6
:102B3000696C653A20004E6F7720002F6175746FC5
:102B400025632E67002020506C616E6E65724275A1
:102B50006666657242797465733A20002046726534
:102B600065204D656D6F72793A2000436F6D706915
:102B70006C65643A20417072203239203230323133
:102B80000A00204C61737420557064617465643A66
:102B900020323032312D30342D3138207C204175B7
:102BA00074686F723A20426F6E6474656368202F98
:102BB00020496E73616E6974794175746F6D6174CB
:102BC000696F6E0A00322E302E375F4457372E332E
:102BD0000A004D61726C696E0020536F66747761F4
:102BE00072652052657365740A00205761746368CA
:102BF000646F672052657365740A002042726F77B4
:102C00006E206F75742052657365740A00204578D4
:102C10007465726E616C2052657365740A00506F42
:102C200077657255700A0073746172740A004739CF
:102C3000310A47315A350A4739300A4D38340A4D7E
:102C400031303453300A4D3134305330004D31304F
:102C50003031006572726F722077726974696E67C5
:102C600020746F2066696C650A00446F6E6520737E
:102C70006176696E672066696C652E0A004D32398F
:102C800000456E6473746F707300255320256320B4
:102C9000256320256320256300205A3A0020593AF5
:102CA0000020583A00656E6473746F707320686911
:102CB000743A200000000A0B02090C0D0E080703ED
:102CC00004010000000000000000000000000000FF
:102CD00000000000000000000000000000000000F4
:102CE00012111000000000000000000000000000B1
:102CF000000000000000000000006001F40170010D
:102D0000EA019001E001B001D601D001CC0100023E
:102D1000C2013002B8016002AE019002A401D002EB
:102D20009A012003900170038601C0037C013004E6
:102D30007201A004680120055E01B005540160061F
:102D40004A0120074001F0073601F0082C01100A63
:102D50002201500B1801C00C0E01500E040130105E
:102D6000FA002012F0005014E600C016DC007019C2
:102D7000D200501CC800501FBE007022B400B02505
:102D8000AA00F028A000202C9600302F8C001032D2
:102D90008200A0347800F0366E00E0386400803A9B
:102DA0005A00403B5500E03B5000F03C4600C03D1F
:102DB0003C00603E3200E03E2800303F1E00503FA5
:102DC0001900703F1400A03F0A00C03F0000D03F30
:102DD000F6FFE03FECFFFFFFFF50726F62696E6726
:102DE000204661696C656400205A3A200020593AF7
:102DF000200042656420583A20003D3D6F6E5573B7
:102E00006572436F6E6669726D5265717569726540
:102E1000643D3D00220A00556E6B6E6F776E206335
:102E20006F6D6D616E643A202200204200205000D8
:102E30006F6B00204500205A00205900204D393288
:102E400020580020453A00205A3A0020593A0058AC
:102E50003A0020746F6F206C6F6E67206578747213
:102E60007573696F6E2070726576656E7465640A3D
:102E70000020636F6C6420657874727573696F6E7F
:102E80002070726576656E7465640A0043616E6ECB
:102E90006F7420656E746572207375626469723A2E
:102EA00020004D323520500A4D3234005265737582
:102EB0006D65005549205061757365004E6F204D5A
:102EC00061746368203A004D32320A4D323100524B
:102ED0006566726573680050675570005067446F8F
:102EE000776E0049732046696C6520004973204461
:102EF00069722000476F5570446972004861732001
:102F00004D656469610046696C656E616D6520534D
:102F1000656C6563746564004D3130303043004D3D
:102F2000313030300046696C616D656E74205374C9
:102F300061742030202D20330046696C616D656E10
:102F40007420537461742030202D20320046696C47
:102F5000616D656E7420537461742030202D2031B2
:102F6000002046696C616D656E7420526573706FE8
:102F70006E7365204E6F00526573756D65205965DF
:102F80007320647572696E67207072696E74000ACE
:102F9000204E6F2046696C616D656E7400496E76D7
:102FA000616C6964204F7074696F6E004D3530300C
:102FB0000053746F72652053657474696E67730093
:102FC0004265642050494420537461727465640002
:102FD0004D3939390A4D323830503053313630009E
:102FE000424C546F756368205265736574004D35AB
:102FF00030320A4D35303000496E697420454550F5
:10300000524F4D00486F74656E6420504944205300
:1030100074617274656400456E676C697368204101
:103020006C726561647920536574004368696E65EC
:103030007365204E6F7420537570706F7274656481
:1030400000496E4C616E6743686F696365000A20D2
:103050002A2A2A7265636461742E646174615B302C
:103060005D203D004732380A47312046313030304C
:10307000205A313000556E737570706F72746564CC
:10308000204F7074696F6E2053656C65637465645E
:103090000047323652323535004D313930533535EF
:1030A0000A4732380A4732390A4D3430300A4D3136
:1030B0003034533231350A4732380A4D31303953C2
:1030C0003231350A4D34323053310A4731583130BC
:1030D000305931303046353030300A47315A300AB5
:1030E0004D3530300A4D31313720536574205A2028
:1030F0004F666673657400473120463130303020AA
:103100005A302E30004732380A47312046313030AD
:1031100030205A302E30004D353030005A204F6666
:1031200066736574203A202573004D353030005A9F
:10313000204F6666736574203A2025730047323845
:103140000A473146313530305A302E300047323858
:103150005A0A473146313530305A302E30004D381A
:103160003400473146313030305A302E300047324B
:10317000380A473146313030305A302E30004D61F8
:103180006E75616C53657454656D70005265717530
:103190006573746564204F66667365742042657953
:1031A0006F6E64204C696D697473005A204F6666B7
:1031B000736574203A20257300526F756E64696ED2
:1031C0006720746F20737465700052657175657344
:1031D000746564204F6666736574200053746F7065
:1031E000205472696767657265640053746F70205C
:1031F0004E6F0053746F705072696E740048616E48
:10320000646C6520446174612041646A7573742044
:10321000322053657474696E672053637265656EFE
:10322000200048616E646C652044617461205072B6
:10323000696E7446696C6520332053657474696ED9
:10324000672053637265656E200048616E646C652B
:103250002044617461205072696E7446696C652007
:10326000322053657474696E672053637265656EAE
:1032700020004D38340048616E646C6520446174F0
:1032800061205072696E7446696C6520506F73746A
:103290000048616E646C65204461746120507269FD
:1032A0006E7446696C652050726500426567696E90
:1032B000537769746368003D3D20436865636B6BB9
:1032C00065793D3D007265636461742E616464726A
:1032D000203D3D007265636461742E646174615BBE
:1032E000305D203D3D0077616974776179203D3D17
:1032F0000020202A2A2A2A2A2A2A5254535F486167
:103300006E646C65446174612A2A2A2A2A2A2A2A50
:103310002000526573656E643A200000002200258B
:103320000028002B002E00310034000201000005AF
:103330000108010B0100002100240027002A002DB4
:10334000003000330001010000040107010A0105FB
:10335000050505070508080808020202020A0A080E
:103360000804040404010101010101010103030334
:103370000303030303040707070C0C0C0C0C0C0CD1
:103380000C0202020206060606060606060B0B0BD8
:103390000B0B0B0B0B010210202008081020401013
:1033A0002040800201020108040201010204081009
:1033B0002040808040201008040201800402018027
:1033C0004020100804020108040201010204081050
:1033D00020408001020408102040804444582031DD
:1033E00030532050726F2052656164792E00507204
:1033F000696E74696E672E2E2E005072696E74208D
:10340000506175736564006E6F7469666963617499
:10341000696F6E20005049442054756E65204669DE
:103420006E697368656400005401760111241FBE43
:10343000CFEFD1E2DEBFCDBF00E00CBF13E0A0E0D4
:10344000B2E0E4E0F5E502E00BBF02C007900D92A8
:10345000AE3FB107D9F725E1AEEFB3E001C01D9251
:10346000AB3DB207E1F71AE1C5E1DAE100E006C0E1
:1034700021970109802FFE010F94AF26C431D10797
:1034800080E00807A9F70F94CD140D94702A0C94CE
:1034900000009F92AF92BF92CF92DF92EF92FF9285
:1034A0000F931F93CF93DF9300D01F921F92CDB73E
:1034B000DEB7EEE3FAE10027BB27462F572FA82FF0
:1034C000AA2341F4A52F542FB85FAA2319F4A52FDE
:1034D0005527B85FA03138F45295A295452F4F700B
:1034E000507FA42BBC5FA03428F4550FAA1F550FA2
:1034F000AA1FBE5FA03818F4550FAA1FB395550F29
:10350000AA1FEA0FF01F449151E0AA27B85081F199
:10351000C8F0B0FF02C0440F551FB1FF04C0440FF4
:10352000551F440F551FB2FF06C052954295142FE8
:103530001F70407F512BB3FF1BC0A52F542F442772
:103540000C94B81AB195B0FF02C055954795B1FFDC
:1035500004C05595479555954795B2FF05C05295BE
:10356000407F4295452B5F70B3FF02C0452F552722
:10357000DD24CC24BB24B2E0649FD018C108B00A7B
:10358000B00B749FC018B108B00B849FB018B1097C
:10359000659FC018B108B00B759FB018B109859F21
:1035A000B0196A9FB018B1097A9FB0194D9DA12C2E
:1035B00099243327992722275D9DA00C911C301F49
:1035C000901F201FAD9D900C311D901F201F4C9D02
:1035D000A00C911C301F901F201F5C9D900C311D72
:1035E000901F201FAC9D300D911D201F4B9D900CF6
:1035F000311D901F201F5B9D300D911D201FAB9D25
:10360000900D211D4B9F300D911D201F5B9F900D34
:10361000211DAB9F200DB1E0BB24CC24DD24639F92
:10362000D018C108B00AB00B739FC018B108B00B16
:10363000839FB018B109699FC018B108B00B799F7A
:10364000B018B109899FB019629FB018B109729F73
:10365000B019D61AC70AB80A20F0B1E03B0F901F84
:10366000201F1124792F632F90E0822F0F900F904D
:103670000F900F900F90DF91CF911F910F91FF90BE
:10368000EF90DF90CF90BF90AF909F900895AF9252
:10369000BF92CF92DF92EF92FF920F931F93CF933F
:1036A000DF93C1E3DCE004EE18E081E4A82E8CE0B7
:1036B000B82EC12CD12C7601C3946991799189914E
:1036C00099910F94F91F288939894A895B890F9448
:1036D0005A200F942B28F801619371938193919351
:1036E0008F01C616D706E806F90610F46B017C01B7
:1036F000AC16BD0611F76FEF7FEFCB01A701960166
:103700000F9438262093F4083093F5084093F60878
:103710005093F708DF91CF911F910F91FF90EF9099
:10372000DF90CF90BF90AF900895CF92DF92EF924D
:10373000FF928091F007882309F457C0C090EC07EE
:10374000D090ED07E090EE07F090EF0720E030E03A
:10375000A901C701B6010F94F41F882309F445C0DD
:1037600020E030E040E05FE3C701B6010F945A204B
:103770009B01AC010F945A202BED3FE049E450E44B
:103780000F945A209B01AC0160E070E080E89FE359
:103790000F94B2276B017C01C092790CD0927A0C05
:1037A000E0927B0CF0927C0C609165027091660255
:1037B000072E000C880B990B0F94FB1F2AE037EDA6
:1037C00043E25CE30F945A20A70196010F945A201C
:1037D000609361027093620280936302909364022B
:1037E000FF90EF90DF90CF900895C12CD12C80E80E
:1037F000E82E8FE3F82ED0CF0F931F93CF93DF9354
:1038000050E0FC01E40FF51F8081440F551F440F69
:10381000551F46565A4FEA01882329F1888199811C
:10382000AA81BB81EB01088119812A813B81009724
:10383000A105B10569F40C591F4F2F4F3F4FDA0115
:103840000D931D932D933C9313978FEF808306C0A8
:10385000081B190B2A0B3B0B37FDF7CFDF91CF91DC
:103860001F910F910895188219821A821B82F6CF38
:10387000CF93DF9324E0829FC0011124EC01C95350
:10388000D74FFC01E350F84F8F50984FDC012D913A
:103890003D914D915C9160817181828193810F9402
:1038A000B826688379838A839B83DF91CF910895BB
:1038B0008091950590919605A0919705B0919805F6
:1038C0008093410290934202A0934302B09344023A
:1038D000809193059091940590936802809367027C
:1038E00008958091410290914202A0914302B091CB
:1038F00044028093950590939605A0939705B09305
:103900009805809167029091680290939405809346
:10391000930584E690E0909368028093670208958F
:103920008091351290913612891B877089F48091AD
:10393000890D81110DC080917D0C90917E0C892B99
:1039400039F481E09091A306911103C080E00895BD
:1039500081E00895CF93DF93DB01F9019C919130D1
:10396000C1F0943080F094509C938830D1F48081E1
:103970009181009771F0019791838083480F591FBF
:10398000EA01188206C08C3539F49C5F9C93943010
:1039900041F4DF91CF9108958B3339F781E08C9317
:1039A000F8CF20813181B9016F5F7F4F71836083D0
:1039B000420F531FEA018883808191818F359105E1
:1039C0006CF7E7CF0F931F9381E00091D91310910B
:1039D000DA132091DB133091DC134091D513509111
:1039E000D6136091D7137091D813041715072607C3
:1039F000370708F480E01F910F91089590E080E070
:103A00000895282F9091EB07833021F495FD0FC086
:103A100094FD0FC0892F90E0B0E0A0E004C0B695FF
:103A2000A795979587952A95D2F78170089581E09B
:103A3000089580E00895FC016591759185919491B8
:103A400008958F929F92AF92BF92CF92DF92EF92A2
:103A5000FF92CF93DF93EC018090C3089090C4084D
:103A6000A090C508B090C60820E030E0A901C501CB
:103A7000B4010F94F41F882309F454C0C880D9807E
:103A8000EA80FB80A7019601C501B4010F94F41FE1
:103A900018160CF04CC02091BB083091BC08409126
:103AA000BD085091BE08C701B6010F94F41F8823CA
:103AB00031F1C092BB08D092BC08E092BD08F092F0
:103AC000BE082091BF083091C0084091C1085091B4
:103AD000C208688179818A819B810F945A209B0159
:103AE000AC0160E070E080E89FE30F94B72660933C
:103AF0000F02709310028093110290931202609152
:103B00000F02709110028091110290911202DF91C8
:103B1000CF91FF90EF90DF90CF90BF90AF909F90AC
:103B20008F90089560E070E080E89FE3F0CF60E060
:103B300070E0CB01ECCFCF92DF92EF92FF92CF9368
:103B4000DF93EC01CC80DD80EE80FF8027E137EB56
:103B500041ED58EBC701B6010F94182987FD23C02A
:103B600023E030E04BE953E4C701B6010F94F41FA2
:103B70001816CCF0C880D980EA80FB8027E137EBAB
:103B800041ED58EBC701B6010F94182987FD0BC012
:103B9000C1E023E030E84DE953E4C701B6010F94DA
:103BA000F41F18160CF4C0E08C2FDF91CF91FF901A
:103BB000EF90DF90CF9008952FEB280F2A3108F077
:103BC00047C0E22FF0E08091320590913305A0913B
:103BD0003405B091350504C0B695A795979587959E
:103BE0002A95D2F780FD02C081700895EC5EFA4FED
:103BF000E081EE2341F18091810790918207E80FE7
:103C0000F92FF11D808190ED980F9A3030F08E32AF
:103C100051F4818180538A3098F4F0930305E09346
:103C2000020581E008958D3211F08B3249F48181D3
:103C300090ED980F9A3088F38E3211F48281EACF9A
:103C4000F0E0E0E0EACF1092030510920205E9CF20
:103C500080E008950E94DC1D882341F081E02091DE
:103C6000020530910305232B09F480E008958F921B
:103C70009F92AF92BF92CF92DF92EF92FF92C0904D
:103C8000D105D090D205E090D305F090D40520E086
:103C900030E0A901C701B6010F94F41F8823E1F1B8
:103CA000A701960160E070E080E89FE30F94B227DF
:103CB0006B017C018090D5059090D605A090D7052A
:103CC000B090D80520E030E0A901C501B4010F94FF
:103CD000F41F882329F1A501940160E070E080E8D9
:103CE0009FE30F94B227C092D804D092D904E092F7
:103CF000DA04F092DB046093DC047093DD048093BB
:103D0000DE049093DF04FF90EF90DF90CF90BF90A0
:103D1000AF909F908F900895C12CD12C7601CACF7F
:103D200060E070E0CB01DFCF129A08955F9A809136
:103D30002F0C8E7F80932F0C8A9A80912F0C8D7F71
:103D400080932F0C809108018095817080930601EB
:103D500080912F0C8B7F80932F0C0C94941E269AAD
:103D60002E9A0895833B21E0920714F083EB91E0B3
:103D70009093E6118093E5110C94AAEDEDE0F6E046
:103D8000108211821282138214820C94AAED4F9237
:103D90005F926F927F928F929F92AF92BF92CF92DB
:103DA000DF92EF92FF920F931F93CF93DF93EC017B
:103DB0002091C9053091CA054091CB055091CC05A1
:103DC000688179818A819B810F94B7266B017C0180
:103DD0002091CD053091CE054091CF055091D00571
:103DE0006C817D818E819F810F94B7264B015C0190
:103DF000A70196016091030270910402809105026F
:103E0000909106020F94F41F882309F450C0C092C9
:103E10000302D0920402E0920502F0920602209181
:103E2000D8043091D9044091DA045091DB04C701E1
:103E3000B6010F945A202B013C010F945A286B01B4
:103E40007C0120E030E0A9010F94F41F87FD70C0D1
:103E500020E030E040E450E4C701B6010F94182997
:103E600018162CF4C12CD12CC0E4EC2EFE2CA7018A
:103E70009601C301B2010F94B7266093D0047093EA
:103E8000D1048093D2049093D304C701B6010F9458
:103E900024286093CE04062E000C770B6F5F7F4FB3
:103EA0006430710514F064E070E06093CC04D0914C
:103EB00001021091CE04A501940160910702709156
:103EC00008028091090290910A020F94F41F811157
:103ED00033C0D11381C02091B4043091B504409116
:103EE000B6045091B7046091D0047091D1048091D0
:103EF000D2049091D3040F945A202091B8043091A9
:103F0000B9044091BA045091BB040F94B826DF91D4
:103F1000CF911F910F91FF90EF90DF90CF90BF90C6
:103F2000AF909F908F907F906F905F904F9008958B
:103F3000C12CD12C76019BCF80920702909208026F
:103F4000A0920902B0920A022091DC043091DD04B3
:103F50004091DE045091DF04C501B4010F945A2052
:103F60004B015C010F945A286B017C0120E030E08A
:103F7000A9010F94F41F87FDF3C020E030E040E476
:103F800050E4C701B6010F94182918162CF4C12C5F
:103F9000D12CB0E4EB2EFE2CA7019601C501B40193
:103FA0000F94B7266093D4047093D5048093D604FD
:103FB0009093D704C701B6010F9424286093CF04CF
:103FC000062E000C770B6F5F7F4F6430710514F085
:103FD00064E070E06093CD04C091CF04D11305C0BC
:103FE000809102028C1709F470C08091CE049091E8
:103FF000CF0490930202809301020C2E000CDD0B83
:1040000025E01203C0011124FC01EC0FFD1FEE0F8F
:10401000FF1FEE0FFF1FE957F84F208131814281CA
:1040200053812093C8043093C9044093CA04509329
:10403000CB040091CD04002E000C110BFC01E00F0D
:10404000F11FEE0FFF1FEE0FFF1FE957F84F6081C2
:104050007181828193810F94B7266093C404709319
:10406000C5048093C6049093C7042091CC0435E026
:104070002303F0011124CE0FDF1FCC0FDD1FCC0F67
:10408000DD1FC957D84F288139814A815B81209330
:10409000C0043093C1044093C2045093C304E00FA2
:1040A000F11FEE0FFF1FEE0FFF1FE957F84F608162
:1040B0007181828193810F94B7266093BC047093C1
:1040C000BD048093BE049093BF048090D40490906C
:1040D000D504A090D604B090D7042091C4043091A8
:1040E000C5044091C6045091C704C501B4010F94A2
:1040F0005A202091C8043091C9044091CA045091BB
:10410000CB040F94B8266B017C01C092B804D09206
:10411000B904E092BA04F092BB042091BC0430913F
:10412000BD044091BE045091BF04C501B4010F9479
:104130005A202091C0043091C1044091C204509192
:10414000C3040F94B826A70196010F94B726609375
:10415000B4047093B5048093B6049093B704BBCEB7
:10416000C12CD12C760118CFCF92DF92EF92FF9223
:10417000CF93DF93EC0108960E94211D6B017C0117
:1041800020E030E0A9010F94F41F20E030E0A90105
:10419000882359F0CE010E94C71E9B01AC01C701C4
:1041A000B6010F945A209B01AC01688579858A85F8
:1041B0009B850F94B726688779878A879B87DF91CD
:1041C000CF91FF90EF90DF90CF9008952F923F9284
:1041D0004F925F926F927F928F929F92AF92BF9217
:1041E000CF92DF92EF92FF920F931F93CF93DF93C3
:1041F000D62FC72FFC0180809180A280B380C5019B
:10420000B40120E831E541E050E00F943826C901BF
:104210006DE671E00F949B266B017C01C501B40132
:1042200020E13EE040E050E00F943826CA01B90199
:1042300028E130E040E050E00F943826362E272E5B
:10424000062F172F8CE3482E512C612C712CC501A1
:10425000B401A30192010F943826B62EA72ECA01ED
:10426000B901A30192010F943826CB01C114D104E6
:1042700079F1AF92BF927F936F932F923F92FF920B
:10428000EF92DF92CF9288E496E19F938F93CF9342
:10429000DF930F948B1F8DB79EB70E960FB6F894D1
:1042A0009EBF0FBE8DBF8D2F9C2FDF91CF911F9191
:1042B0000F91FF90EF90DF90CF90BF90AF909F90C5
:1042C0008F907F906F905F904F903F902F900895C8
:1042D000E114F104C9F0AF92BF927F936F932F92D4
:1042E0003F92FF92EF9288E396E19F938F93CF9353
:1042F000DF930F948B1FEDB7FEB73C960FB6F89483
:10430000FEBF0FBEEDBFCFCF012BB9F0AF92BF9272
:104310007F936F932F923F928CE296E19F938F93BE
:10432000CF93DF930F948B1F8DB79EB70A960FB66E
:10433000F8949EBF0FBE8DBFB6CF892BA9F0AF9268
:10434000BF927F936F9384E296E19F938F93CF9375
:10435000DF930F948B1FEDB7FEB738960FB6F89426
:10436000FEBF0FBEEDBF9FCFAF92BF9280E296E13E
:104370009F938F93CF93DF930F948B1F0F900F908A
:104380000F900F900F900F908ECFEF92FF920F93A0
:104390001F93CF93DF93CDB7DEB78C01EDB6FEB69A
:1043A0000F94411F01962DB73EB7281B390B0FB64E
:1043B000F8943EBF0FBE2DBF8DB79EB70196B801D2
:1043C0000F943A1F0F9405110FB6F894FEBE0FBE5E
:1043D000EDBEDF91CF911F910F91FF90EF90089567
:1043E0008C38910514F08CE890E090937B118093C9
:1043F0007A110C94A4BAAB01BC014093D913509329
:10440000DA136093DB137093DC1381E495E10C9471
:104410005CAB2F923F924F925F926F927F928F92FE
:104420009F92AF92BF92CF92DF92EF92FF920F9343
:104430001F93CF93DF93CDB7DEB760970FB6F89495
:10444000DEBF0FBECDBF8B876C87042F122F282FA6
:1044500030E03E872D87462F50E05A87498785E018
:10446000982E929EC001939E900D1124988B8F8759
:10447000FA01E80FF91FEE0FFF1FEE0FFF1FE957BC
:10448000F84F60817181828193819B01AC010F940F
:10449000AA29882309F445C14B85400F6C85610F1B
:1044A000949EC0011124E985FA85E80FF91FEE0FEB
:1044B000FF1FEE0FFF1FE957F84FC080D180E28049
:1044C000F380040F909EA0011124E985FA85E40F82
:1044D000F51FEE0FFF1FEE0FFF1FE957F84F00818A
:1044E000918082807380262F30E0EF85F889E20F7B
:1044F000F31FEE0FFF1FEE0FFF1FE957F84F20804D
:104500007181798372817A8373817B83610F70E01B
:10451000EF85F889E60FF71FEE0FFF1FEE0FFF1F65
:10452000E957F84FF88BEF87F081FC83EF85F88926
:10453000F181FD83EF85F889F281FE83EF85F889AB
:10454000F381FF83FC01E20FF31FEE0FFF1FEE0F5D
:10455000FF1FE957F84F20812887A180B280638030
:10456000FA01E60FF71FEE0FFF1FEE0FFF1FE957CF
:10457000F84F4080518032801381202F392D482DF3
:10458000572D602F792D882D972D0F94AA298823D8
:1045900021F000E0912C812C712C9601A701B6012D
:1045A000C7010F94AA29882321F0C02ED92CE82C0A
:1045B000F72C2C813D814E815F816C817D818E81C4
:1045C0009F810F94AA29882321F01C821D821E82BC
:1045D0001F82222D39814A815B81622D79818A81F6
:1045E0009B810F94AA29882339F02C803D8139833F
:1045F0004E814A835F815B839201432D512FB2012B
:10460000832D912F0F94AA29882321F0412C512C1E
:10461000312C10E028853A2D4B2D562D68857A2DAA
:104620008B2D962D0F94AA29882321F04886A52C3E
:10463000B32C612E85E02D853E85829FF001839FFE
:10464000F00D112449855A85E40FF51FEE0FFF1F69
:10465000EE0FFF1FE957F84FFA87E9879601A70188
:10466000B601C7010F94B826202F392D482D572D9C
:104670000F94B7266B017C01222D39814A815B8121
:10468000622D79818A819B810F94B8262C813D818E
:104690004E815F810F94B7269B01AC01C701B60123
:1046A0000F94B8266B017C0128853A2D4B2D562D91
:1046B00068857A2D8B2D962D0F94B8269201432D67
:1046C000512F0F94B7269B01AC01C701B6010F947F
:1046D000B82620E030E040E450E40F94B227E985AA
:1046E000FA8560837183828393836C858B85609662
:1046F0000FB6F894DEBF0FBECDBFDF91CF911F91F3
:104700000F91FF90EF90DF90CF90BF90AF909F9070
:104710008F907F906F905F904F903F902F900D946F
:10472000630F60960FB6F894DEBF0FBECDBFDF916A
:10473000CF911F910F91FF90EF90DF90CF90BF909E
:10474000AF909F908F907F906F905F904F903F9031
:104750002F9008958091020590910305009731F004
:104760004AE050E070E060E00D940F1E60E070E001
:10477000CB0108958091020590910305009731F0D7
:104780004AE050E070E060E00D94E11C60E070E011
:10479000CB010895CF93DF93EB010E942A1E88235B
:1047A00019F00E94BA23EB01CE01DF91CF91089559
:1047B0000E94BA2397FD0CC00E94BA236F3F710577
:1047C0008105910509F034F40E94BA23862F0895DB
:1047D00080E008958FEF0895CF93C62F0E942A1E80
:1047E000882319F0CF910C94D8238C2FCF91089562
:1047F0008091020590910305892B41F00E94D823F6
:1048000091E0811101C090E0892F089591E0FCCFE3
:10481000CF93DF93C82FD62F0E942A1E882321F022
:10482000DF91CF910C94F8238C2F0E94DC1D811115
:1048300001C08D2FDF91CF9108950E94BA23CB0143
:104840000895CF93DF93EB010E942A1E882321F065
:10485000DF91CF910C941D24CE01DF91CF9108956B
:104860000F931F93CF9380910205909103050097BA
:10487000E9F0FC018F01C1912C2F2F7D81F0C5340F
:1048800011F0C536B9F7F801108270E060E00F94BE
:10489000831BF801C083CF911F910F91089570E0A1
:1048A00060E0CF911F910F910D94831B60E070E049
:1048B000CB01F1CFCF92DF92EF92FF926A017B01A1
:1048C0000E942A1E882331F0FF90EF90DF90CF9056
:1048D0000C943024C701B601FF90EF90DF90CF9089
:1048E00008954F925F926F927F928F929F92AF92B4
:1048F000BF92CF92DF92EF92FF921F93CF93DF93FD
:1049000000D01F92CDB7DEB719821A821B821C829B
:10491000CE0101964C018EE6C82E87E0D82E9FE18D
:10492000E92E9CE0F92E27ECA22E28E0B22E10E012
:1049300088E5810F0E942A1EF40181934F0188238C
:1049400009F4E0C00E9430242B013C01812F0E9419
:10495000011D882309F4CCC0F701208131814281F7
:104960005381C301B2010F94B826F60160837183AD
:10497000828393831F5FF4E0CF0ED11C84E0E80EA6
:10498000F11C94E0A90EB11C133091F685E40E944D
:104990002A1E8C83882309F4C0C00E9430246B0136
:1049A0007C0183E00E94011D882371F020912B0C73
:1049B00030912C0C40912D0C50912E0CC701B6015A
:1049C0000F94B8266B017C01C0927A07D0927B07C6
:1049D000E0927C07F0927D078091C805882359F109
:1049E0008091DD1382FF27C08C81882321F189818A
:1049F000811103C08A818823F1F02DEC3CEC4CE45A
:104A00005DE36091120870911308809114089091F1
:104A100015080F94B8269B01AC016091270C70918A
:104A2000280C8091290C90912A0C0F9418291816A3
:104A300014F40F94A90E40E050E0BA0186E40E94FD
:104A40005A2420E030E0A9010F941829181684F4A4
:104A50000E94302420E030E040E752E40F94B22777
:104A60006093410270934202809343029093440208
:104A70008091DD0B83FD28C080918E06882321F173
:104A800020912B0C30912C0C40912D0C50912E0C20
:104A900060917A0770917B0780917C0790917D07E8
:104AA0000F94B72620919B0630919C0640919D065D
:104AB00050919E060F94B82660939B0670939C06B7
:104AC00080939D0690939E060F900F900F900F90ED
:104AD000DF91CF911F91FF90EF90DF90CF90BF902B
:104AE000AF909F908F907F906F905F904F900895C0
:104AF000F5012081318142815381C301B2010F94BC
:104B0000B72633CFF70180819181A281B381F6016D
:104B100080839183A283B3832DCF80912B0C9091BE
:104B20002C0CA0912D0CB0912E0C80937A079093B1
:104B30007B07A0937C07B0937D074ECFCF92DF9287
:104B4000EF92FF926B017C0183E3C816D104E1046C
:104B5000F10470F082E3C81AD108E108F10862E3B9
:104B600070E080E090E00E94DDA20E941EBEECCFCB
:104B7000C701B6010E94DDA2FF90EF90DF90CF90B9
:104B80000C941EBE0F931F93CF93DF9305E41CE09C
:104B9000CEE5D1E1F80121913191419151918F01FF
:104BA00060E070E080E89FE30F94B2276993799307
:104BB00089939993F1E1CE36DF0761F70F94E80C02
:104BC000DF91CF911F910F910C94471BCF92DF92F1
:104BD000EF92FF92CF93DF932091300C222329F1A3
:104BE000EC0108960E94211D6B017C0120E030E061
:104BF000A9010F94F41F20E030E0A901882359F0A7
:104C0000CE010E94C71E9B01AC01C701B6010F94E3
:104C10005A209B01AC01688579858A859B850F9414
:104C2000B826688779878A879B87DF91CF91FF9025
:104C3000EF90DF90CF9008952F923F924F925F9226
:104C40006F927F928F929F92AF92BF92CF92DF929C
:104C5000EF92FF920F931F93CF93DF93CDB7DEB701
:104C60006C970FB6F894DEBF0FBECDBF8C015B0111
:104C70005A834983FC01EA5BFF4F208131814281E5
:104C8000538129873A874B875C87CA01B9010F9402
:104C9000F91F6B017C01D5012D913D914D915C91E6
:104CA0000F945A200F9496272B013C01E981FA8139
:104CB0002081318142815381C701B6010F945A206E
:104CC0000F9496274B015C01C301B2010F942B286E
:104CD000698B7A8B8B8B9C8B68377105810591056D
:104CE00040F428E730E040E050E0298B3A8B4B8BD2
:104CF0005C8BC501B4010F942B286D877E878F874D
:104D0000988B683771058105910540F448E750E0BC
:104D100060E070E04D875E876F87788BF801EE5A10
:104D2000FF4F4080518062807380C301B2010F94B5
:104D3000FB1F69837A838B839C8369897A898B893A
:104D40009C890F94F91F6D8B7E8B8F8B988F20E041
:104D500030E0A90169817A818B819C810F94F41FD5
:104D6000882309F4E1C1A7019601C701B6010F9498
:104D70005A204B015C012D893E894F89588DCA010B
:104D8000B9010F945A209B01AC01C501B4010F94E5
:104D9000B7264B015C0129813A814B815C81CA01B4
:104DA000B9010F94B8269B01AC01C501B4010F9461
:104DB000B2270F9496270F942B286D837E838F83C1
:104DC000988766277727CB016419750986099709A3
:104DD0000F94FB1F4B015C016D857E858F85988943
:104DE0000F94F91F2B013C0120E030E0A901C5011F
:104DF000B4010F94F41F882309F49AC1A30192010E
:104E0000C301B2010F945A20698F7A8F8B8F9C8FC8
:104E1000A7019601C701B6010F945A209B01AC016E
:104E2000698D7A8D8B8D9C8D0F94B7266B017C01DB
:104E3000A5019401C501B4010F94B8269B01AC01F2
:104E4000C701B6010F94B2270F945A28D80195963E
:104E50008D909D90AD90BC909897750164012D81C7
:104E60003E814F815885C21AD30AE40AF50A0F948D
:104E70002B28C61AD70AE80AF90AF7FE8EC02D8930
:104E80003E894F89588DCA01B9010F945A206B0190
:104E90007C0129813A814B815C81CA01B9010F945F
:104EA000B82669877A878B879C8720E030E0A90144
:104EB00069817A818B819C810F94F41F882309F486
:104EC0003BC1C501B4010F94F91F29853A854B8573
:104ED0005C850F945A20A70196010F94B7266D8325
:104EE0007E838F839887A3019201C301B2010F943F
:104EF0005A209B01AC016D817E818F8198850F9432
:104F0000B8262B013C0120E030E040E850E4698104
:104F10007A818B819C810F945A209B01AC01C30143
:104F2000B2010F94B2270F9496272B013C0120E089
:104F300030E0A9010F94182918161CF0412C512CAF
:104F40003201C301B2010F942B286D837E838F83BE
:104F5000988786169706A806B90620F48D829E8249
:104F6000AF82B8866D817E818F8198850F94F91FFD
:104F700029853A854B855C850F945A20A7019601B7
:104F80000F94B8260F9466290F942B2869877A8787
:104F90008B879C87C12CD12C760169857A858B857E
:104FA0009C8529893A894B895C89621B730B840B28
:104FB000950B0F94F91F29813A814B815C810F94E5
:104FC000B22720E034E244EF59E40F945A200F94C2
:104FD0002B284B015C0169857A858B859C852D8505
:104FE0003E854F855889621B730B840B950B0F947C
:104FF000F91F29813A814B815C810F94B22720E00F
:1050000034E244EF59E40F945A200F942B282B01DB
:105010003C013FE683169104A104B10408F090C05E
:10502000F401EE0FFF1FEE0FFF1FEE57F74E8591B5
:105030009591A591B4918983292E3A2EBD8B4FE687
:10504000441651046104710408F083C0F201EE0FAC
:10505000FF1FEE0FFF1FEE57F74E459155916591DB
:1050600074919A01CB014D815E816F817885D80161
:1050700099964D935D936D937C939C974C0D5D1D1C
:105080006E1D7F1DF80145A756A767A770ABE65BAD
:10509000FF4F49895A896B897C8940835183628398
:1050A0007383D5968D929D92AD92BC92D897F8015C
:1050B00041AE52AE63AE74AEFD964981408321820B
:1050C00032825D8953833496208331838283938334
:1050D00069857A858B859C85D1966D937D938D931B
:1050E0009C93D4973D962D853E854F855889208386
:1050F0003183428353836C960FB6F894DEBF0FBEA4
:10510000CDBFDF91CF911F910F91FF90EF90DF9076
:10511000CF90BF90AF909F908F907F906F905F9057
:105120004F903F902F90089560E070E0CB0141CE0A
:1051300060E070E0CB0188CE60E070E0CB01F3CEA0
:10514000C501B4010E94491A6983272E382E9D8B10
:1051500076CFC301B2010E94491A9B0184CF80918E
:10516000351290913612891B877019F490E080E017
:10517000089590913212992351F0833030F48FEFDB
:10518000890F19F080933212F1CF10923212809170
:1051900036122CE5829FC00111248350974FFC01E9
:1051A000208120FDE3CF209136122F5F27702093BE
:1051B00033123091361220913412321304C02091F0
:1051C000331220933412089590916F0081E091FD85
:1051D00002C080E0089590916F009D7F90936F00D2
:1051E000089580FF04C09091990590FD8E7F81FF06
:1051F00005C090919905969590FD8D7F82FF06C020
:10520000909199059695969590FD8B7F08958F9234
:105210009F92AF92BF92CF92DF92EF92FF92CF9385
:10522000DF9320914502222309F49EC0EC01809176
:105230009905C82ED12CF12CE12C80FF2CC0809038
:10524000470290904802A0904902B0904A022881FB
:1052500039814A815B81C501B4010F941829181660
:1052600024F488829982AA82BB8280905302909013
:105270005402A0905502B0905602288139814A818B
:105280005B81C501B4010F94F41F87FF04C08882BD
:105290009982AA82BB82D701C601B695A795979538
:1052A000879580FF2CC080904B0290904C02A0907C
:1052B0004D02B0904E022C813D814E815F81C5012F
:1052C000B4010F941829181624F48C829D82AE82A2
:1052D000BF828090570290905802A0905902B090DF
:1052E0005A022C813D814E815F81C501B4010F942A
:1052F000F41F87FF04C08C829D82AE82BF8282E051
:10530000F694E794D794C7948A95D1F7C0FE2CC041
:10531000C0904F02D0905002E0905102F0905202A3
:10532000288539854A855B85C701B6010F94182900
:10533000181624F4C886D986EA86FB86C0905B02DC
:10534000D0905C02E0905D02F0905E022885398585
:105350004A855B85C701B6010F94F41F87FF04C01F
:10536000C886D986EA86FB86DF91CF91FF90EF90C1
:10537000DF90CF90BF90AF909F908F900895CF9285
:10538000DF92EF92FF920F931F93C12CD12C7601E5
:105390008C012BE23CE047E25CE063E27CE08FE1E1
:1053A0009CE00E940DF51F910F91FF90EF90DF9010
:1053B000CF9008950D94E80C8091A006811105C04E
:1053C00080917F07882309F463C080918605659BDF
:1053D00059C0816080938605909103018091860574
:1053E00091FF52C0826080938605809186054B9B19
:1053F0004DC08460809386058091ED0580FF10C0CC
:105400008091A10680FF0CC08091860580FF08C0B6
:1054100080917E07816080937E0780E00E94A8C60D
:105420008091ED05869580FF11C08091A10686953B
:1054300080FF0CC08091860581FF08C080917E07A7
:10544000826080937E0781E00E94A8C68091ED056E
:105450008695869580FF1CC08091A10686958695CD
:1054600080FF16C080917F07882391F08091860588
:1054700082FF0EC080917E07846080937E0782E069
:105480000C94A8C68E7FA6CF8D7FADCF8B7FB2CF79
:1054900008958091A006811104C080917F07882320
:1054A00031F062E070E080E090E00C949E25089579
:1054B0000F931F9380911C11813019F50E9410A346
:1054C0000091A2051091A3052091A4053091A50596
:1054D000601B710B820B930B28EE33E040E050E031
:1054E0000F9438266091A6057091A7058091A805B4
:1054F0009091A905620F731F841F951F1F910F9133
:1055000008956091AA057091AB058091AC059091CA
:10551000AD05D6CF10921C111092A2051092A305D2
:105520001092A4051092A5051092AA051092AB0541
:105530001092AC051092AD051092A6051092A70529
:105540001092A8051092A9050895CF92DF92EF92CC
:10555000FF92CF93DF93C62FFC01C080D180E28001
:10556000F38020E030E0A901C701B6010F94F41FD9
:1055700020E030E0A90187FD14C020E030E048ECD5
:1055800052E4C701B6010F94182924E630E040E048
:1055900050E0181634F0C701B6010F9424289B017F
:1055A000AC01C230A0F4D0E0C850D74FAFEFB0E0AC
:1055B0000F94792624E630E040E050E00F945A261C
:1055C0002F3F310519F010F02FEF30E02883DF91E5
:1055D000CF91FF90EF90DF90CF90089580910901D7
:1055E00080FD06C08091DD1383FB882780F9089534
:1055F00080E00895CF92DF92EF92FF92FC01C0808D
:10560000D180E280F380663019F510921206109274
:1056100013061092140610921506109216060E9498
:10562000A4BA20E030E0A901C701B6010F94F41F2D
:1056300087FF1DC0C12CD12C7601C701B6010F9484
:105640002529CB01FF90EF90DF90CF900C94F021B3
:105650000E94BE1E20E030E0A901C701B6010F94F0
:10566000F41F87FF15C0C12CD12C760122C020E089
:1056700030E04CE053E4C701B6010F941829181626
:10568000E4F6C12CD12C9CE0E92E93E4F92ED5CF81
:1056900020E030E849ED53E4C701B6010F94182922
:1056A00018163CF4C12C80E8D82E89EDE82E83E44E
:1056B000F82EC701B6010F942529CB01FF90EF907A
:1056C000DF90CF900C94B21E90912F0C977081E0D8
:1056D000973009F080E008952091840520FF14C0E0
:1056E00020E83EE3629FA001639F500D729F500D22
:1056F0001124CA019695879596958795009731F064
:105700008A950000E9F708950C949E250895CF939B
:10571000DF931092DE0B10927F0C1092810C10928E
:10572000800C1092830510928205CFEFDFEF8091FD
:10573000DD1385FD07C00E94BDA6D0935C12C09307
:105740005B12F5CF8FEF9FEF90935C1280935B120B
:10575000DF91CF9108958F929F92AF92BF92CF9297
:10576000DF92EF92FF920F931F93CF93DF931092EC
:105770003705109236052FE320933105109230053E
:1057800010922F0510922E051092320510923305BB
:1057900010923405109235059C01F90190812F5F1C
:1057A0003F4F9032D1F39E34C9F4818190ED980F30
:1057B0009A3020F08D3211F08B3281F432969F01B5
:1057C0002F5F3F4F808180538A3008F47BC09F0158
:1057D0002F5F3F4F8081803209F476C0F0938207BB
:1057E000E09381078F010F5F1F4FC0816AE270E075
:1057F000C8010F94062A009731F0FC01319780818F
:105800008032E1F31182CD3429F0C43519F0C73468
:1058100009F04BC0F80180810F5F1F4F8032D1F338
:1058200080538A3008F041C0C093310530E020E059
:105830004AE0DF011196429FC001439F900D112461
:105840009C01205331098081280F311D87FD3A9535
:10585000818190ED980F9A30C8F1309330052093F4
:105860002F058E3261F4329690E04AE0DF013196E6
:105870008C9150ED580F5A3058F190932E05CD0170
:10588000DC0101964C914032D9F3CD3489F52E31AB
:10589000310539F018F52731310519F02C31310572
:1058A00039F5B0933705A0933605DF91CF911F915D
:1058B0000F91FF90EF90DF90CF90BF90AF909F90AF
:1058C0008F900895F9017BCFF90181CFFD01B1CF10
:1058D000949F800D112490ED980FC8CF2537310586
:1058E00038F027373105E8F2203A83E03807C9F26B
:1058F000D091810740E050E0BA0110E000E0C12CF7
:10590000D12C7601C394FD0131968C91882309F442
:105910007FC08132E1F4CD34D1F420323105B9F4C5
:1059200040933205509333056093340570933505E9
:10593000F0933705E093360563E270E0CF010F94F2
:10594000062A009709F4B1CFFC011082AECF815432
:105950008A3108F058C0DF019D91903291F0A0ED9E
:10596000A90FAA30E8F09E3271F4918190539A30D9
:10597000B8F00115110519F48F010150110990E0DB
:1059800013C0FD01E8CF9D3211F09B3291F7918158
:10599000A0EDA90FAA3020F09E3259F79281E6CFF0
:1059A0009E2F9D1B309759F3A82FB0E04601570159
:1059B00004C0880C991CAA1CBB1C8A95D2F74829E4
:1059C00059296A297B29AC5EBA4F9C938081815406
:1059D000DF018A3108F497CFDF018191882309F430
:1059E00092CF90ED980F9A30B8F393ED980F9230D4
:1059F00098F38B3289F3CD010196EC91E03209F0F6
:105A000082CFDC01F8CF0115110501F78D01DECF42
:105A100010933705009336054093320550933305B4
:105A2000609334057093350540CF4F925F926F922B
:105A30007F928F929F92AF92BF92CF92DF92EF921E
:105A4000FF92CF93DF9300D000D01F921F92CDB76B
:105A5000DEB75C01DB01CD90DD90ED90FC90E09134
:105A60003012F0913112FE83ED8384819581A681FD
:105A7000B78189839A83AB83BC839C01AD01C70145
:105A8000B6010F94B7262B013C01F501808091806F
:105A9000A280B380AD81BE818D919D910D90BC910E
:105AA000A02D8D839E83AF83B88727E137EB41ED2F
:105AB00058EBC301B2010F94182987FDD1C023E030
:105AC00030E04BE953E4C301B2010F94F41F181600
:105AD0000CF4C6C02D813E814F815885C501B401AB
:105AE0000F94B7262B013C0127E137EB41ED58EB32
:105AF0000F94182987FDB4C023E030E84DE953E442
:105B0000C301B2010F94F41F18160CF4A9C020E0D1
:105B100030E0A9016D817E818F8198850F94B82630
:105B20002B013C0120E030E040E251E40F94F41FEF
:105B300087FF06C0412C512C30E2632E31E4732ED6
:105B400027E137EB41ED58E3C301B2010F94B726CB
:105B50009B01AC01C501B4010F94182987FD80C0D9
:105B600020E030E84DE953E46D817E818F81988596
:105B70000F94B8262B013C0120E030E041E953E4CA
:105B80000F941829181634F4412C512C21E9622E57
:105B900023E4722E27E137EB41ED58E3C301B20154
:105BA0000F94B8269B01AC01C501B4010F94F41FFA
:105BB00018160CF455C020E030E0A90169817A8103
:105BC0008B819C810F94B8264B015C0120E030E072
:105BD00040EA51E40F94F41F87FF06C0812C912CFA
:105BE00090EAA92E91E4B92E27E137EB41ED58E375
:105BF000C501B4010F94B7269B01AC01C701B601E2
:105C00000F94182987FD2CC020E030E04BE953E4C5
:105C100069817A818B819C810F94B8264B015C014C
:105C200020E030E04CE853E40F941829181634F4BF
:105C3000812C912C8CE8A82E83E4B82E27E137EB39
:105C400041ED58E3C501B4010F94B8269B01AC01A6
:105C5000B1E0B983C701B6010F94F41F18160CF414
:105C60001982898128960FB6F894DEBF0FBECDBF8A
:105C7000DF91CF91FF90EF90DF90CF90BF90AF90EA
:105C80009F908F907F906F905F904F900895E9E084
:105C9000F8E082EBDF011D928A95E9F70895809183
:105CA000C805811104C00E94472E0C941EB4809137
:105CB000DD1382FD0D94A90E0895809109088823B3
:105CC00061F09091BA08891308C08091DD1383FFB9
:105CD00004C087E498E00C94E8B280E00895FC01E9
:105CE000238121110C941DAF0895EFE6F0E080812F
:105CF000826080830895CF92DF92EF92FF92CF93DC
:105D0000DF93C82F0E94E42894E0C99FE00111248A
:105D1000FE01E550FA4FC080D180E280F38081110E
:105D20000E94752EC25ADE4EC701B6010F94FB1FAA
:105D3000288139814A815B810F945A20DF91CF916C
:105D4000FF90EF90DF90CF9008958F929F92AF9247
:105D5000BF92CF92DF92EF92FF921F93CF93DF9388
:105D6000CDB7DEB760970FB6F894DEBF0FBECDBFDC
:105D7000182F80E00E947B2E4B015C0180928705EA
:105D800090928805A0928905B0928A0581E00E94D0
:105D90007B2E6B017C01C0928B05D0928C05E0922A
:105DA0008D05F0928E0582E00E947B2E60938F0518
:105DB0007093900580939105909392051D861E86A1
:105DC0001F86188A89829A82AB82BC82CD82DE824B
:105DD000EF82F88669877A878B879C8783E00E94A9
:105DE0007B2E6D877E878F87988B8091300C8823E0
:105DF00021F0CE0101960E94B4201E3FD9F480E12B
:105E0000FE013196AFE1BCE001900D928A95E1F779
:105E100060960FB6F894DEBF0FBECDBFDF91CF9175
:105E20001F91FF90EF90DF90CF90BF90AF909F9029
:105E30008F90089584E0189FF0011124DF01A15E86
:105E4000B34F81E090E08C0F9D1FE80FF91F408158
:105E50005181628173814D935D936D937C93139710
:105E6000D7CFCF92DF92EF92FF92CF93DF93C82FDD
:105E70000E94E42894E0C99FE0011124FE01E15151
:105E8000FA4FC080D180E280F38081110E94752E8C
:105E9000C25ADE4EC701B6010F94FB1F288139811B
:105EA0004A815B810F945A20DF91CF91FF90EF9050
:105EB000DF90CF9008950E94E4289091361290933D
:105EC0003512909334129093331294E690933212D9
:105ED00020ED33E03093FC082093FB0881110E94F1
:105EE000752E81E08093EE050895CF93DF93CDB7B3
:105EF000DEB72C970FB6F894DEBF0FBECDBF0F9460
:105F0000C60D0E94E4289CE0EBEFF5E0DE0111965F
:105F100001900D929A95E1F781110E94752ECE01A4
:105F200001960E9488C62C960FB6F894DEBF0FBE6D
:105F3000CDBFDF91CF9108952F923F924F925F9204
:105F40006F927F928F929F92AF92BF92CF92DF9289
:105F5000EF92FF920F931F93CF93DF9300D0CDB7B3
:105F6000DEB780901F0C9090200CA090210CB09078
:105F7000220C4090230C5090240C6090250C7090C3
:105F8000260CC090270CD090280CE090290CF090A3
:105F90002A0C0E94471B0E94951B02E61BE187E426
:105FA00092E09B838A8386E5282E8BE1382E198226
:105FB00089810E94381CC8010E941B1DEA81FB8157
:105FC0006193719381939193FB83EA83C1010E9452
:105FD0001B1DEA81FB816087718782879387F98126
:105FE000FF5FF9830C5F1F4F84E0280E311CF330F4
:105FF000F9F689ED95E00F942B0E0E94371E0E9452
:10600000C225A501940160911F0C7091200C809114
:10601000210C9091220C0F94F41F81111CC0A3013C
:1060200092016091230C7091240C8091250C909129
:10603000260C0F94F41F81110EC02091270C309173
:10604000280C4091290C50912A0CC701B6010F94DD
:10605000F41F8823B9F00F900F900F90DF91CF912C
:106060001F910F91FF90EF90DF90CF90BF90AF9076
:106070009F908F907F906F905F904F903F902F9068
:106080000C94752F0F900F900F90DF91CF911F916F
:106090000F91FF90EF90DF90CF90BF90AF909F90C7
:1060A0008F907F906F905F904F903F902F900895CA
:1060B0008091721190917311892B79F480917211F2
:1060C00090917311892B49F42091721130917311C1
:1060D00081E0232B19F480E0089581E00895109267
:1060E000E5048091220290912302A0912402B091B4
:1060F00025028093E5059093E605A093E705B0930C
:10610000E80508959091891110928911923071F0EB
:10611000943079F0913099F4813089F48091E504DC
:10612000882369F0109226020C946F3010921E0C96
:1061300008958CE697E190937E0C80937D0C0895F2
:106140009091DD1393FB882780F993FF06C081E0CF
:1061500090914415911101C080E00895CF93C091B2
:106160008505CF7739F50E94A030882319F18091F9
:10617000D5139091D613A091D713B091D81300974F
:10618000A105B105B9F0BC01CD016D597F4F8F4F0D
:106190009F4F24E630E040E050E00F9438266091B5
:1061A000D9137091DA138091DB139091DC130F9463
:1061B0003826C22F8C2FCF910895E8EFF8E0108297
:1061C0001182089581E008958F929F92AF92BF92BD
:1061D000CF92DF92EF92FF920F93CF93DF931F92B4
:1061E000CDB7DEB75C017B0149016B01C40ED51E42
:1061F000F501808191810F9412268983002311F08B
:10620000F7018083BE016F5F7F4FC4010E9494ED50
:10621000F50180819181019691838083FFEFEF1AD0
:10622000FF0AEC14FD0421F780E00F90DF91CF917D
:106230000F91FF90EF90DF90CF90BF90AF909F9025
:106240008F9008950F93AB010091DD0521E00227A7
:106250002EED35E0BC018EEB95E00E94E4300F910D
:1062600008959091D10095FD0CC09091D00095FFBC
:1062700008C08093D6008091D00080648093D000C5
:106280000895209114042F5F2F770FB607FC27C0C5
:1062900090911504921328C09091D00095FF1EC0D4
:1062A0009091150440911404941306C09091D1006C
:1062B0009F7D9093D10012C0E92FF0E0EC5EFB4F80
:1062C00032819F5F9F773093D60090931504309171
:1062D000D00030643093D000491741F3D9CF90916A
:1062E0001504921301C0FBCFE0911404F0E0EC5EC2
:1062F000FB4F8283209314048091D10080628093AD
:10630000D10008958F929F92AF92BF92CF92DF9269
:10631000EF92FF920F931F93CF93DF937C0121E5C0
:10632000E20EF11CD7014C914A3509F0A4C06C0172
:10633000B2E5CB0ED11CF6013081353A09F09BC095
:10634000EC01C05BDF4F2881233008F494C08C013E
:1063500000561F4FD8014C93E15BFF4F30833196BD
:106360002083EF54F1093081E05BFF4F30833038F8
:10637000B1F43196AC54B1093C913083E854F10941
:10638000AF5ABF4F50E040E02250330B4217530743
:10639000CCF4808132968D934F5F5F4FF7CF2330DF
:1063A00031F5313809F074C0FC01EC55FF4FDC01C8
:1063B000AC5ABF4F2C9120833196885A9F4FDC01F5
:1063C0008C9180834801B12CA12C888190E00296A9
:1063D0008A159B050CF43FC0F40181914F010E9486
:1063E00031310E94D7EDFFEFAF1ABF0AEECF32383E
:1063F00021F5FC01EC5AFF4F30814181E05BFF4FFA
:10640000408331963083DC01AA55BF4F50E040E015
:106410002350330B42175307ACF6FA01EE7FE45AD0
:10642000FF4FE80FF91F608171817C9311966C9387
:1064300011974E5F5F4F1296EDCF243019F6333827
:1064400009F6FC01EC5AFF4F20813181E05BFF4FE0
:1064500030833196B0CF80E5DE011D928A95E9F751
:106460008AE1F80111928A95E9F78AE5D7018C93C0
:1064700085EAF6018083DF91CF911F910F91FF9004
:10648000EF90DF90CF90BF90AF909F908F90089546
:10649000323809F097CFADCFAF92BF92CF92DF9253
:1064A000EF92FF920F931F93CF93DF93EC0184E65B
:1064B000C82E80E2D82EE12CF12C02E8A12C90E22B
:1064C000B92E15E000936A13C0926B13D0926C132F
:1064D000E0926D13F0926E13B0927413A092731346
:1064E0001093671387E193E10E9482318FEFC81AFE
:1064F000D80AE80AF80A88E7C81680E2D806E10454
:10650000F10401F724E630E240E050E0BE0187E10B
:1065100093E1DF91CF911F910F91FF90EF90DF906A
:10652000CF90BF90AF900C94DCEDCF92DF92EF92C2
:10653000FF920F931F93CF93DF93CDB7DEB77C010C
:10654000CDB6DEB60F94411F01962DB73EB7281B7E
:10655000390B0FB6F8943EBF0FBE2DBF0DB71EB757
:106560000F5F1F4FB701C8010F943A1FC8010E9467
:106570004C320FB6F894DEBE0FBECDBEDF91CF9188
:106580001F910F91FF90EF90DF90CF9008958F9221
:106590009F92AF92BF92CF92DF92EF92FF920F93B2
:1065A0001F93CF93DF930E94872B3AE0C32E30E2F4
:1065B000D32EE12CF12C15E002E846015701CAE088
:1065C000D0E010927413109273131093671300931A
:1065D0006A1380926B1390926C13A0926D13B09219
:1065E0006E1387E193E10E94823121978FEF881A21
:1065F000980AA80AB80A209721F78AE0C80ED11C89
:10660000E11CF11C82EDC81680E2D806E104F10419
:10661000A1F6C12C20E2D22EE12CF12CD5E0C2E86B
:106620001092741310927313D0936713C0936A136C
:10663000C0926B13D0926C13E0926D13F0926E13B4
:1066400087E193E10E9482311092741310927313C8
:10665000D0936713C0936A13D701C6018C529F4F22
:10666000AF4FBF4F80936B1390936C13A0936D1338
:10667000B0936E1387E193E10E9482318FEFC81AC5
:10668000D80AE80AF80A8AE0C81680E2D806E104C7
:10669000F10431F69EEDC92E90E2D92EE12CF12CB9
:1066A000D5E0C2E81092741310927313D09367135D
:1066B000C0936A13C0926B13D0926C13E0926D1367
:1066C000F0926E1387E193E10E9482318FEFC81A36
:1066D000D80AE80AF80A86EEC81680E2D806E1046D
:1066E000F10401F7CC24C39482E1D82EE12CF12CE3
:1066F0000AE010E0D5E0C2E810937413009373131E
:10670000D0936713C0936A13C0926B13D0926C132B
:10671000E0926D13F0926E1387E193E10E94823153
:106720001093741300937313D0936713C0936A1379
:10673000D701C6018096A11DB11D80936B13909364
:106740006C13A0936D13B0936E1387E193E10E94D5
:1067500082318FEFC81AD80AE80AF80A85E1C8160C
:1067600082E1D806E104F10439F682E190E09093E9
:10677000741380937313D0936713C0936A1384E1E7
:1067800090E1A0E0B0E080936B1390936C13A09322
:106790006D13B0936E1387E193E1DF91CF911F9159
:1067A0000F91FF90EF90DF90CF90BF90AF909F90B0
:1067B0008F900C9482311F920F920FB60F9211247A
:1067C0000BB60F922F938F939F93EF93FF9380912C
:1067D000150420911404821306C08091D1008F7D8E
:1067E0008093D10012C0E82FF0E0EC5EFB4F928165
:1067F0008F5F8F779093D600809315049091D0008F
:1068000090649093D000281741F3FF91EF919F91EE
:106810008F912F910F900BBE0F900FBE0F901F9076
:1068200018951F920F920FB60F9211240BB60F926C
:106830000F931F932F933F934F935F936F937F9388
:106840008F939F93AF93BF93CF93DF93EF93FF9378
:10685000C091D60000913905D091380511E01D0F87
:106860001F7390911304913108F09FC0E92FF0E05D
:106870008827E25CFB4C8F4F0D94AF264F347E345B
:106880008D349C34A334D534A734D534AB34AF34F1
:10689000D534B334B734BB34C234D534CD34C0323C
:1068A00029F028F5CA3011F0CD3031F5011731F05B
:1068B000ED2FF0E0E85CFA4FC283D12FD09338057A
:1068C000FF91EF91DF91CF91BF91AF919F918F9108
:1068D0007F916F915F914F913F912F911F910F91F8
:1068E0000F900BBE0F900FBE0F901F901895CD34D8
:1068F00081F081E0CE3471F080E10CC0CA3338F40D
:10690000C033A0F6C03291F2CD32B1F7CFCFCD3443
:1069100099F782E080931304C9CFC13359F018F47A
:10692000C03221F2E9CF88E0C433A1F38BE0C83351
:1069300089F3E2CF83E0EECF84E0C03359F386E001
:10694000C13341F3D9CF85E0C833B1F6E3CF87E057
:10695000C23391F6DFCF89E0C13371F6DBCF8AE035
:10696000C03351F6D7CF8CE0C73331F6D3CF8DE0AB
:10697000C63311F6CFCFC03209F498CF8EE0C335BD
:1069800049F2BACF80ED8C0F8A3008F08FCF9FE0AC
:10699000909313048093120489CFCA3019F0CD303C
:1069A00009F084CF1092130481CFCA3019F0CD3092
:1069B00009F07CCF8091D1138823A1F3973089F01F
:1069C00038F4953079F710923C0210921E0CEACF01
:1069D0009A3059F09F3031F7809112040E94823032
:1069E000E1CF81E080930C06DDCF81E080930B0640
:1069F000D9CF9091C00095FFFCCF8093C600089539
:106A0000CF93DF93EC018991882319F00E94F93428
:106A1000FACF8DE00E94F9348AE0DF91CF910C9497
:106A2000F934CF92DF92EF92FF92CF936B017C010A
:106A3000C42F4A3069F4F7FE0BC0F094E094D09470
:106A4000C094C11CD11CE11CF11C8DE20E94F934E0
:106A50004C2FC701B601CF91FF90EF90DF90CF9000
:106A60000C9456A6CF93DF93EC01FE0184912196FE
:106A7000882319F00E94F934F8CFDF91CF9108955F
:106A8000CF93DF93D0911C118EE39BE10E943235AE
:106A90008AE00E94F93480919B0C873009F449C048
:106AA00083E08093960C81E080936E0280E190E019
:106AB000909374138093731385E080936713C2E8F7
:106AC000C0936A1384E190E1A0E0B0E080936B137F
:106AD00090936C13A0936D13B0936E1387E193E1C1
:106AE0000E94823161E070E080E090E00E946C2BB7
:106AF00081E09AE5909374138093731385E390E09B
:106B0000909376138093751387E080936713C093F7
:106B10006A1384E890E0A0E0B0E080936B13909358
:106B20006C13A0936D13B0936E1387E193E10E94F1
:106B3000823180911C11813089F1823061F50E948F
:106B4000582A6093A6057093A7058093A805909393
:106B5000A90581E080931C110E9410A36093A205F7
:106B60007093A3058093A4059093A505D23089F076
:106B700080918F0690919006019690939006809355
:106B80008F061092AE051092AF051092B0051092CC
:106B9000B10581E004C00E948A2ADBCF80E0DF914A
:106BA000CF910895CF93C82FCB010E94323585EB4A
:106BB00097E10E94323586EA97E1CC2311F08BEA07
:106BC00097E10E9432358AE0CF910C94F93483ED3D
:106BD00097E10E9432358CB16DEC77E185FB882717
:106BE00080F90E94D2358091030167EC77E18695A8
:106BF00081700E94D23589B161EC77E183FB8827EF
:106C000080F90E94D2358CB168EB77E18295817072
:106C10000C94D23580911C118130C1F581E897E147
:106C20000E9432358AE00E94F93481E09AE590931F
:106C300074138093731387E590E090937613809399
:106C4000751387E08093671382E880936A1384E862
:106C500090E0A0E0B0E080936B1390936C13A0934E
:106C60006D13B0936E1387E193E10E94823182E04D
:106C700080931C110E9410A36093AA057093AB052A
:106C80008093AC059093AD0581E0089580E0089570
:106C90000F931F930E9410A300918A0610918B06F8
:106CA00020918C0630918D060115110521053105C5
:106CB00009F067C020914912222309F45FC0E091D6
:106CC000471221502093491221E02E0F20934712A2
:106CD00030914A12231302C01092471224E0E29F1F
:106CE000F0011124E55BFD4E008111812281338189
:106CF00000938606109387062093880630938906B2
:106D0000600F711F811D911D60938A0670938B0621
:106D100080938C0690938D068091880690918906C9
:106D2000892B61F11FB7F89480E797E10E94323513
:106D30008AE00E94F93484E096E090937413809383
:106D4000731380EA90E8909376138093751387E02D
:106D50008093671382E880936A1380EA90E0A0E052
:106D6000B0E080936B1390936C13A0936D13B0936A
:106D70006E1387E193E10E9482311FBF1F910F9133
:106D80000895601B710B820B930B97FDF7CF409812
:106D900010928A0610928B0610928C0610928D0625
:106DA000EDCF0F931F93CF93DF938C01EB01909165
:106DB000491220914A12921305C00E9448360E943F
:106DC0001EBEF5CF8091481234E0839FF00111245C
:106DD000E55BFD4E11830083D383C2839F5F909355
:106DE00049128F5F281739F080934812DF91CF91B5
:106DF0001F910F91089510924812F8CFCF92DF9211
:106E0000EF92FF921F93CF93DF93182F662351F0D9
:106E10001092E4041092E0041092E1041092E20453
:106E20001092E3040E9410A36B017C018091E004A6
:106E30009091E104A091E204B091E304A7019601CE
:106E4000281B390B4A0B5B0BDA01C901B7FD3DC0AA
:106E50002091E40417FD13C0412F012E000C550BA7
:106E60004C5F5F4F822F022E000C990B4817590779
:106E700064F184EF91E0A0E0B0E0211724F488EE03
:106E800093E0A0E0B0E08C0D9D1DAE1DBF1D809372
:106E9000E0049093E104A093E204B093E304217032
:106EA000C22F30E0D32F84E28C9FB0018D9F700DF4
:106EB0007C1B112460597C4F82E390E00E94D13604
:106EC0008091E4048F5F8093E404DF91CF911F9160
:106ED000FF90EF90DF90CF900895CF93DF9300D095
:106EE0001F92CDB7DEB786EF96E10E9432358AE079
:106EF0000E94F93480919B0C8330D9F119821A8257
:106F00001B821C8260E0CE0101960E94A52A198294
:106F10001A821B821C8261E0CE0101960E94A52A82
:106F200081E080936D021092950C80936E0281E057
:106F30009AE5909374138093731383E390E0909396
:106F400076138093751387E08093671382E88093AC
:106F50006A1384E890E0A0E0B0E080936B13909314
:106F60006C13A0936D13B0936E1387E193E10E94AD
:106F700082310F900F900F900F90DF91CF91089575
:106F80006F927F928F929F92AF92BF92CF92DF9239
:106F9000EF92FF920F931F93CF93DF93CDB7DEB79E
:106FA00064970FB6F894DEBF0FBECDBF1092D0002D
:106FB0008091D00082608093D0001092D50080E153
:106FC0008093D4008091D10080618093D100809122
:106FD000D10088608093D1008091D1008068809337
:106FE000D1008091D1008F7D8093D1008AE580937C
:106FF00068138093181385EA80936913809319139B
:10700000E7EBF3E18AE1DF011D928A95E9F78091D0
:10701000940C882309F473C283E090E09093741376
:107020008093731385E08093671382E880936A13DB
:107030008FE190E1A0E0B0E080936B1390936C132C
:10704000A0936D13B0936E1387E193E10E94823198
:1070500084E690E0909374138093731305E000939B
:10706000671312E810936A1386E090E1A0E0B0E0A5
:1070700080936B1390936C13A0936D13B0936E1366
:1070800087E193E10E9482318BE090E0909374134A
:10709000809373130093671310936A1380E092E157
:1070A000A0E0B0E080936B1390936C13A0936D13EA
:1070B000B0936E1387E193E10E94823110927413B2
:1070C000109273130093671310936A1384E390E193
:1070D000A0E0B0E080936B1390936C13A0936D13BA
:1070E000B0936E1387E193E10E9482311092741382
:1070F000109273130093671310936A138AE390E15D
:10710000A0E0B0E080936B1390936C13A0936D1389
:10711000B0936E1387E193E10E9482318091E31175
:107120009091E411909374138093731300936713F9
:1071300010936A1386E390E1A0E0B0E080936B13B4
:1071400090936C13A0936D13B0936E1387E193E14A
:107150000E948231809178119091791190937413EB
:10716000809373130093671310936A138CE390E179
:10717000A0E0B0E080936B1390936C13A0936D1319
:10718000B0936E1387E193E10E94823182E090E038
:1071900090937413809373130093671310936A137F
:1071A0008EE190E1A0E0B0E080936B1390936C13BC
:1071B000A0936D13B0936E1387E193E10E94823127
:1071C00081E080936D0270E6C72E70E1D72EE12C2E
:1071D000F12C109274131092731300936713109391
:1071E0006A13C0926B13D0926C13E0926D13F092FD
:1071F0006E1387E193E10E948231BFEFCB1ADB0A65
:10720000EB0AFB0AE4E7CE16E0E1DE06E104F10456
:1072100001F7CE0101967C0184E1D7011D928A9588
:10722000E9F781E08F9390E99F938F939CE29F937E
:107230008F939F9383E993E09F938F93FF92EF92B5
:107240000F94402A20E630E140E050E060EA73E02D
:1072500087E193E10E94DCED2AE630E140E050E076
:107260006CEA73E087E193E10E94DCED24E730E112
:1072700040E050E0B70187E193E10E94DCED2EE7AA
:1072800030E140E050E068EB73E087E193E10E9479
:10729000DCED109274131092731300936713109324
:1072A0006A138EE090E1A0E0B0E080936B139093BE
:1072B0006C13A0936D13B0936E1387E193E10E945A
:1072C000823110927413109273130093671310930A
:1072D0006A138FE090E1A0E0B0E080936B1390938D
:1072E0006C13A0936D13B0936E1387E193E10E942A
:1072F00082310FB6F894DEBF0FBECDBF4AE0C42E78
:1073000040E2D42EE12CF12C55E0752E62E8662E79
:10731000460157010AE010E01092741310927313A3
:107320007092671360926A1380926B1390926C1341
:10733000A0926D13B0926E1387E193E10E948231A7
:1073400001501109FFEF8F1A9F0AAF0ABF0A0115FA
:10735000110511F78AE0C80ED11CE11CF11C92ED59
:10736000C91690E2D906E104F10491F6C12C30E28D
:10737000D32EE12CF12C05E012E810927413109238
:1073800073130093671310936A13C0926B13D09218
:107390006C13E0926D13F0926E1387E193E10E94FB
:1073A0008231109274131092731300936713109329
:1073B0006A13D701C6018C529F4FAF4FBF4F8093C6
:1073C0006B1390936C13A0936D13B0936E1387E1BE
:1073D00093E10E948231AFEFCA1ADA0AEA0AFA0A86
:1073E000BAE0CB16B0E2DB06E104F10431F62EED93
:1073F000C22E20E2D22EE12CF12C05E012E81092F0
:107400007413109273130093671310936A13C0924E
:107410006B13D0926C13E0926D13F0926E1387E1B0
:1074200093E10E948231EFEFCE1ADE0AEE0AFE0AE5
:10743000F6EECF16F0E2DF06E104F10401F7CC240A
:10744000C39482E1D82EE12CF12C9AE0A92EB12C24
:1074500005E012E8B0927413A092731300936713BF
:1074600010936A13C0926B13D0926C13E0926D1359
:10747000F0926E1387E193E10E948231B09274130F
:10748000A09273130093671310936A13D701C60178
:107490008096A11DB11D80936B1390936C13A093E4
:1074A0006D13B0936E1387E193E10E9482318FEFE9
:1074B000C81AD80AE80AF80A95E1C91692E1D9066D
:1074C000E104F10439F68CE596E10E9432358AE058
:1074D0000E94F93464960FB6F894DEBF0FBECDBF9C
:1074E000DF91CF911F910F91FF90EF90DF90CF90A0
:1074F000BF90AF909F908F907F906F90089582E0A3
:1075000090E08CCD0E94C0371092810581E080937D
:107510006E028EE097E10E9432358AE00C94F934D5
:107520000F931F93CF938C01C62F87E093E10E94A6
:107530003235C8010E9432358AE30E94F93480E373
:107540008C0F0E94F9348AE0CF911F910F910C9417
:10755000F9348AE894E10E94323560E08AE794E1E8
:107560000E94903A60E085E694E10E94903A61E0E2
:107570008EE594E10E94903A61E083E594E10E94F7
:10758000903A61E083E494E10E94903A60E08AE3FB
:1075900094E10E94903A61E080E394E10E94903A85
:1075A00061E086E294E10E94903A61E08FE194E12B
:1075B0000E94903A61E087E194E10E94903A61E094
:1075C00089E094E10E94903A61E08BEF93E10E94A0
:1075D000903A60E08CEE93E10E94903A60E08EED8C
:1075E00093E10E94903A60E088EC93E10E94903A27
:1075F00061E087EB93E10E94903A61E088EA93E1D1
:107600000E94903A61E081EA93E10E94903A60E042
:107610008AE993E10E94903A61E081E993E10E9456
:10762000903A61E08CE793E10E94903A61E08EE647
:1076300093E10E94903A61E08BE593E10E94903AD9
:1076400060E08EE493E10E94903A61E089E493E186
:107650000E94903A61E08CE393E10E94903A60E0EE
:1076600088E293E10E94903A60E085E193E10E9414
:10767000903A60E080EE93E10E94FE1C682F6170FA
:107680008CE093E10C94903A80913205827149F438
:10769000809134058C7829F480913505837009F444
:1076A00075C082E40E94DC1D882351F00E94AA2349
:1076B0006093410C7093420C8093430C9093440C64
:1076C00083E50E94DC1D882351F00E9430246093E2
:1076D000710C7093720C8093730C9093740C84E50E
:1076E0000E94DC1D882351F00E9430246093750CA9
:1076F0007093760C8093770C9093780C88E50E94B9
:10770000DC1D882351F00E9430246093D4087093CC
:10771000D5088093D6089093D70889E50E94DC1D90
:10772000882351F00E9430246093D8087093D908C0
:107730008093DA089093DB088AE50E94DC1D882399
:10774000B1F00E9430246093DC087093DD088093D0
:10775000DE089093DF082DEC3CEC4CEC5DE30F94DD
:10776000F41F181624F08DE99DE00E94323585E45F
:107770000E94DC1D882351F00E9430246093E008B1
:107780007093E1088093E2089093E3080895AF9224
:10779000BF92CF92DF92EF920F931F93CF93DF931D
:1077A0005B01EA016901882309F463C086E99DE071
:1077B0000E943235F501608171818281938146E0BA
:1077C0000E945EB6E1100BC08DE89DE00E9432354C
:1077D000688179818A819B8146E00E945EB686E855
:1077E0009DE00E943235F601608171818281938132
:1077F00043E00E945EB68FE79DE00E943235F801BB
:10780000608171818281938143E00E945EB686E748
:107810009DE00E943235F601208131814281538101
:10782000F80160817181828193810F94B72643E0D2
:107830000E945EB6EE20F9F08AE00E94F93481E6FB
:107840009DE00E943235688179818A819B8146E082
:107850000E945EB68AE00E94F9348AE0DF91CF91FF
:107860001F910F91EF90DF90CF90BF90AF900C944D
:10787000F934E110E4CFDF91CF911F910F91EF9098
:10788000DF90CF90BF90AF9008950F931F93CF9349
:107890008C01C62F8EE797E00E943235C8010E9406
:1078A0003235CC2331F08AE0CF911F910F910C94A7
:1078B000F934CF911F910F9108950E94ECF110922D
:1078C0001E0C10923C020E94A030882351F080913F
:1078D000DD1382FD06C08CE697E190937E0C8093C9
:1078E0007D0C61E085E697E10E94453C0C944035B3
:1078F0000F931F93CF93DF938C016F3F19F4109276
:107900005D1160E020915D11862F062E000C990B11
:107910002817190609F08CF560935D1160E08FE27D
:1079200097E10E94453CC8010E9432358AE00E94DE
:10793000F934C8010F94411F800F911FEC01C01B47
:10794000D10BC034D1053CF00197FC012491207C7F
:107950002038D1F3F3CFDD27AE01B8018DE191E1FD
:107960000F94621FC35EDE4E18828DE191E1DF91BC
:10797000CF911F910F910C944C32DF91CF911F91B9
:107980000F91089510921E0C10923C028091DD130D
:1079900080648093DD1361E08DE397E10E94453CB4
:1079A00042E557E16AE577E185E00E94FAEF60E0A1
:1079B00084E497E10C94783C0F931F93CF938C0150
:1079C000C62F60E088E897E00E94453CC8010E940D
:1079D0003235CC2331F08AE0CF911F910F910C9476
:1079E000F934CF911F910F91089561E080E997E0FC
:1079F0000C94DC3CEF92FF920F931F93CF937C018A
:107A00008B01C42F60E088E897E00E94453CC701E5
:107A10000E94323580E20E94F934C8010E9432355A
:107A2000CC2319F08C2F0E94F9348AE0CF911F915A
:107A30000F91FF90EF900C94F934DF92EF92FF9248
:107A40000F931F93CF93DF93D82E7B018A01E90117
:107A50000E94F53CD092891140E0B70189E798E097
:107A60000E94FA3C0115110531F040E0B80182E7AF
:107A700098E00E94FA3C209731F040E0BE0182E796
:107A800098E00E94FA3C61E08DE698E0DF91CF91AA
:107A90001F910F91FF90EF90DF900C94DC3CAF9220
:107AA000BF92CF92DF92EF92FF920F931F93CF93EB
:107AB000DF9385E697E00E943235C0E0D7E0D150F1
:107AC00021F080E20E94F934FACF8C2F0E9433EE2D
:107AD000CF5FC53099F78AE00E94F93407E817E0D4
:107AE000C0E080E20E94F9348C2F0E9433EE5801EE
:107AF000D5E080E20E94F934F501C080D180E280B7
:107B0000F380A7019601C701B6010F94AA29882323
:107B100069F180E20E94F9348DE30E94F9348DE32B
:107B20000E94F9348DE30E94F9348DE30E94F93408
:107B30008DE30E94F934D150F4E1AF0EB11CD111A4
:107B4000D8CF8AE00E94F934CF5F0C5F1F4FC53059
:107B500041F68AE0DF91CF911F910F91FF90EF9056
:107B6000DF90CF90BF90AF900C94F93420E030E0DC
:107B7000A901C701B6010F94182987FD03C08BE244
:107B80000E94F93443E0C701B6010E945EB6D3CF2C
:107B9000811107C08FEC9DE00E9432358AE00C9481
:107BA000F93483ED9DE0F8CFCF93DF93EB010E9492
:107BB0003235CE01DF91CF910C94F1EECF93C62FE9
:107BC0000E9432358C2FCF910C9433EECF92DF92FE
:107BD000EF92FF926A017B010E94323542E0C701B9
:107BE000B601FF90EF90DF90CF900C945EB6CF92ED
:107BF000DF92EF92FF926A017B010E9432354AE0E8
:107C0000C701B601FF90EF90DF90CF900C94113533
:107C1000CF93DF93EB010E943235CE01DF91CF91FC
:107C20000C943AEE4F925F926F927F928F929F9256
:107C3000AF92BF92CF92DF92EF92FF920F931F937A
:107C4000CF93DF9300D000D01F921F92CDB7DEB745
:107C50008091800581110AC480917E0590917F05F5
:107C60009C012F5F3F4F30937F0520937E058E3E12
:107C7000924008F4FBC38091E3119091E41190933A
:107C800074138093731305E00093671312E8109345
:107C90006A1386E390E1A0E0B0E080936B139093C9
:107CA0006C13A0936D13B0936E1387E193E10E9460
:107CB000823180917811909179119093741380930F
:107CC00073130093671310936A138CE390E1A0E0A1
:107CD000B0E080936B1390936C13A0936D13B093EB
:107CE0006E1387E193E10E9482318091E5119091BA
:107CF000E61190937413809373130093671310939A
:107D00006A1384E390E1A0E0B0E080936B1390935A
:107D10006C13A0936D13B0936E1387E193E10E94EF
:107D2000823180917A1190917B119093741380939A
:107D300073130093671310936A138AE390E1A0E032
:107D4000B0E080936B1390936C13A0936D13B0937A
:107D50006E1387E193E10E94823181E08093800578
:107D600010927F0510927E0580919B0C882339F13B
:107D70000E94901C811123C080917D058F5F8093AC
:107D80007D0580917D05853620F010927D0510924D
:107D90009B0CE0919B0CE150E73008F06AC00E2E7E
:107DA000000CFF0B8827E852F14C8F4F0D94AF2643
:107DB000E23E313FFD4029416A41A241353F1092E8
:107DC0007D05DFCF0E94642B882309F452C081E037
:107DD00080936E0288EE96E10E9432358AE00E941E
:107DE000F93480E190E0909374138093731385E0ED
:107DF0008093671312E810936A1384E190E1A0E086
:107E0000B0E080936B1390936C13A0936D13B093B9
:107E10006E1387E193E10E94823181E09AE59093AD
:107E200074138093731386E390E09093761380939A
:107E3000751387E08093671310936A1384E890E0CA
:107E4000A0E0B0E080936B1390936C13A0936D133C
:107E5000B0936E1387E193E10E94823110929B0CE4
:107E600008C00E94642B882321F00E94901C882364
:107E7000A9F380916E02882309F433C780918105AC
:107E80008111C0C284E096E09093741380937313C1
:107E900080EA90E8909376138093751317E010931F
:107EA000671302E800936A1380EA90E0A0E0B0E074
:107EB00080936B1390936C13A0936D13B0936E1318
:107EC00087E193E10E9482318091690290916A0278
:107ED000A0916B02B0916C020097A105B10509F069
:107EE0003FC2109274131092731315E0109367132E
:107EF00000936A138AE890E1A0E0B0E080936B13EE
:107F000090936C13A0936D13B0936E1387E193E17C
:107F10000E94823189E090E09093741380937313F0
:107F20001093671300936A138CE890E1A0E0B0E02F
:107F300080936B1390936C13A0936D13B0936E1397
:107F400087E193E10E9482318091690290916A02F7
:107F5000A0916B02B0916C020097F1E0AF07B10500
:107F600008F441C2B0937413A093731390937613E3
:107F70008093751387E08093671382E880936A1378
:107F800088E890E1A0E0B0E080936B1390936C13CD
:107F9000A0936D13B0936E1387E193E10E94823139
:107FA0008091690290916A02A0916B02B0916C027B
:107FB000BA2FA92F982F8827009721E0A207B10593
:107FC00008F417C2B0937413A093731390937613AD
:107FD0008093751387E08093671312E810936A13F8
:107FE00081EA90E0A0E0B0E080936B1390936C1373
:107FF000A0936D13B0936E1387E193E10E948231D9
:108000008091300C882309F4FAC183E090E09093CA
:1080100074138093731385E08093671310936A132E
:1080200085E490E1A0E0B0E080936B1390936C1333
:10803000A0936D13B0936E1387E193E10E94823198
:1080400080918105875E8093810520918105822F33
:1080500090E0253608F021C2909374138093731337
:1080600085E08093671382E880936A1380E090E153
:10807000A0E0B0E080936B1390936C13A0936D130A
:10808000B0936E1387E193E10E9482310E94901CAD
:10809000811114C20E94A030811105C09091840505
:1080A00091FD0E94901C9091840580FB91F9909322
:1080B000840591FD03C28091DD1382FDFFC1809193
:1080C0001C118150823008F4F9C160917A117091CD
:1080D0007B11072E000C880B990B0F94FB1F6B0173
:1080E0007C0120E030E0A9010F94F41F882309F4FB
:1080F000BBC66091781170917911072E000C880B26
:10810000990B0F94FB1F2B013C0120E030E040E075
:1081100050E4C701B6010F94B726A30192010F9452
:10812000182918160CF4C2C66091E3117091E4117D
:10813000072E000C880B990B0F94FB1F6D837E8319
:108140008F8398876091E5117091E611072E000CDE
:10815000880B990B0F94FB1F4B015C0120E030E072
:1081600040E251E40F94B7262D813E814F8158851E
:108170000F94182918160CF499C620E030E040E05E
:1081800050E4C701B6010F94B826A30192010F94E1
:10819000F41F87FD10C020E030E040E251E4C5014B
:1081A000B4010F94B8262D813E814F8158850F94DC
:1081B000F41F87FF6AC684E190E090937413809364
:1081C000731385E08093671382E880936A1384E1D8
:1081D00090E1A0E0B0E080936B1390936C13A093B8
:1081E0006D13B0936E1387E193E10E948231809109
:1081F000960C81117CC682E07AC68AED96E10E94D7
:1082000032358AE00E94F93481E09AE59093741344
:108210008093731380E490E09093761380937513AA
:1082200017E01093671382E880936A1384E890E064
:10823000A0E0B0E080936B1390936C13A0936D1348
:10824000B0936E1387E193E10E94823110939B0CEF
:1082500010CE8091850C882309F40BCE0E94642BEC
:10826000882309F406CE0E94901C811102CE8CEC6A
:1082700096E10E9432358AE00E94F9348091860CA2
:1082800090E0B0E0A0E0895B9F4FAE4FB54A21E09F
:108290003AE530937413209373139093761380937D
:1082A000751387E08093671382E880936A1384E8EC
:1082B00090E0A0E0B0E080936B1390936C13A093D8
:1082C0006D13B0936E1387E193E10E948231109297
:1082D000850CC4CD0E94642B882309F4CACD0E946A
:1082E000901C8111C6CD81E080936E0210929B0C90
:1082F0008EEB96E10E9432358AE00E94F93481E0EB
:108300009AE590937413809373138EE490E09093A6
:1083100076138093751387E08093671382E88093C8
:108320006A1384E890E0A0E0B0E080936B13909330
:108330006C13A0936D13B0936E1387E193E10E94C9
:10834000823197CD0E94901C811193CD19821A829F
:108350001B821C8262E0CE0101960E946FF57ECDE9
:108360000196A11DB11D35E0B695A7959795879506
:108370003A95D1F70197A109B1090097E1E0AE075D
:10838000B10548F1B0937413A093731390937613CF
:10839000809375131093671312E810936A138AE899
:1083A00090E1A0E0B0E080936B1390936C13A093E6
:1083B0006D13B0936E1387E193E10E94823188E0E0
:1083C00090E0909374138093731385E08093671308
:1083D00010936A13A9CD909374138093731385E05F
:1083E00080936713D9CF909374138093731385E0B0
:1083F000C2CD909374138093731385E0ECCD82E02B
:1084000090E005CE8A3F08F020CE8EEF8093810564
:108410008DEA96E10E9432358AE00E94F93481E0CB
:1084200080936E0281E09AE59093741380937313A6
:108430008DE290E0909376138093751387E080939C
:10844000671382E880936A1384E890E0A0E0B0E0CC
:1084500080936B1390936C13A0936D13B0936E1372
:1084600087E193E10E9482311092800528960FB631
:10847000F894DEBF0FBECDBFDF91CF911F910F915A
:10848000FF90EF90DF90CF90BF90AF909F908F9034
:108490007F906F905F904F900895845691099093CC
:1084A00074138093731385E08093671382E880933D
:1084B0006A1381E090E1A0E0B0E0DCCD8CE090E0D8
:1084C000909374138093731315E01093671382E8ED
:1084D00080936A1384E190E1A0E0B0E080936B1395
:1084E00090936C13A0936D13B0936E1387E193E197
:1084F0000E9482310E94582A20E13EE040E050E094
:108500000F9438262115310581E04807510508F4FC
:1085100070C0509374134093731330937613209369
:10852000751387E08093671312E810936A1380E154
:1085300090E1A0E0B0E080936B1390936C13A09354
:108540006D13B0936E1387E193E10E9482310E9414
:10855000582A20E13EE040E050E00F9438262CE31A
:1085600030E040E050E00F943826309374132093AD
:10857000731305E00093671310936A1382E190E18F
:10858000A0E0B0E080936B1390936C13A0936D13F5
:10859000B0936E1387E193E10E9482310E94AE3066
:1085A000882309F45CC48F5F80937C05E82EF12C4E
:1085B000833330F5EE0CFF1CF0927413E0927313CA
:1085C0000093671310936A138EE090E1A0E0B0E08F
:1085D00080936B1390936C13A0936D13B0936E13F1
:1085E00087E193E10E948231109274131092731309
:1085F0002BC030937413209373131093671394CF8D
:1086000084E690E090937413809373130093671340
:1086100010936A138EE090E1A0E0B0E080936B13BA
:1086200090936C13A0936D13B0936E1387E193E155
:108630000E948231A2E3EA1AA0E8FA0AEE0CFF1CBB
:10864000F0927413E09273130093671310936A13FC
:108650008FE090E1A0E0B0E080936B1390936C13F7
:10866000A0936D13B0936E1387E193E10E94823162
:108670000E94AE3090E0909374138093731385E062
:108680008093671382E880936A1386E190E1A0E00B
:10869000B0E080936B1390936C13A0936D13B09321
:1086A0006E1387E193E10E94823120E030E0A9015E
:1086B00060912C1270912D1280912E1290912F1298
:1086C0000F94B82620E030E048EC52E40F945A2092
:1086D0000F942428709374136093731305E0009330
:1086E000671312E810936A1386E290E1A0E0B0E00D
:1086F00080936B1390936C13A0936D13B0936E13D0
:1087000087E193E10E948231809165029091660237
:1087100090937413809373130093671310936A13E9
:1087200080E093E1A0E0B0E080936B1390936C1332
:10873000A0936D13B0936E1387E193E10E94823191
:1087400020E030E040E251E46091450C7091460C2D
:108750008091470C9091480C0F945A200F942B282D
:1087600070937413609373130093671310936A13D9
:1087700082E492E1A0E0B0E080936B1390936C13DD
:10878000A0936D13B0936E1387E193E10E94823141
:1087900020E030E040E251E46091490C70914A0CD5
:1087A00080914B0C90914C0C0F945A200F942B28D5
:1087B00070937413609373130093671310936A1389
:1087C00086E492E1A0E0B0E080936B1390936C1389
:1087D000A0936D13B0936E1387E193E10E948231F1
:1087E00020E030E040E251E460914D0C70914E0C7D
:1087F00080914F0C9091500C0F945A200F942B287D
:1088000070937413609373130093671310936A1338
:108810008AE492E1A0E0B0E080936B1390936C1334
:10882000A0936D13B0936E1387E193E10E948231A0
:1088300020E030E040E251E46091510C7091520C24
:108840008091530C9091540C0F945A200F942B2824
:1088500070937413609373130093671310936A13E8
:108860008EE492E1A0E0B0E080936B1390936C13E0
:10887000A0936D13B0936E1387E193E10E94823150
:1088800020E030E048EC52E460912412709125120F
:1088900080912612909127120F945A200F94242829
:1088A00070937413609373130093671310936A1398
:1088B00086E392E1A0E0B0E080936B1390936C1399
:1088C000A0936D13B0936E1387E193E10E94823100
:1088D00020E030E048EC52E46091281270912912B7
:1088E00080912A1290912B120F945A200F942428D1
:1088F00070937413609373130093671310936A1348
:108900008AE392E1A0E0B0E080936B1390936C1344
:10891000A0936D13B0936E1387E193E10E948231AF
:1089200080917502909176029093741380937313E3
:108930000093671310936A1382E592E1A0E0B0E020
:1089400080936B1390936C13A0936D13B0936E137D
:1089500087E193E10E9482318091730290917402C9
:1089600090937413809373130093671310936A1397
:1089700084E592E1A0E0B0E080936B1390936C13D8
:10898000A0936D13B0936E1387E193E10E9482313F
:1089900020E030E040E251E46091E8117091E9118B
:1089A0008091EA119091EB110F945A200F942B288B
:1089B00070937413609373130093671310936A1387
:1089C00086E592E1A0E0B0E080936B1390936C1386
:1089D000A0936D13B0936E1387E193E10E948231EF
:1089E0002CEA35EC47E25EE36091EC117091ED11F9
:1089F0008091EE119091EF110F94B22720E030E0BA
:108A000040E251E40F945A200F942B287093741372
:108A1000609373130093671310936A138AE592E1CE
:108A2000A0E0B0E080936B1390936C13A0936D1350
:108A3000B0936E1387E193E10E9482312CEA35EC0A
:108A400047E25EE36091F0117091F1118091F211B3
:108A50009091F3110F945A2020E030E040E251E46D
:108A60000F945A200F942B287093741360937313F0
:108A70000093671310936A138EE592E1A0E0B0E0D3
:108A800080936B1390936C13A0936D13B0936E133C
:108A900087E193E10E94823120E030E040E251E43E
:108AA00060917D1170917E1180917F119091801164
:108AB0000F945A200F942B287093741360937313A0
:108AC0000093671310936A1382E692E1A0E0B0E08E
:108AD00080936B1390936C13A0936D13B0936E13EC
:108AE00087E193E10E9482312CEA35EC47E25EE3B4
:108AF0006091811170918211809183119091841104
:108B00000F94B22720E030E040E251E40F945A2065
:108B10000F942B287093741360937313009367134F
:108B200010936A1386E692E1A0E0B0E080936B13A5
:108B300090936C13A0936D13B0936E1387E193E140
:108B40000E9482312CEA35EC47E25EE360918511A8
:108B50007091861180918711909188110F945A20FD
:108B600020E030E040E251E40F945A200F942B288B
:108B700070937413609373130093671310936A13C5
:108B80008AE692E1A0E0B0E080936B1390936C13BF
:108B9000A0936D13B0936E1387E193E10E9482312D
:108BA00080918F0C811105C08091910C882309F46C
:108BB0006DC06091E3117091E411072E000C880BD9
:108BC000990B0F94FB1F20E030E048EC52E40F9427
:108BD0005A206B017C016091E5117091E611072E1E
:108BE000000C880B990B0F94FB1F9B01AC01C70174
:108BF000B6010F94B2270F942B286536710510F03B
:108C000064E670E0709374136093731305E000934F
:108C1000671312E810936A1384E290E1A0E0B0E0D9
:108C200080936B1390936C13A0936D13B0936E139A
:108C300087E193E10E9482316091E3117091E41128
:108C4000072E000C880B990B0F94FB1F6B017C0106
:108C500020E030E04AE253E40F941829181624F477
:108C600080918F0C811146C16091E5117091E611E0
:108C7000072E000C880B990B0F94FB1F9B01AC0176
:108C8000C701B6010F94182987FFAFC18091850CE9
:108C9000882339F18091840C91E0980F9093840C93
:108CA00090E0909374138093731385E0809367131F
:108CB00082E880936A1382E490E1A0E0B0E08093C0
:108CC0006B1390936C13A0936D13B0936E1387E1A5
:108CD00093E10E9482318091840C8A3010F01092CE
:108CE000840C0E94EE2A882309F4B5C16091990C86
:108CF00070919A0CEE24E394F12C61157105A9F0A2
:108D000090E080E00F94F91F20E030E040E85EE35F
:108D10000F945A200F94962720E030E040E85FE35C
:108D20000F94B8260F942B287B0101E010E080916E
:108D30007F0C811102C010E000E080915B129091E5
:108D40005C128F3F980711F40E94B3AF90935C12AE
:108D500080935B12080F191FB80190E080E00F9418
:108D6000F91F20E030E040E85EE30F945A200F94B2
:108D700096274B015C01F0927413E092731305E0A7
:108D80000093671312E810936A1380E193E1A0E067
:108D9000B0E080936B1390936C13A0936D13B0931A
:108DA0006E1387E193E10E948231C501B4010F94F3
:108DB0002B287093741360937313009367131093AD
:108DC0006A1382E193E1A0E0B0E080936B1390938B
:108DD0006C13A0936D13B0936E1387E193E10E941F
:108DE000823107EB13E1AAE1FA2E809138059091C8
:108DF000390520917A0530917B05891B8F7309F421
:108E000049C12A3131050CF0DBC1909138058091C0
:108E100039054FEF5FEF981749F0E82FF0E0E85C75
:108E2000FA4F42818F5F8F7380933905F901E954BE
:108E3000FC4E40838091B7138A3509F0B3C162E0DC
:108E400070E080E090E00E946C2B80917A05909118
:108E50007B05019690937B0580937A05C6CF10928F
:108E6000741310927313ACCB6091E5117091E611FD
:108E7000072E000C880B990B0F94FB1F20E030E0AD
:108E8000A9010F94F41F811134C98CE090E09093F4
:108E900074138093731385E08093671382E8809343
:108EA0006A1384E190E1A0E0B0E0F3CB8DE090E0C4
:108EB000909374138093731385E08093671382E813
:108EC00080936A1384E190E1A0E0B0E080936B139B
:108ED00090936C13A0936D13B0936E1387E193E19D
:108EE0000E9482318091960C811101C081E08093B3
:108EF000960CDBCB10928F0C20E030E040E251E486
:108F00006091870C7091880C8091890C90918A0CEB
:108F10000F945A200F942428709374136093731342
:108F20000093671310936A1384E590E1A0E0B0E02A
:108F300080936B1390936C13A0936D13B0936E1387
:108F400087E193E10E94823120E030E040E251E489
:108F500060918B0C70918C0C80918D0C90918E0C8B
:108F60000F945A200F9424287093741360937313F2
:108F70000093671310936A1388E590E1A0E0B0E0D6
:108F800080936B1390936C13A0936D13B0936E1337
:108F900087E193E10E9482318CE896E10E943235AC
:108FA0008AE00E94F93481E09AE5909374138093EB
:108FB000731381E490E0909376138093751387E0A8
:108FC0008093671310936A1384E890E0A0E0B0E008
:108FD00080936B1390936C13A0936D13B0936E13E7
:108FE00087E193E10E94823151CE6091910C66231A
:108FF00009F44CCE062E000C770B83E796E10E9415
:10900000083E8AE00E94F9341092910C84E090E0CE
:10901000909374138093731385E08093671312E821
:1090200010936A138EE890E1A0E0B0E080936B1398
:1090300090936C13A0936D13B0936E1387E193E13B
:109040000E94823181E09AE59093741380937313A8
:1090500083E590E0B0CF109274131092731305E083
:109060000093671312E810936A1380E193E1A0E084
:10907000B0E080936B1390936C13A0936D13B09337
:109080006E1387E193E10E94823110927413109263
:10909000731393CE121613060CF492C080911B1317
:1090A00090911C13A0911D13B0911E138C34E0E11C
:1090B0009E07A105B10509F4D7C98A349041A105DD
:1090C000B10509F4D1C920E030E040E251E46091FB
:1090D0001F0C7091200C8091210C9091220C0F9408
:1090E0005A200F942428709374136093731305E02F
:1090F0000093671312E810936A1388E490E1A0E0EC
:10910000B0E080936B1390936C13A0936D13B093A6
:109110006E1387E193E10E94823120E030E040E26B
:1091200051E46091230C7091240C8091250C909156
:10913000260C0F945A200F94242870937413609374
:1091400073130093671310936A138AE490E1A0E00D
:10915000B0E080936B1390936C13A0936D13B09356
:109160006E1387E193E10E94823120E030E040E21B
:1091700051E46091270C7091280C8091290C9091FA
:109180002A0C0F945A200F94242870937413609320
:1091900073130093671310936A138CE490E1A0E0BB
:1091A000B0E056C9121613060CF01FCEF8012F2D91
:1091B00011922A95E9F710927B0510927A0515CE47
:1091C000909118138091B713981321C0909119139F
:1091D0008091B81398131BC023303105C4F09091CF
:1091E000B913909317138091BA1380931A13933085
:1091F000D1F4982F9D7F9038B1F49091BB139F3498
:1092000009F059C09091BC139B3409F054C0E7EBAE
:10921000F3E18AE1DF011D928A95E9F710927B055F
:1092200010927A053BCF833809F045C08091BB137B
:109230009091BC13982789279827B0E0A0E08093ED
:109240001B1390931C13A0931D13B0931E13C09077
:10925000BD13D12CF12CE12CC0921F13D0922013FE
:10926000E0922113F09222132EEB33E140E050E024
:10927000BA014C155D056E057F0508F04AC0DB019B
:10928000CA01B695A795979587950696880F991F59
:10929000FC01E95EFC4ED9018C9111969C918927C5
:1092A00098278927918380834E5F5F4F6F4F7F4F51
:1092B0002E5F3F4FDECF813861F58091BB1390E088
:1092C000B0E0A0E080931B1390931C13A0931D1398
:1092D000B0931E138091BC13482F50E070E060E003
:1092E00040931F1350932013609321137093221304
:1092F000ADEBB3E1E3E2F3E190E030E020E0821790
:10930000930739F04D9150E0419351932F5F3F4FB8
:10931000F6CFE7EBF3E18AE1DF011D928A95E9F7E9
:1093200010927B0510927A050E9411F6B7CE3F92FB
:109330004F925F926F927F928F929F92AF92BF9265
:10934000CF92DF92EF92FF920F931F93CF93DF9311
:109350008091340587FD38C0809135058370A1F573
:10936000C0913012D0913112488159816A817B813C
:109370008DEF95E10E94E63D4C815D816E817F819C
:1093800089E39EE20E94E63D40912C1250912D12FD
:1093900060912E1270912F1286E39EE20E94E63DAC
:1093A0008AE0DF91CF911F910F91FF90EF90DF90B6
:1093B000CF90BF90AF909F908F907F906F905F9075
:1093C0004F903F900C94F9346090241270902512C5
:1093D0008090261290902712A0902812B090291207
:1093E00000912A1210912B12C0902C12D0902D12A5
:1093F000E0902E12F0902F1288E50E942A1EC82FAE
:10940000882309F49AC00E943024362E472E582E05
:10941000D92F20E030E046E953EC0F94182987FD5E
:109420000DC020E030E046E953E4632D742D852D16
:109430009D2F0F94F41F18160CF081C06CE271E0A0
:109440008AEE95E10E94083E6CE271E085EE95E1BE
:109450000E94083E82EE95E10E943235C0E089E527
:109460000E942A1E882361F10E943024362E472E46
:10947000582ED92F20E030E046E953EC0F941829FC
:1094800087FD0DC020E030E046E953E4632D742DE4
:10949000852D9D2F0F94F41F18160CF055C06CE20B
:1094A00071E08FEC95E10E94083E6CE271E08AEC7D
:1094B00095E10E94083E87EC95E10E943235C0E0BC
:1094C0008AE50E942A1E882309F443C00E943024A2
:1094D0006B017C0120E030E040E151EC0F94182951
:1094E00087FD0AC020E030E040E151E4C701B60149
:1094F0000F94F41F18166CF567EF7FEF85EB95E17D
:109500000E94083E69E070E080EB95E10E94083E11
:109510008DEA95E1DF91CF911F910F91FF90EF9030
:10952000DF90CF90BF90AF909F908F907F906F9083
:109530005F904F903F900C943235C1E090CF632CF8
:10954000742C852C9D2E8BCFA32CB42C052D1D2F78
:10955000B7CFCC23E1F0C301D401809324129093C0
:109560002512A0932612B0932712C501D80180932B
:10957000281290932912A0932A12B0932B12C09212
:109580002C12D0922D12E0922E12F0922F12DF9117
:10959000CF911F910F91FF90EF90DF90CF90BF90F0
:1095A000AF909F908F907F906F905F904F903F9083
:1095B00008958EE597E00C94323588E597E00C9499
:1095C000323584E690E09093BF058093BE051092FB
:1095D000DF051092DE050C94CFDBEF92FF920F9324
:1095E0001F93CF93DF93CDB7DEB762970FB6F89492
:1095F000DEBF0FBECDBF0E94F128882309F43FC013
:1096000044EE53E082FF02C048EC53E024EE33E026
:1096100081FF02C02AEC33E080FD2EC084EE93E08F
:109620005F934F933F932F939F938F9387E298E19C
:109630009F938F938E010F5F1F4F1F930F930F9474
:109640008B1F0E94DD4AC8010E940035C8010E949C
:10965000B4F10FB6F894DEBF0FBECDBF81E06296C5
:109660000FB6F894DEBF0FBECDBFDF91CF911F9133
:109670000F91FF90EF9008958CEC93E0D1CF80E0B4
:10968000EECFCF92DF92EF92FF928AE50E942A1EE0
:10969000882309F45AC00E94302420E030E040E0E2
:1096A00050EC0F94F41FC12CD12CE12C90ECF92E2E
:1096B00087FD0FC00E94302420E030E040E050E4FD
:1096C0000F94182918160CF462C00E9430246B0104
:1096D0007C0120914D0C30914E0C40914F0C5091DB
:1096E000500CC701B6010F945A200F942428CB01C7
:1096F0000E943DF180E50E94DC1D81114EC0A70152
:10970000960160912C1270912D1280912E129091E1
:109710002F120F94B82660932C1270932D12809301
:109720002E1290932F120E94DD4A40912C125091DC
:109730002D1260912E1270912F128EE995E10E94E8
:10974000E63D8AE00E94F93405C083E50E942A1EA6
:109750008111A1CF8091340587FD24C0809135050A
:10976000837001F50E94DD4A40912C1250912D1218
:1097700060912E1270912F128FE895E10E94E63DC4
:109780008AE0FF90EF90DF90CF900C94F934C12CD9
:10979000D12CE12C80E4F82E9CCF0E94F82381117B
:1097A000AECFD8CF82E50E94DC1D8111DBCFFF90C8
:1097B000EF90DF90CF900895CF9384E50E942A1E0A
:1097C000C0E08823D9F00E94D823C82F1816B4F41B
:1097D0000E94DD4A8DE40E94F93480912F0590911A
:1097E00030050E94F1EE6C2FCC0F770B8DEA9EE0D6
:1097F0000E94083E8AE00E94F934CFEF8C2FCF916F
:1098000008954F925F926F927F928F929F92AF9244
:10981000BF92CF92DF92EF92FF92CF93DF93CDB7BB
:10982000DEB72C970FB6F894DEBF0FBECDBF4090C9
:10983000C7085090C8086090C9087090CA08209165
:109840004702309148024091490250914A02C301B7
:10985000B2010F94B82669837A838B839C838090AE
:10986000CB089090CC08A090CD08B090CE08209165
:109870004B0230914C0240914D0250914E02C50175
:10988000B4010F94B8266D837E838F839887C09030
:10989000CF08D090D008E090D108F090D208209165
:1098A0004F02309150024091510250915202C70133
:1098B000B6010F94B82669877A878B879C87209199
:1098C0005302309154024091550250915602C30107
:1098D000B2010F94B8262B013C0120915702309120
:1098E00058024091590250915A02C501B4010F9497
:1098F000B8264B015C0120915B0230915C024091E3
:109900005D0250915E02C701B6010F94B8266B014B
:109910007C010E94DD4A88EE9DE00E94323583E59D
:109920000E94DC1D882321F00E94F82380934502C9
:1099300080914502811151C08FEC9DE00E9432352B
:1099400080EE9DE00E94323549815A816B817C8195
:1099500082EF9CE10E94E63D4D815E816F817885BA
:1099600089E39EE20E94E63D49855A856B857C85A8
:1099700086E39EE20E94E63D8EED9DE00E94323538
:1099800086ED9DE00E943235B301A20182EF9CE199
:109990000E94E63DB501A40189E39EE20E94E63DF6
:1099A000B701A60186E39EE20E94E63D8AE02C967E
:1099B0000FB6F894DEBF0FBECDBFDF91CF91FF9001
:1099C000EF90DF90CF90BF90AF909F908F907F905F
:1099D0006F905F904F900C94F93483ED9DE0AECF83
:1099E0005F926F927F928F929F92AF92BF92CF922F
:1099F000DF92EF92FF920F931F93CF93DF931F920B
:109A0000CDB7DEB77C0139018B015B01A40EB51E19
:109A1000D12CC12CA016B10609F450C0F7018080EA
:109A20009180F80151908F015982C4010F94122640
:109A30005816B9F1652DC4010F941A26FFEFCF1AFD
:109A4000DF0AC6018F779927892B21F162E070E048
:109A500080E090E00E94DDA2C4010F94122699815B
:109A60008917F9F00E94DD4A8FE694E00E943235B2
:109A700081E00F90DF91CF911F910F91FF90EF90B8
:109A8000DF90CF90BF90AF909F908F907F906F901E
:109A90005F90089562E070E080E090E00E949E2573
:109AA000DBCFBE016F5F7F4FC3010E9494EDF701D2
:109AB00080819181019691838083ACCF80E0D9CF62
:109AC000CF92DF92EF92FF920F931F93CF93DF938A
:109AD000CDB7DEB7CA5AD1090FB6F894DEBF0FBEB4
:109AE000CDBFCF55DF4F188219821A821B82C15A0F
:109AF000D0408091CE039091CF03A091D003B0913C
:109B0000D103CB55DF4F88839983AA83BB83C55A82
:109B1000D04084E690E09093BF058093BE051092FC
:109B2000DF051092DE051092E0052EED35E044E0F1
:109B300050E0BE016B557F4F8EEB95E00E94F04CDC
:109B40008091BE059091BF0502969093BF058093CA
:109B5000BE051092DF051092DE0581E0C655DF4F8D
:109B60008883CA5AD040CE0186559F4F0E94F4D1B7
:109B70002EED35E048E450E061E37CE08EEB95E0CB
:109B80000E94F04C2EED35E040E150E064ED78E0CD
:109B90008EEB95E00E94F04C8AE097EDA3EABCE3DF
:109BA000CF55DF4F88839983AA83BB83C15AD040A6
:109BB000CE018F559F4F0E94EBD18DEF97E00E9411
:109BC00006D286E292E00E94FDD182E292E00E94FB
:109BD000EBD18091C3089091C408A091C508B091C1
:109BE000C60889839A83AB83BC838E010F5F1F4FA6
:109BF000C8010E94EBD1CF55DF4F188219821A821B
:109C00001B82C15AD0407E018DE6E80EF11C83E034
:109C1000D7018C938983CE018F559F4F0E94EBD142
:109C2000C7010E94F4D1C8010E94F4D14AE0D42EA9
:109C3000DA94DD2031F0CE018F559F4F0E94EBD199
:109C4000F7CF84E292E10E9406D2CF55DF4F18820F
:109C500019821A821B82C15AD0403AE0D32EDA947C
:109C6000DD2031F0CE018F559F4F0E94EBD1F7CF11
:109C700085E0C82EC982F701C082C8010E94F4D1D4
:109C8000C7010E94F4D12EED35E048E050E061EDCF
:109C900075E08EEB95E00E94F04C2EED35E048E04B
:109CA00050E069EC75E08EEB95E00E94F04C2EEDF3
:109CB00035E044E650E067E877E08EEB95E00E94FF
:109CC000F04C19828FEFD7018C93C8010E94FDD10F
:109CD000C7010E94F4D190E1D92EF8018D2D119287
:109CE0008A95E9F72EED35E040E150E0B8018EEBC2
:109CF00095E00E94F04C1982C8010E94FDD1198A9A
:109D00001A8A1B8A1C8A80E090E0A0E8BFE38D8756
:109D10009E87AF87B88B8091E8119091E911A0914F
:109D2000EA11B091EB1189839A83AB83BC832CEA4F
:109D300035EC47E25EE36091EC117091ED1180919A
:109D4000EE119091EF110F94B2276D837E838F8374
:109D500098872CEA35EC47E25EE36091F011709150
:109D6000F1118091F2119091F3110F945A206987AB
:109D70007A878B879C872EED35E044E150E0B8016F
:109D80008EEB95E00E94F04C84E190E09A83898309
:109D9000C8010E94D9D180917D1190917E11A0912E
:109DA0007F11B091801189839A83AB83BC832CEAA5
:109DB00035EC47E25EE360918111709182118091F0
:109DC0008311909184110F94B2276D837E838F83CA
:109DD00098872CEA35EC47E25EE36091851170913B
:109DE000861180918711909188110F945A2069876C
:109DF0007A878B879C87C8010E94E2D18CE0EBE7D1
:109E0000F2E0D80101900D928A95E1F7C8010E9415
:109E1000E2D11982C8010E94F4D18FE790E09A83C1
:109E20008983C8010E94D9D1E7E8F2E0D801019006
:109E30000D92CA94E1F72EED35E045E050E0B8010F
:109E40008EEB95E00E94F04C8091C8058983C80193
:109E50000E94FDD180E2ECE8F2E0D80101900D9281
:109E60008A95E1F72EED35E040E250E0B8018EEB47
:109E700095E00E94F04CD7011C92C7010E94FDD1D1
:109E800080EF97E00E94FDD18CEE97E00E94EBD12D
:109E9000CF55DF4F188219821A821B82C15AD040D7
:109EA000CE018F559F4F0E94EBD180E2F8011192B5
:109EB0008A95E9F72EED35E040E250E0B8018EEBEF
:109EC00095E00E94F04CFE01F99688E0DF011D92BA
:109ED0008A95E9F744E650E060E070E049835A83F0
:109EE0006B837C834D835E836F83788783E090E010
:109EF000A0E0B0E089879A87AB87BC874D875E87F3
:109F00006F87788B498B5A8B6B8B7C8B8D8B9E8B61
:109F1000AF8BB88F898F9A8FAB8FBC8F8D8F9E8FB1
:109F2000AF8FB8A38EE190E0A0E0B0E089A39AA340
:109F3000ABA3BCA38DA39EA3AFA3B8A789A79AA7E1
:109F4000ABA7BCA78DA79EA7AFA7B8AB89AB9AABB1
:109F5000ABABBCAB8DAB9EABAFABB8AF2EED35E0D2
:109F600040E450E0B8018EEB95E00E94F04CF8011F
:109F70008D2D11928A95E9F72EED35E040E150E004
:109F8000B8018EEB95E00E94F04CD8011D92DA9456
:109F9000E9F72EED35E040E150E0B8018EEB95E0B9
:109FA0000E94F04CCF55DF4F188219821A821B8213
:109FB000C15AD040CE018F559F4F0E94EBD12CE06B
:109FC000D22EF8018D2D11928A95E9F72EED35E00C
:109FD0004CE050E0B8018EEB95E00E94F04C8CE62E
:109FE000D8011D928A95E9F72EED35E04CE650E058
:109FF000B8018EEB95E00E94F04C82EB95E00E9458
:10A00000E2D12EED35E048E050E060EC75E08EEBFB
:10A0100095E00E94F04CF7011192DA94E9F7C755E8
:10A02000DF4F1882C95AD04080E090E0A0E4B0E44D
:10A03000C356DF4F88839983AA83BB83CD59D04011
:10A04000C7010E9406D2CE0187559F4F0E94F4D1CE
:10A05000CE0183569F4F0E94EBD180E3D7011D9222
:10A060008A95E9F78EE69BE10E9432358AE00E94EC
:10A07000F9342EED35E040E350E0B7018EEB95E08A
:10A080000E94F04C8091E005811128C00091BE052E
:10A090001091BF058091DE059091DF05F701918356
:10A0A000808384E690E09093BF058093BE052EEDFB
:10A0B00035E044E050E060EF72E08EEB95E00E9406
:10A0C000F04CC7010E94D9D191E00137134009F447
:10A0D00090E08091E005892B8093E0058091E00578
:10A0E000811105C060E082EA9BE10E94783C82E831
:10A0F0009BE10E9432358AE00E94F9349091E0059C
:10A1000081E08927C655DF4F0FB6F894DEBF0FBE3A
:10A11000CDBFDF91CF911F910F91FF90EF90DF9016
:10A12000CF900895CF93DF9300D01F92CDB7DEB7C5
:10A1300080918E068823C1F083E390E09C838B831B
:10A140001A8219829E012F5F3F4F40E150E06FE875
:10A1500076E0CE0103960E94F04C82E89BE10E94DB
:10A1600032358AE00E94F9340F900F900F900F90D3
:10A17000DF91CF910895CF92DF92EF92FF92CF932C
:10A18000C82F80911C118150823008F069C00E9454
:10A190006D3710921C110E9410A36093AA05709352
:10A1A000AB058093AC059093AD05C090AE05D09003
:10A1B000AF05E090B005F090B1050E94582AAB01C0
:10A1C000BC014093AE055093AF056093B00570930A
:10A1D000B1058091930690919406A0919506B09157
:10A1E00096068C199D09AE09BF09840F951FA61FFD
:10A1F000B71F8093930690939406A0939506B0930F
:10A200009606C1110AC0C1E00E9492508C2FCF91D6
:10A21000FF90EF90DF90CF900895809191069091FC
:10A220009206019690939206809391060E94582A76
:10A23000C0909706D0909806E0909906F0909A0604
:10A24000C616D706E806F906F0F60E94582A60936B
:10A250009706709398068093990690939A06D3CFA9
:10A26000C0E0D2CFCF93DF9300D01F921F92CDB723
:10A27000DEB781E080938E0680E1EFE8F6E0DF0153
:10A280001D928A95E9F70E94925086E18D8382E3C0
:10A2900090E09C838B831A8219829E012F5F3F4F2F
:10A2A00041E050E0BE016B5F7F4FCE0103960E94FC
:10A2B000F04C0F900F900F900F900F90DF91CF9177
:10A2C0000895CF93DF93CDB7DEB7A8970FB6F89474
:10A2D000DEBF0FBECDBF8C01F42E0E94D1BA0E940A
:10A2E000D94A88E397E00E9432350115110511F42F
:10A2F0000FE217E08091840580FD79C08160809332
:10A3000084058BE197E00E9432358AE00E94F9349F
:10A31000CC24C3948AE5D82ED0927413C0927313C0
:10A320008FE090E0909376138093751397E0792EE9
:10A330007092671322E8E22EE0926A1334E8832ECB
:10A34000912CA12CB12C80926B1390926C13A09243
:10A350006D13B0926E1387E193E10E948231D09227
:10A360007413C092731388E590E0909376138093F2
:10A37000751370926713E0926A1380926B13909238
:10A380006C13A0926D13B0926E1387E193E10E945B
:10A3900082318AE289838A838B838C83F801DE0190
:10A3A0001596BE016F5F7F4FCD01861B970B2491E1
:10A3B000319621110CC0FB01E80FF91F8AE29F01C1
:10A3C000261B370B2832310524F48193F8CF2D93C7
:10A3D000EBCF20E630E140E050E087E193E10E94DE
:10A3E000DCED6AE070E080E090E00E946C2B61E0C0
:10A3F00086E297E00E94453C89EE93E030E60197C3
:10A4000029F0232F2A950000E9F7F9CFF89489EE77
:10A4100093E038EE019729F0232F2A950000E9F701
:10A42000F9CF0E94D1BAFF2031F00E94961E0E94FF
:10A43000AF1EA895FECF0E94941EF9CF80917E0793
:10A44000882319F010927E07089540E070E060E0E4
:10A4500088E997E10E94615180919C0C90919D0C3C
:10A460002FEF3FEF981751F0E92FF0E0E456F34F4C
:10A47000228130E09F5F9F7790939D0CC9010895E2
:10A480001F920F920FB60F9211240F900FBE0F90D4
:10A490001F9018951F920F920FB60F9211240BB6B2
:10A4A0000F920F931F932F933F934F935F936F934D
:10A4B0007F938F939F93AF93BF93CF93DF93EF934C
:10A4C000FF93C091C60000919D0CD0919C0C11E0AF
:10A4D0001D0F1F7790911104913108F09FC0E92F53
:10A4E000F0E08827E958FD4A8F4F0D94AF26885237
:10A4F000B752C652D552DC520E53E0520E53E452BC
:10A50000E8520E53EC52F052F452FB520E530653E3
:10A51000C03229F028F5CA3011F0CD3031F50117DD
:10A5200031F0ED2FF0E0E456F34FC283D12FD093FA
:10A530009C0CFF91EF91DF91CF91BF91AF919F91D3
:10A540008F917F916F915F914F913F912F911F91CB
:10A550000F910F900BBE0F900FBE0F901F9018958C
:10A56000CD3481F081E0CE3471F080E10CC0CA338B
:10A5700038F4C033A0F6C03291F2CD32B1F7CFCF6C
:10A58000CD3499F782E080931104C9CFC13359F0DB
:10A5900018F4C03221F2E9CF88E0C433A1F38BE094
:10A5A000C83389F3E2CF83E0EECF84E0C03359F3C0
:10A5B00086E0C13341F3D9CF85E0C833B1F6E3CFAC
:10A5C00087E0C23391F6DFCF89E0C13371F6DBCF8C
:10A5D0008AE0C03351F6D7CF8CE0C73331F6D3CF02
:10A5E0008DE0C63311F6CFCFC03209F498CF8EE09C
:10A5F000C33549F2BACF80ED8C0F8A3008F08FCF87
:10A600009FE0909311048093120489CFCA3019F00F
:10A61000CD3009F084CF1092110481CFCA3019F0E7
:10A62000CD3009F07CCF8091D1138823A1F39730EE
:10A6300089F038F4953079F710923C0210921E0C94
:10A64000EACF9A3059F09F3031F7809112040E947E
:10A650008230E1CF81E080930C06DDCF81E08093F2
:10A660000B06D9CF8EBD0DB407FEFDCF08958FEF39
:10A670008EBD0DB407FEFDCF8EB508959091640098
:10A680009B7F90936400982F906A96959CBD80FD67
:10A6900003C091E0863009F490E09DBD0895CF930A
:10A6A000DF93EB010E943235CE01DF91CF910C9404
:10A6B0001BAB2F923F924F925F926F927F928F923D
:10A6C0009F92AF92BF92CF92DF92EF92FF920F9341
:10A6D0001F93CF93DF93009709F0AAC11092810CCA
:10A6E0001092800C9093830580938205BAE0CB2E64
:10A6F000B0E2DB2EE12CF12C15E002E84601570117
:10A70000C4E1D0E01092BA121092B9121093AD12B7
:10A710000093B0128092B1129092B212A092B31232
:10A72000B092B4128DE592E10E94823121972FEF11
:10A73000821A920AA20AB20A209721F744E1C40EB3
:10A74000D11CE11CF11C8AE5C81680E2D806E104A0
:10A75000F104A1F6C12CA0E2DA2EE12CF12CD5E017
:10A76000C2E81092BA121092B912D093AD12C093EF
:10A77000B012C092B112D092B212E092B312F09223
:10A78000B4128DE592E10E9482311092BA121092B9
:10A79000B912D093AD12C093B012D701C6018C523A
:10A7A0009F4FAF4FBF4F8093B1129093B212A093BF
:10A7B000B312B093B4128DE592E10E948231EFEFB3
:10A7C000CE1ADE0AEE0AFE0AFAE0CF16F0E2DF0643
:10A7D000E104F10431F6FEEDCF2EF0E2DF2EE12CA4
:10A7E000F12CD5E0C2E81092BA121092B912D093AF
:10A7F000AD12C093B012C092B112D092B212E092D8
:10A80000B312F092B4128DE592E10E9482312FEFE3
:10A81000C21AD20AE20AF20A46EEC41640E2D4068E
:10A82000E104F10401F7CC24C394E2E1DE2EE12C33
:10A83000F12C0AE010E0D5E0C2E81093BA120093C0
:10A84000B912D093AD12C093B012C092B112D0928F
:10A85000B212E092B312F092B4128DE592E10E942E
:10A8600082311093BA120093B912D093AD12C093F3
:10A87000B012D701C6018096A11DB11D8093B112FF
:10A880009093B212A093B312B093B4128DE592E1FB
:10A890000E9482318FEFC81AD80AE80AF80AE5E068
:10A8A000CE16E2E1DE06E104F10439F60091800CF7
:10A8B0001091810C0115110509F0D6C080917F0C13
:10A8C000882309F4E1C02AE030E240E050E062ED84
:10A8D00073E08DE592E10E94DCEDC1E0D0E003E0A1
:10A8E00010E0E090800CF090810C35E0332E42E8CF
:10A8F000242E44244A94542C64E0662E712C7FE16B
:10A90000C72E74E0D72E8091800C9091810C800F1F
:10A91000911FE816F90608F0D5C0C7010E94F7EEAE
:10A92000882309F481C0809197116AE871E1882336
:10A9300011F067E971E1FB0101900020E9F7CF0117
:10A940000197861B970BF4E1FC9F9001FD9F300D52
:10A950001124265F3F4D50E040E0459710F0FB0189
:10A96000128A8DE592E10E94DCEDCE018F5F9D4E53
:10A97000B0E0A0E021964E0124E0880C991C2A95B5
:10A98000E1F7FDEF8F1AFFE99F0AB12CA12C20916E
:10A99000DD1324FF7EC07092BA126092B912309219
:10A9A000AD122092B0128093B1129093B212A09384
:10A9B000B312B093B4128DE592E10E948231D0922D
:10A9C000BA12C092B9123092AD122092B012809297
:10A9D000B1129092B212A092B312B092B4128DE55D
:10A9E00092E10E948231B7018DE297E10E94D43D4D
:10A9F0008091971167E971E1811102C06AE871E104
:10AA00008AE297E10E944F536EED7BE086E297E188
:10AA10000E944F536AE871E185E297E10E944F532B
:10AA200081E297E10E9432352FEFE21AF20A6BCFF2
:10AA30002091800C3091810CA90141505109609105
:10AA40008205709183056817790738F42C5F3F4FB2
:10AA50003093810C2093800C45CE4430510508F48E
:10AA60003DCE24503109F4CF0430110569F48091B2
:10AA70007F0C882331F083E090E09093810C8093E9
:10AA8000800CD0E0C0E02DCFD0E0C0E004E010E0CA
:10AA900028CF1092BA121092B9123092AD122092B1
:10AAA000B0128093B1129093B212A093B312B093EC
:10AAB000B4128DE592E10E9482315092BA12409216
:10AAC000B91281CFDF91CF911F910F91FF90EF903D
:10AAD000DF90CF90BF90AF909F908F907F906F90BE
:10AAE0005F904F903F902F900895AF92BF92CF927A
:10AAF000DF92EF92FF920F931F93CF93DF93CDB727
:10AB0000DEB7E6970FB6F894DEBF0FBECDBF00915B
:10AB1000360510913705F80101900020E9F73197CB
:10AB20006F01C01AD10AF801CF01801B910B8C155F
:10AB30009D053CF481918F32B9F7DF0111971C928A
:10AB4000F3CF8BE1EDEFF3E1DE015C9601900D9226
:10AB50008A95E1F7F12CE12CEC14FD040CF05DC0BA
:10AB6000F801EE0DFF1D8081811103C08FEFE81AFF
:10AB7000F80A5801AE0CBF1CF5018081882309F446
:10AB80004CC0FFEFEF1AFF0AF801EE0DFF1D7F0129
:10AB9000E01AF10A81918111FACFCE014C960E9400
:10ABA000AEAF8BE1FE017C96DE01119601900D9215
:10ABB0008A95E1F7B501CE0101960E94BCA7CE01AE
:10ABC00001960E946F2E8FE20E94F93480919711B6
:10ABD00081113BC08FED93E00E941BAB8091DD1390
:10ABE00084FF1BC019821C8221E0A501BE01645EA6
:10ABF0007F4FCE0101960E94F0B1811129C08AE0F9
:10AC00000E94F9340E94DD4AB5018CE096E10E9471
:10AC10004F53CE0101960E946F2E8AE00E94F934B4
:10AC2000CE014C960E946F2EE6960FB6F894DEBFCA
:10AC30000FBECDBFDF91CF911F910F91FF90EF908D
:10AC4000DF90CF90BF90AF90089587E991E1C4CF96
:10AC5000CE014C960E941DAF8BE1FE013196DE01C4
:10AC60005C9601900D928A95E1F7CE0101960E94C3
:10AC70006F2E72CF2F923F924F925F926F927F9280
:10AC80008F929F92AF92BF92CF92DF92EF92FF92FC
:10AC90000F931F93CF93DF9300D000D000D01F926B
:10ACA0001F92CDB7DEB7B82E8091890D843008F0A1
:10ACB000D1C10E9410A36B017C018091890D81118B
:10ACC00008C080919C0C90919D0C891B8F7709F492
:10ACD000A4C681E6A82E13C08A3019F08D3009F081
:10ACE000F6C01092840D8091220D9091230DFC01ED
:10ACF000E25EF24F1682892BF1F40E941EBE809113
:10AD0000890D843008F0ECC080919C0C90919D0CD2
:10AD1000891B8F7709F4E4C00E942C5297FFDCCF87
:10AD20000E94D94A85EB95E00E94323580919C0CB7
:10AD300080939D0CE4CF1092230D1092220D04E21B
:10AD40001DE0F8018191803209F446C08E3409F08B
:10AD5000A9C060EB75E0C8010F94711F4C01892BED
:10AD600041F06EE470E0C80104960F94062A009743
:10AD700009F4C8014AE050E070E060E001960F94E9
:10AD8000E11C2B013C0180911E0D90911F0DA091A3
:10AD9000200DB091210D0196A11DB11D4816590637
:10ADA0006A067B0629F060E08DE795E0892851F17D
:10ADB0006AE270E0C8010F94352A9C01009729F1DE
:10ADC000982F901B912C992349F09150F801E90F8D
:10ADD000F11D80819826F7CF8F01B3CF4AE050E074
:10ADE00070E060E0C90101960F94E11C292D30E06C
:10ADF00050E040E0621773078407950751F060E068
:10AE00008EE595E00E94E9F47ACF60E084E395E076
:10AE1000F9CF40921E0D50921F0D6092200D70923E
:10AE2000210D8091E3068130E1F067E470E0C80114
:10AE30000F94062A0097A9F04AE050E070E060E025
:10AE400001960F94E11C643071058105910548F469
:10AE500083E994E00E94323560E089E894E00E9442
:10AE6000783CC0928307D0928407E0928507F092E5
:10AE700086078091240D8B3309F441CF8091890D91
:10AE8000843008F03CCF80918B0D8A9DC001112445
:10AE900064E27DE08457924F0F94112A80E00E9473
:10AEA000A3F42DCF8091DD1380FFBBCF6DE77CE253
:10AEB000C8010F94711F009731F0FC01838180530A
:10AEC0008A3008F0AECF60E08AE095E09BCF22E2C6
:10AED0003DE044E25DE064E87DE00E94AA1C0FCF03
:10AEE0008091DD1382FFB6C01A82198271E6F72EB7
:10AEF000E0E1EE2EF9E6DF2E8091890D843008F036
:10AF0000A9C00E94E21C8111A5C041E050E0BE0131
:10AF10006B5F7F4F81E495E10E9470AD0D8110E081
:10AF2000019711F00FEF1FEF8091491590914A158D
:10AF3000A0914B15B0914C158093D9139093DA13CF
:10AF4000A093DB13B093DC130E94E21C0F3F1007A9
:10AF500049F4811107C00E94D94A83ED95E00E940F
:10AF60003235CACF40918B0D242F30E00A3061F08A
:10AF70000D3051F0882309F45FC089819A810097D0
:10AF800019F001969A8389831092960489819A8197
:10AF9000F29EF001F39EF00D1124E757F24FE80FF7
:10AFA000F91F1382892B69F50E941EBE0E94E21CC4
:10AFB000882309F4A1CF0E94A45D81E495E10E9459
:10AFC0001DAF8091D413882391F181508093D413C5
:10AFD0008D9DC001112462E0845E994F0E9472B47D
:10AFE000E091D41324E0E29FF0011124E85EF94FD0
:10AFF00060817181828193810E94FB210E9425A73B
:10B000007BCF1A82198281E00E94A3F48091D91328
:10B010009091DA13A091DB13B091DC138093850D2E
:10B020009093860DA093870DB093880DBFCF0E949B
:10B0300026AFE092E30660CF4F9DA0011124445754
:10B04000524F9E012F5F3F4F66E974E0802F0E94B0
:10B05000AA1C52CF0E9410A36B017C01B11004C046
:10B0600080911B11882351F0C0926E11D0926F1104
:10B07000E0927011F0927111BB24B39480910E058F
:10B0800090910F05A0911005B09111050097A105B1
:10B09000B105B1F040916E1150916F116091701136
:10B0A00070917111840F951FA61FB71FA7019601FC
:10B0B000281B390B4A0B5B0BDA01C901B7FF92C1A0
:10B0C0008091140290911502A0911602B09117027E
:10B0D000892B8A2B8B2B09F099C10E9410A34B015D
:10B0E0005C0180911E0C811108C020913512909155
:10B0F000361281E0291301C080E02091E3113091E4
:10B10000E41191E089272A3A31050CF480E091E0BE
:10B1100040919B0450919C0460919D0470919E0409
:10B12000452B462B472B09F490E0981789F088238C
:10B1300009F4BDC1D501C40180569444A24FBF4F4C
:10B1400080939B0490939C04A0939D04B0939E04D1
:10B1500040902B0C50902C0C60902D0C70902E0C6D
:10B1600020919704309198044091990450919A0449
:10B17000C301B2010F94F41F882319F180919B043D
:10B1800090919C04A0919D04B0919E0440929704DC
:10B19000509298046092990470929A04892B8A2B99
:10B1A0008B2B09F449C0D501C40180569444A24FA9
:10B1B000BF4F80939B0490939C04A0939D04B093F5
:10B1C0009E0480919B0490919C04A0919D04B09159
:10B1D0009E040097A105B10579F1881A990AAA0A77
:10B1E000BB0AB7FC29C010929B0410929C041092D9
:10B1F0009D0410929E0483E396E00E94323560E045
:10B200008FE196E00E94783C8091E5119091E611E3
:10B210001816190624F490E080E00E94B21E809176
:10B220007A1190917B111816190634F410927B1143
:10B2300010927A110E94A4BA8091A3049091A40460
:10B24000A091A504B091A60446015701881A990A55
:10B25000AA0ABB0AD501C401B7FDB9C120913512B4
:10B260009091361240912D0280912C02291323C116
:10B270009091F808899FC0011124880F892F881F99
:10B28000990B91958D838091F908489FC0011124F5
:10B29000880F892F881F990B91958E830E9410A388
:10B2A00069837A838B839C8340E0BE016F5F7F4F0D
:10B2B000CE0105960E94FC1B6D8170E089E00E9422
:10B2C00007A241E0BE016F5F7F4FCE0105960E944D
:10B2D000FC1B6E8170E087E00E9407A28091170638
:10B2E000882309F467C10091200210912102C8014E
:10B2F00002972091E5113091E611281739070CF4D7
:10B3000059C1809036128F82188619861A861B863C
:10B31000809135129F80891509F4E7C0892D90E04E
:10B320003CE5A32EA89EF001A99EF00D1124E35048
:10B33000F74F458956896789708D452B462B472BDA
:10B3400081F4418D528D638D748D452B462B472B97
:10B3500041F4458D568D678D70A1452B462B472BAB
:10B36000E1F12CE5B22EB89E9001B99E300D11246A
:10B37000A9014350574F1A01FA01618172818381FB
:10B3800094810F9466294B015C01F10161A172A1C6
:10B3900083A194A10F94F91F2B013C01F10165A138
:10B3A00076A187A190A50F94F91F9B01AC01C30161
:10B3B000B2010F94B227A50194010F945A204B01BA
:10B3C0005C01288539854A855B850F9418291816F4
:10B3D00024F488869986AA86BB868F818F5F8770C2
:10B3E0008F8396CF0E94D94A60918107709182071E
:10B3F00082EE95E00E944F538AE00E94F93440E0CB
:10B4000070E060E090E080E00E9461519091351220
:10B4100080913612981749F0C0926E11D0926F1138
:10B42000E0927011F092711158CEBB2019F0109279
:10B43000A70453CE0E9410A300916E1110916F11BA
:10B44000209170113091711180901402909015022A
:10B45000A0901602B0901702080D191D2A1D3B1D61
:10B46000601B710B820B930B97FDE1CF8091A704BA
:10B47000811133CE81E08093A7045F9A80912F0CD5
:10B480008E7F80932F0C8A9A80912F0C8D7F8093D2
:10B490002F0C809108018095817080930601809126
:10B4A0002F0C8B7F80932F0C0E94941E16CE80E071
:10B4B00090E0DC0145CE209136125CE5259F90019D
:10B4C00011242350374FF901EA5AFF4F9081899F89
:10B4D000C0011124880F892F881F990B91958D83A6
:10B4E000295A3F4FF9018081D0CE20911A02309124
:10B4F0001B0240911C0250911D02688579858A8546
:10B500009B850F945A204B015C01B801012E000C61
:10B51000880B990B0F94FB1F9B01AC01C501B40173
:10B520000F94B82669837A838B839C8340911E0293
:10B5300050911F02B801CE0101960E94DCBD8980A6
:10B540009A80AB80BC8040909F045090A004609093
:10B55000A1047090A204A3019201C501B4010F944B
:10B56000F41F87FF16C028E431EE4AE75FE3C3010A
:10B57000B2010F945A2020E037ED43EA5CE30F94C8
:10B58000B826A50194010F945A2069837A838B838E
:10B590009C8369817A818B819C8160939F047093E5
:10B5A000A0048093A1049093A2040F942428CB01BB
:10B5B0000E94B21EF4E6CF0ED11CE11CF11CC09219
:10B5C000A304D092A404E092A504F092A6040E94E1
:10B5D0001EBE8091E306882309F4E0C18091260213
:10B5E000882309F4A3C08091E50481119FC0809154
:10B5F0001B11811108C080911C11813021F08091B4
:10B60000DD1382FF93C0F894649B10C080912202E6
:10B6100090912302A0912402B09125028093E50528
:10B620009093E605A093E705B093E8056091E505E2
:10B630007091E6058091E7059091E805789420E007
:10B6400030E0A9010F94F41F87FF70C001E0009360
:10B65000E50480911B11811167C088E496E00E9487
:10B6600032358AE00E94F93484E08093960C82E0BF
:10B670008093820C81E09AE5909374138093731306
:10B680008EE490E0909376138093751387E0809317
:10B69000671382E880936A1384E890E0A0E0B0E04A
:10B6A00080936B1390936C13A0936D13B0936E13F0
:10B6B00087E193E10E9482310E94F53C0093891159
:10B6C00040E36CE876E089E798E00E94FA3C61E0AC
:10B6D0008DE698E00E94DC3C1091120560E0102796
:10B6E00081E498E069F48AE796E00E94453C80E3B3
:10B6F0000E94F9348AE00E94F93460E08DE596E01A
:10B700000E94453C88E696E00E94323580E30E9424
:10B71000F9348AE00E94F934112331F083E696E08F
:10B7200090937E0C80937D0C0E94A45D9091090102
:10B73000892F80958170109100021817C9F020910F
:10B74000DD1320622093DD138093000290FD3FC142
:10B7500064EF71E080E090E00E949E250E9448AF77
:10B760008091DD1383FD7CC1111133C10E94C7326A
:10B770000E9410A36B017C01109113021123F1F0C0
:10B78000809113058823D1F04091A8045091A90419
:10B790006091AA047091AB0446015701841A950A7E
:10B7A000A60AB70AB501A40177FD1AC0833009F4CF
:10B7B0002FC10CF01EC181300CF023C1212F30E0CD
:10B7C000A8EEB3E00F948C26C60ED71EE81EF91E15
:10B7D000C092A804D092A904E092AA04F092AB040B
:10B7E00080911C11813009F073C00E9410A36B017D
:10B7F0007C018091B0049091B104A091B204B09109
:10B80000B304A7019601281B390B4A0B5B0BDA0125
:10B81000C901B7FD3AC0D701C601805F984DAF4F4F
:10B82000BF4F8093B0049093B104A093B204B0933F
:10B83000B3048090AE059090AF05A090B005B09095
:10B84000B1050E94582AAB01BC014093AE0550934C
:10B85000AF056093B0057093B10580919306909108
:10B860009406A0919506B091960688199909AA099F
:10B87000BB09840F951FA61FB71F80939306909353
:10B880009406A0939506B09396068091AC0490918F
:10B89000AD04A091AE04B091AF0446015701881ADF
:10B8A000990AAA0ABB0AD501C401B7FD11C020E854
:10B8B000C20E2EEED21E26E3E21EF11CC092AC0494
:10B8C000D092AD04E092AE04F092AF040E94925088
:10B8D0000E9448360E94123E80910D05882379F11E
:10B8E0000E9410A36B017C018091090590910A05CB
:10B8F000A0910B05B0910C0546015701881A990AD1
:10B90000AA0ABB0AD501C401B7FD19C020910D05D3
:10B9100030E0A8EEB3E00F948C26C60ED71EE81ECA
:10B92000F91EC0920905D0920A05E0920B05F0922B
:10B930000C0580E00E9402B78AE00E94F9348091F1
:10B940000805882359F10E9410A36B017C018091A6
:10B95000040590910505A0910605B0910705A70182
:10B960009601281B390B4A0B5B0BDA01C901B7FDA5
:10B9700015C02091080530E0A8EEB3E00F948C26A6
:10B98000C60ED71EE81EF91EC0920405D09205050A
:10B99000E0920605F09207050E94E3A62B960FB6EB
:10B9A000F894DEBF0FBECDBFDF91CF911F910F91F5
:10B9B000FF90EF90DF90CF90BF90AF909F908F90CF
:10B9C0007F906F905F904F903F902F9008950E94CE
:10B9D00037AF123008F0CCCE0E94C73260E085EC61
:10B9E00096E056C083ED96E090937E0C80937D0C9C
:10B9F000BFCE843009F0E2CE0E94DD4A8AED96E0A7
:10BA000004C00E94DD4A89E097E00E943235D6CE1C
:10BA10000E94DD4A82EF96E0F8CF809183079091F3
:10BA20008407A0918507B0918607A7019601281B7E
:10BA3000390B4A0B5B0BDA01C901885E9340A109FF
:10BA4000B109B7FD46C98DEC95E00E943235C09230
:10BA50008307D0928407E0928507F092860739C960
:10BA60001230C8F48DE996E00E9432358AE00E94D7
:10BA7000F9340E94872B90E080E00E945953109285
:10BA80009A0C1092990C1092980C60E086EB96E05C
:10BA90000E94783C6DCE123009F06ACE0E94A2B3AB
:10BAA000882379F081E00E9478B342EB50E069E0AE
:10BAB00078E082EE93E10E9470AD82EE93E10E9405
:10BAC0001DAF0E945D2E81118DCF0E94472E0E94D6
:10BAD0001EB40E9473B34CCECF93DF938091351286
:10BAE00090913612891B8095877019F40E943A56FE
:10BAF000F5CF809135128F5F8770A09135129CE54C
:10BB0000A99FD0011124FD01E350F74FEF011992D5
:10BB10009A95E9F798E09083AE5EB64F90E1E7E33F
:10BB2000F2E101900D929A95E1F7209135129091F2
:10BB30003612291303C094E6909332128093351283
:10BB4000DF91CF910C94752E909135128091361221
:10BB5000981306C08091FB089091FC08892B21F076
:10BB600080E00E943A56F0CF0895FC012081318197
:10BB7000428153816091510C7091520C8091530C11
:10BB80009091540C0F945A200F94252960934312DE
:10BB900070934412809345129093461290913512FF
:10BBA0008091361298130C946C5D0E94A45D0E94E3
:10BBB000E4284091431250914412609145127091D3
:10BBC0004612409307065093080660930906709347
:10BBD0000A0681110C94752E08954F925F926F9210
:10BBE0007F928F929F92AF92BF92CF92DF92EF920D
:10BBF000FF920F931F93CF93DF93EC018B015A01B8
:10BC0000F9012091510C3091520C4091530C5091FC
:10BC1000540C60817181828193810F945A200F941A
:10BC200025296B017C0120914D0C30914E0C4091E7
:10BC30004F0C5091500CF50160817181828193818C
:10BC40000F945A200F9425294B015C012091490C37
:10BC500030914A0C40914B0C50914C0CF801608192
:10BC60007181828193810F945A200F9425292B0191
:10BC70003C012091450C3091460C4091470C50916D
:10BC8000480C688179818A819B810F945A200F9496
:10BC9000252960933712709338128093391290934C
:10BCA0003A1240923B1250923C1260923D127092B6
:10BCB0003E1280923F1290924012A0924112B09296
:10BCC0004212C0924312D0924412E0924512F09276
:10BCD00046129091351280913612981791F0DF91AB
:10BCE000CF911F910F91FF90EF90DF90CF90BF9079
:10BCF000AF909F908F907F906F905F904F900C943B
:10BD00006C5D0E94A45D0E94E42840913F12509116
:10BD10004012609141127091421200913B121091B9
:10BD20003C1220913D1230913E12C0903712D090BB
:10BD30003812E0903912F0903A12C092FB05D0927E
:10BD4000FC05E092FD05F092FE050093FF051093BF
:10BD50000006209301063093020640930306509399
:10BD600004066093050670930606409143125091B5
:10BD70004412609145127091461240930706509309
:10BD800008066093090670930A06882391F0DF91F4
:10BD9000CF911F910F91FF90EF90DF90CF90BF90C8
:10BDA000AF909F908F907F906F905F904F900C948A
:10BDB000752EDF91CF911F910F91FF90EF90DF9043
:10BDC000CF90BF90AF909F908F907F906F905F903B
:10BDD0004F9008954F925F926F927F928F929F92B1
:10BDE000AF92BF92CF92DF92EF92FF920F931F9389
:10BDF000CF93DF93CDB7DEB72C970FB6F894DEBFA5
:10BE00000FBECDBF2B013C0129873A874B875C874A
:10BE100047015801F601E080F1800281138120E0A2
:10BE200030E0A901B701C8010F94F41F882309F479
:10BE300088C05E2D4F2D302F212F852F942FA32FBB
:10BE4000B22F89839A83AB83BC8320E030E0A901C1
:10BE5000B701C8010F94F41F811108C0E0903D02A2
:10BE6000F0903E0200913F0210914002C701D801BC
:10BE70008D839E83AF83B887A50194016091270CC1
:10BE80007091280C8091290C90912A0C0F94F41F2A
:10BE900087FF0CC08092270C9092280CA092290C4E
:10BEA000B0922A0CCE0101960E94BF2940921F0C2D
:10BEB0005092200C6092210C7092220C89859A85F8
:10BEC000AB85BC858093230C9093240CA093250C08
:10BED000B093260CCE0105960E94BF29A5019401BE
:10BEE0006091270C7091280C8091290C90912A0C5C
:10BEF0000F941829181664F48092270C9092280C3D
:10BF0000A092290CB0922A0CCE0101960E94BF2962
:10BF10000E94A45D2C960FB6F894DEBF0FBECDBF75
:10BF2000DF91CF911F910F91FF90EF90DF90CF9015
:10BF3000BF90AF909F908F907F906F905F904F9049
:10BF4000089550E040E030E820E477CFCF92DF92D0
:10BF5000EF92FF920F931F936A01E090270CF090ED
:10BF6000280C0091290C10912A0CFB0120813181B1
:10BF700042815381FC0160817181828193810E94A1
:10BF8000EA5E1F910F91FF90EF90DF90CF900895A0
:10BF9000CF92DF92EF92FF920F931F936B01FC0100
:10BFA000E080F18002811381EFE1FCE024813581A2
:10BFB0004681578160817181828193810E94EA5E0E
:10BFC0001F910F91FF90EF90DF90CF900895AF9267
:10BFD000BF92CF92DF92EF92FF920F931F93CF9376
:10BFE000DF9300D01F92CDB7DEB7FC01E080F18077
:10BFF00002811381611112C0A090270CB090280C0F
:10C00000C090290CD0902A0C9501A601B701C80157
:10C010000F94F41F87FF02C07501860120E030E015
:10C0200048EC53E4B701C8010F94F41F87FD04C026
:10C03000E12CF12C08EC13E4C701D80189839A8321
:10C04000AB83BC8360EE72E0CE0101960E94C85FB4
:10C050000F900F900F900F90DF91CF911F910F9144
:10C06000FF90EF90DF90CF90BF90AF900895BF9278
:10C07000CF92DF92EF92FF920F931F93CF93DF93B4
:10C0800000D01F92CDB7DEB7B82E882351F180E0E3
:10C0900090E0A0E2B1E489839A83AB83BC83C09033
:10C0A0002C12D0902D12E0902E12F0902F1220E042
:10C0B00030E0A901C701B6010F94F41F87FF0CC03F
:10C0C000A701960160E070E080E291E40F94B7264A
:10C0D00069837A838B839C8360E0CE0101960E9402
:10C0E000E75F60911F0C7091200C8091210C909162
:10C0F000220C2091230C3091240C4091250C50915E
:10C10000260C19821A821B821C82E090270CF09068
:10C11000280C0091290C10912A0CFE0131966F0118
:10C120000E94EA5EB0927F070E94492A0F900F900A
:10C130000F900F90DF91CF911F910F91FF90EF9093
:10C14000DF90CF90BF90089580917F07882319F0EA
:10C1500080E00E94376080E008952F923F924F92D6
:10C160005F926F927F928F929F92AF92BF92CF9287
:10C17000DF92FF920F931F93CF93DF93CDB7DEB77C
:10C1800060970FB6F894DEBF0FBECDBFF82E282EF5
:10C19000312CF101EA52F24D4490042C000C550868
:10C1A000660877086101CC0CDD1CCC0CDD1C82E03C
:10C1B000F81609F407C1C301B2010F94FB1F2B014C
:10C1C0003C01C6018A58974E0E941B1D4B015C0121
:10C1D000A3019201C501B4010F945A204B015C01E7
:10C1E000C6018659974E0E941B1D20E030E040ECAE
:10C1F0005FE30F945A20A30192010F945A20AB01E0
:10C20000BC0100E010E098018F2D0F942D1320E069
:10C2100030E0A901C501B4010F94F41F882309F48B
:10C2200040C092E000E010E020E431E4F91619F09B
:10C2300000E010E09801B501A40170588F2D0F9413
:10C240002D13A5019401C501B4010F94B8264B012B
:10C250005C01E2E000E010E020EC30E4FE16E1F0EA
:10C26000F101E55AF74E6491611107C00E94DD4A61
:10C2700089E398E10E9432356AE070E090E080E066
:10C280000F94F91F9B01AC0160E070E088E492E438
:10C290000F94B2278B019C01B501A4018F2D0F943F
:10C2A0002D1381E090E0A0E0B0E00F2C04C0880FD7
:10C2B000991FAA1FBB1F0A94D2F720912F0C282B7D
:10C2C00020932F0C20919905822B80939905C6010C
:10C2D000825A974E0E941B1DF601E15EF34F608368
:10C2E000718382839383F2E0FF121AC020912C1293
:10C2F00030912D1240912E1250912F126091270CE7
:10C300007091280C8091290C90912A0C0F94B726DB
:10C310006093270C7093280C8093290C90932A0C1F
:10C32000F601EF50F84F10821182128213828F2D86
:10C330000E94381C0E94DA29F601E15EF34F8081E9
:10C340009181A281B381F601E259F84F80839183F4
:10C35000A283B38382E0F81609F462C08CE0ECEAB1
:10C36000F2E0DE01119601900D928A95E1F7E1E08D
:10C37000F0E0EC0FFD1FEC0DFD1D80809180A28090
:10C38000B38020E030E0A901C501B4010F94F41F8F
:10C3900081114BC060960FB6F894DEBF0FBECDBFC3
:10C3A000DF91CF911F910F91FF90DF90CF90BF90C1
:10C3B000AF909F908F907F906F905F904F903F9045
:10C3C0002F90089580917F07811103C081E00E9422
:10C3D00037608EE798E10E941B1D20E030E0A90144
:10C3E0000F94F41F882309F4E6CEC301B2010F9421
:10C3F000FB1F2B013C018EE798E10E941B1D4B01A6
:10C400005C0120E030E040EA50E40F94F41F87FF25
:10C41000DFCE812C912C80EAA82E80E4B82ED8CED5
:10C420000E94A4608111B6CF99CF20E030E0A9012D
:10C43000C501B4010F94182987FF04C0B7FAB0945E
:10C44000B7F8B094F601E15EF34F6F01A5019401D6
:10C45000C301B2010F945A209B01AC01F601608127
:10C460007181828193810F94B726F6016083718375
:10C4700082839383F2E080E090E0A0E4B1E4FF16D1
:10C4800021F080E090E0A8E4B2E48D879E87AF873A
:10C49000B88BCE010D960E94BF297CCFCF93DF933E
:10C4A00000D01F92CDB7DEB780E090E0A0EAB0E404
:10C4B00089839A83AB83BC8361E0CE0101960E949D
:10C4C000E75F0F900F900F900F90DF91CF9108953D
:10C4D0008F929F92AF92BF92CF92DF92EF92FF9294
:10C4E0000F931F93CF93DF93CDB7DEB72C970FB683
:10C4F000F894DEBF0FBECDBF8B0140E050E068E492
:10C5000072E44D835E836F83788740E050E060EA99
:10C5100070E449875A876B877C878130B9F1823014
:10C5200009F459C020E030E040E050E46091270C6D
:10C530007091280C8091290C90912A0C0F94B826A8
:10C540004B017C0120E030E048EC53E40F941829C3
:10C55000181634F4812C912C88ECE82E93E4F92EF3
:10C56000F801A084B184C284D3849401A701B501E9
:10C57000C6010F941829181614F054016701C5015B
:10C58000D60189839A83AB83BC8348C0BE01675FB1
:10C590007F4FC80108960E94C85FB8016C5F7F4F4B
:10C5A000AE014B5F5F4FC8010E94A65F0E94752FCE
:10C5B0002C960FB6F894DEBF0FBECDBFDF91CF91A2
:10C5C0001F910F91FF90EF90DF90CF90BF90AF90B1
:10C5D0009F908F900895F80120853185428553857D
:10C5E0006091270C7091280C8091290C90912A0C55
:10C5F0000F94B8266B017C0120E030E048EC53E456
:10C600000F94F41F87FD06C0C12CD12C28ECE22E1C
:10C6100023E4F22EC982DA82EB82FC82BE01675FDC
:10C620007F4FCE010196B7CFEF92FF920F931F93EA
:10C63000CF93DF937C018B010E946F30CFE1DCE070
:10C640002091610230916202409163025091640234
:10C65000F70160817181828193810F94B2272C85CB
:10C660003D854E855F850F94B8266C877D878E87C4
:10C670009F87C8010E94BF29DF91CF911F910F9121
:10C68000FF90EF900C94A45D4F925F926F927F9217
:10C69000AF92BF92CF92DF92EF92FF920F931F93D0
:10C6A000CF93DF9300D000D01F921F92CDB7DEB79B
:10C6B0005C0180E090E0A0E7B2E489839A83AB83D9
:10C6C000BC8380E090E0A0E8B0EC8D839E83AF83D4
:10C6D000B887BE016F5F7F4FCE0105960E9414633D
:10C6E00068E873E180E090E00E949E25C12CD12C87
:10C6F00088ECE82E81E4F82EC982DA82EB82FC8293
:10C7000080E090E0A0E8B0E48D839E83AF83B8879B
:10C71000BE016F5F7F4FCE0105960E94146301E357
:10C720001CE0F80140AC51AC62AC73ACC0AED1AE11
:10C73000E2AEF3AE80E090E0A0EAB1E489839A83B0
:10C74000AB83BC83F50180819181A281B3818D830C
:10C750009E83AF83B887BE016F5F7F4FCE01059682
:10C760000E941463F80140AE51AE62AE73AE129AED
:10C7700064E670E080E090E00E949E2581E02896CB
:10C780000FB6F894DEBF0FBECDBFDF91CF911F91E2
:10C790000F91FF90EF90DF90CF90BF90AF907F9080
:10C7A0006F905F904F9008951F93CF93DF93CDB715
:10C7B000DEB72C970FB6F894DEBF0FBECDBF182F93
:10C7C000882379F020E030E0A9016091D1057091D3
:10C7D000D2058091D3059091D4050F94F41F88233E
:10C7E000F9F08091300C8117D9F00E94A45D8CE0A3
:10C7F000E8EBF2E0DE01119601900D928A95E1F7E7
:10C80000CE0101960E94C71E8091300C882391F0C2
:10C810008FE19CE00E94E6251092300C0E94DA29FC
:10C820002C960FB6F894DEBF0FBECDBFDF91CF912F
:10C830001F91089581E08093300C8FE19CE00E946D
:10C84000B420ECCF2F923F924F925F926F927F92E3
:10C850008F929F92AF92BF92CF92DF92EF92FF9210
:10C860000F931F93CF93DF93CDB7DEB7CB54D1098E
:10C870000FB6F894DEBF0FBECDBF2DB73EB739AFB0
:10C8800028AF87E00E94ED4A81110BC061E086E588
:10C890000E94EC238DA3853060F08CE39DE00E9424
:10C8A0003235A8ADB9AD0FB6F894BEBF0FBEADBF5F
:10C8B00040C33DA1332321F08CE19DE00E9432353D
:10C8C0006AE080E50E94EC23182F8CEF810F8F32F5
:10C8D00018F088EF9CE0E3CF60E085E40E94082434
:10C8E000882309F448C081E08FABE0903012F090CB
:10C8F0003112D7012D913D914D915C9160911F0CAA
:10C900007091200C8091210C9091220C0F94B826EC
:10C91000AB01BC0188E50E945A2469877A878B871E
:10C920009C87F70124813581468157816091230CD2
:10C930007091240C8091250C9091260C0F94B826B0
:10C94000AB01BC0189E50E945A246D877E878F87E1
:10C95000988BBE01635F7F4FCE0109960E94152D13
:10C96000382E81110BC063E684EE9CE00E94783C77
:10C970008CEC9CE094CF92E09FABB7CF8CE40E940C
:10C98000DC1D082F882309F431C10E94D8238EA30F
:10C99000803118F085EA9CE082CFFEA1F13009F4E5
:10C9A00027C160E083E50E9408248AAF882321F034
:10C9B000011102C037E03EA38DA1833020F08BE847
:10C9C0009CE00E9432359091300C9DAF80E00E9437
:10C9D000D4630E94711C1D8A1E8A1F8A188E198EAC
:10C9E0001A8E1B8E1C8E83EF9FE4A3ECB7E48D8F11
:10C9F0009E8FAF8FB8A383EF9FE4A3ECB7EC89A31E
:10CA00009AA3ABA3BCA3A12FB0E0BCA7ABA7EDB783
:10CA1000FEB724E0129FE019F10911240FB6F89433
:10CA2000FEBF0FBEEDBF8DB79EB701969CAF8BAF1B
:10CA30002DA14FA9BE01635F7F4FCE0109960F94D0
:10CA400034119B01AC010F94AA29811162C20E948A
:10CA500010A3611571058105910511F00F947A1BE2
:10CA6000212C1BAA1CAA1DAA1EAAAEA1A150BB0B59
:10CA70002C96BFAFAEAF2C97E22DF0E0F8A7EFA356
:10CA80002BA53CA5E217F3070CF074C23196FEA764
:10CA9000EDA73F932F93FF93EF9387E79CE09F933E
:10CAA0008F9381E89CE09F938F931F920F94701057
:10CAB0008DB79EB709960FB6F8949EBF0FBE8DBF77
:10CAC0009EA1992309F458C10F942B1B2AE030E052
:10CAD00040E050E00F945A260F94FB1F20E030E016
:10CAE00040EA50E40F9418290FEF1FEF181614F0C6
:10CAF00001E010E00F942B1B28E631E040E050E00D
:10CB00000F945A260F94FB1F2B013C010F942B1BF3
:10CB100020E230E040E050E00F945A266B5F7F4FF8
:10CB20008F4F9F4F0F94FB1F4B015C01ADA1A430B1
:10CB3000D1F4BC01A40189E69CE00E94E63DB3016A
:10CB4000A20181E69CE00E94E63D8BE59CE00E940C
:10CB500032350130110519F483E40E94F93487E578
:10CB60009CE00E943235312CC801110FAA0BBB0B7F
:10CB70002A968CAF9DAFAEAFBFAF2A972C96AEADC5
:10CB8000BFAD2C973A161B060CF0F6C02A966CAD7A
:10CB90007DAD8EAD9FAD2A970F94FB1F6B017C017D
:10CBA000BAADBB2341F1AC019B010F94B82620E044
:10CBB00030E040E952E40F945A209B01AC01C301DC
:10CBC000B2010F94B8262B013C0120E030E044EB89
:10CBD00053E40F9418291816FCF420E030E044EBDD
:10CBE00053E4C301B2010F94B726EDCF1EA2D9CEF4
:10CBF00022E02EA3D6CE0F942B1B24E130E040E0A0
:10CC000050E00F945A26675E7F4F8F4F9F4F0F94CF
:10CC1000FB1FA7019601CFCF20E030E0A901C3019F
:10CC2000B2010F94F41F87FF0BC020E030E044EB0B
:10CC300053E4C301B2010F94B8262B013C01ECCFA1
:10CC40000091301210913112F80124813581468112
:10CC500057816D857E858F8598890F94B72622969A
:10CC60006CAF7DAF8EAF9FAF22972BED3FE049E4D5
:10CC700050E4C301B2010F945A2020E030E044E3B5
:10CC800053E40F94B2276B017C010F94AD276FA77B
:10CC900078AB89AB9AABD8012D913D914D915C91C8
:10CCA00069857A858B859C850F94B72626966CAF0F
:10CCB0007DAF8EAF9FAF2697A50194016FA578A990
:10CCC00089A99AA90F945A209B01AC0126966CADB4
:10CCD0007DAD8EAD9FAD26970F94B82669837A837C
:10CCE0008B839C83C701B6010F945829A501940139
:10CCF0000F945A2022962CAD3DAD4EAD5FAD2297DC
:10CD00000F94B8266D837E838F8398874BE351E021
:10CD100070E060E0CE0101960E94DCBD46E351E088
:10CD200070E060E0CE0105960E94DCBDBDA1B4308C
:10CD300099F449815A816B817C818BE49CE00E944B
:10CD4000E63D4D815E816F81788589E39EE20E9498
:10CD5000E63D8AE00E94F934198A1A8A1B8A1C8AE5
:10CD6000AE014F5E5F4FBE016B5F7F4FCE010196FC
:10CD70000E94A65F339402CF20E04FA9BE01635FFB
:10CD80007F4FCE0109960F9434114B015C01312C79
:10CD9000AC019B010F94AA29811102C03324339462
:10CDA000A5019401C501B4010F94AA298111E2C023
:10CDB000EFA1F8A5EE0FFF1FEE0FFF1F2BAD3CAD4F
:10CDC000E20FF31F80829182A282B382A5019401B7
:10CDD0006D8D7E8D8F8D98A10F941829181624F4CF
:10CDE0008D8E9E8EAF8EB8A2A501940169A17AA105
:10CDF0008BA19CA10F94F41F87FF04C089A29AA263
:10CE0000ABA2BCA2A50194016BA97CA98DA99EA986
:10CE10000F94B8266BAB7CAB8DAB9EABADA5BEA51E
:10CE2000BD01BB0F880B990B0F94FB1F6FA378A755
:10CE300089A79AA79B01AC016BA97CA98DA99EA982
:10CE40000F94B2272B013C014D8A5E8A6F8A788E3F
:10CE5000EBADFCADF8ABEFA710E0C12CD12C760107
:10CE6000AFA5B8A96D917D918D919D91B8ABAFA7FC
:10CE7000A30192010F94B7269B01AC010F945A2095
:10CE80009B01AC01C701B6010F94B8266B017C0170
:10CE90001F5F211628F72FA138A549A55AA50F9481
:10CEA000B2270F946629698F7A8F8B8F9C8FBDA1D3
:10CEB000B23068F18DA59EA50E943AEE6BA57CA5C7
:10CEC00086E49CE00E94083E80E49CE00E943235AB
:10CED00043E0C501B4010E945EB680E20E94F934CD
:10CEE00081E0EDA1E3300CF480E0E12C8E010F5DD8
:10CEF0001F4F9E01235E3F4FAE01475E5F4FBE0155
:10CF00006B5E7F4F0E94C73B8AE00E94F9342394F6
:10CF1000B3CD0E94A4600E94581C8DAD0E94D463C2
:10CF20000E94752F88AD99AD0FB6F8949EBF0FBEC5
:10CF30008DBFE8ADF9AD0FB6F894FEBF0FBEEDBFE3
:10CF4000C55BDF4F0FB6F894DEBF0FBECDBFDF91DC
:10CF5000CF911F910F91FF90EF90DF90CF90BF90F6
:10CF6000AF909F908F907F906F905F904F903F9089
:10CF70002F9008950E94A460332069F285E39CE01D
:10CF80000E94323581E0FDA11F160CF080E0EE24F6
:10CF9000E3948E010F5D1F4F9E01235E3F4FAE0154
:10CFA000475E5F4FBE016B5E7F4F0E94C73B698D3E
:10CFB0007A8D8B8D9C8D0052110926E042E00F94F2
:10CFC000C11A9F938F9384E29CE09F938F938EE28C
:10CFD0009CE09F938F931F920F9470102DB73EB7D4
:10CFE000295F3F4F0FB6F8943EBF0FBE2DBF93CFC2
:10CFF0002F923F924F925F926F927F928F929F9269
:10D00000AF92BF92CF92DF92EF92FF920F931F9356
:10D01000CF93DF93CDB7DEB76A970FB6F894DEBF34
:10D020000FBECDBF83E50E94DC1D182F3090300C61
:10D03000882319F00E94F823382E40901F0C50903E
:10D04000200C6090210C7090220C8091230C909108
:10D05000240CA091250CB091260C8B8B9C8BAD8B56
:10D06000BE8B8091270C9091280CA091290CB09137
:10D070002A0C8F8B988FA98FBA8F112329F031102A
:10D0800003C080E00E94D46386E50E94DC1D8A8B89
:10D0900020E030E0A9016091D1057091D205809126
:10D0A000D3059091D4050F94F41F882309F4C9C0C7
:10D0B00083E40E94DC1D882309F49DC00E94302473
:10D0C0006B017C01A7E8B7E0B987A887BF83AE836F
:10D0D000F5E0FD831D861E8628EC2F8702EC1A865C
:10D0E000212C88EC8B8792E49C87AE81BF81B98B21
:10D0F000A88B15E0E889F98981909190A190B19071
:10D10000F98BE88B2A85322D4B855C85C501B401EE
:10D110000F94F41F87FF04C08A86292CAB86BC8637
:10D120002D853E854F85502FC501B4010F941829D8
:10D13000181624F48D869E86AF860B2D1150D1F6DD
:10D14000FD81F150FD838E819F8144969F838E8364
:10D15000F111CBCF2D853E854F85502F6A85722DDD
:10D160008B859C850F94B82620E030E040E05FE39B
:10D170000F945A20A70196010F94B8264B015C0129
:10D180002DEB37E346E855EB0F94182987FD0AC0CD
:10D190002DEB37E346E855E3C501B4010F94F41FC6
:10D1A00018164CF580E00E94D46310E0E884F984FE
:10D1B00000E0D7016D917D918D919D917D016D0173
:10D1C000B4E0CB1AD108A50194010F94B726F6015B
:10D1D0006083718382839383602F812F0F94630F09
:10D1E0000F5F053031F71F5F8885998544969987D1
:10D1F00088871530D9F6AA89AA2381F020E030E08B
:10D20000A9016091D1057091D2058091D3059091CB
:10D21000D4050F94F41F81110E944F3D8AE50E94AE
:10D22000DC1D882351F00E94302469837A838B832C
:10D230009C83CE0101960F942B0E832D0E94D46304
:10D240000BC0311003C09A89992341F30E94DD4A33
:10D2500085E69BE00E943235332051F08091300CFE
:10D26000811106C00E94D94A86E49BE00E943235B3
:10D270000E94DD4A88E39BE00E9432358091300CA9
:10D280000E94C83D0E94DD4A8BE29BE00E9432353D
:10D29000C090C308D090C408E090C508F090C608BC
:10D2A00020E030E0A901C701B6010F941829181633
:10D2B0000CF053C042E0C701B6010E945EB68DE09B
:10D2C0000E94F9348AE00E94F934A301920160912E
:10D2D0001F0C7091200C8091210C9091220C0F94C6
:10D2E000F41F81111FC02B893C894D895E89609193
:10D2F000230C7091240C8091250C9091260C0F9496
:10D30000F41F81110FC02F89388D498D5A8D60917E
:10D31000270C7091280C8091290C90912A0C0F9465
:10D32000F41F81110E94752F6A960FB6F894DEBF24
:10D330000FBECDBFDF91CF911F910F91FF90EF9066
:10D34000DF90CF90BF90AF909F908F907F906F9025
:10D350005F904F903F902F90089586E29BE00E944F
:10D360003235B3CF8F929F92AF92BF92EF92FF92DE
:10D370000F931F93CF93DF9380E00E94D4631092AA
:10D38000CD051092CE051092CF051092D0051092C7
:10D39000C9051092CA051092CB051092CC051092C7
:10D3A000D5051092D6051092D7051092D805109287
:10D3B000D1051092D2051092D3051092D40507E83A
:10D3C00017E0C0E0812C912C80ECA82E8FE7B82EBE
:10D3D0007801D0E0F70181929192A192B1927F0100
:10D3E0006D2F8C2F0F94630FDF5FD53099F7CF5FD0
:10D3F0000C5E1F4FC53061F7DF91CF911F910F91E8
:10D40000FF90EF90BF90AF909F908F900895909174
:10D41000351280913612981308C08091FB089091C4
:10D42000FC08892B11F40C94961E80E00E943A5659
:10D43000EECF2F923F924F925F926F927F928F9298
:10D440009F92AF92BF92CF92DF92EF92FF920F9393
:10D450001F93CF93DF93CDB7DEB7A6970FB6F8949F
:10D46000DEBF0FBECDBF8EE697E00E9407298091F8
:10D47000DD0B83FD7EC020912B0C30912C0C409154
:10D480002D0C50912E0C60917A0770917B07809142
:10D490007C0790917D070F94F41F882309F469C0DD
:10D4A0001091FA08111161C080915F0290916002A1
:10D4B00001972091E3113091E411281739073CF4CA
:10D4C0000E94DD4A8CE098E10E94323511E0209103
:10D4D0002B0C30912C0C40912D0C50912E0C609106
:10D4E0007A0770917B0780917C0790917D070F945C
:10D4F000B7266B017C0120E030E0A9010F941829C8
:10D5000087FF04C0F7FAF094F7F8F09420916102D5
:10D51000309162024091630250916402C701B601EA
:10D520000F945A2020E030E84BE354E40F9418297C
:10D530001816ECF40E94DD4A8DEE97E10E94323518
:10D5400080917A0790917B07A0917C07B0917D072D
:10D5500080932B0C90932C0CA0932D0CB0932E0C3D
:10D560008AE797E00E94B55D04C010E0B0CF1111CA
:10D57000E7CF2AE037ED43E25CE36091410270912E
:10D58000420280914302909144020F945A206B0111
:10D590007C016091670270916802072E000C880B75
:10D5A000990B0F94FB1F9B01AC01C701B6010F94AF
:10D5B0005A20698B7A8B8B8B9C8B8091300C8823C3
:10D5C00009F18090C3089090C408A090C508B0905D
:10D5D000C608C0907607D0907707E0907807F09063
:10D5E000790720E030E0A901C501B4010F94F41FD0
:10D5F0008823D1F1A7019601C501B4010F94182920
:10D60000181694F1C12CD12C76018E010F5E1F4F9C
:10D610002AE737E046E757E062E777E08EE697E0F3
:10D620000E940DF580E1EEE6F7E0AFE1BCE001908D
:10D630000D928A95E1F7A6960FB6F894DEBF0FBE5D
:10D64000CDBFDF91CF911F910F91FF90EF90DF90B1
:10D65000CF90BF90AF909F908F907F906F905F9092
:10D660004F903F902F90089520911F0C3091200CE7
:10D670004091210C5091220C60916E0770916F07C0
:10D6800080917007909171070F94B7266D8B7E8BF8
:10D690008F8B988F2091230C3091240C4091250C76
:10D6A0005091260C609172077091730780917407F6
:10D6B000909175070F94B726698F7A8F8B8F9C8F07
:10D6C0002091270C3091280C4091290C50912A0C64
:10D6D000C701B6010F94B7266D8F7E8F8F8F98A3E9
:10D6E00020912B0C30912C0C40912D0C50912E0C34
:10D6F00060917A0770917B0780917C0790917D07FC
:10D700000F94B7266B017C0120E030E0A9016D8900
:10D710007E898F89988D0F94F41F81110CC020E0B1
:10D7200030E0A901698D7A8D8B8D9C8D0F94F41F4B
:10D73000882309F467CF2D893E894F89588DCA0106
:10D74000B9010F945A204B015C01298D3A8D4B8D04
:10D750005C8DCA01B9010F945A209B01AC01C5012F
:10D76000B4010F94B8264B015C012D8D3E8D4F8D79
:10D7700058A1CA01B9010F945A209B01AC01C501FF
:10D78000B4010F94B8264B015C01A7019601C701B3
:10D79000B6010F945A209B01AC01C501B4010F944E
:10D7A000B8260F9466294B015C012DEB37E346E860
:10D7B00055E30F94F41F87FF0FC020E030E0A9016C
:10D7C000C701B6010F9418294601570187FF04C00D
:10D7D000B7FAB094B7F8B0942DEB37E346E855E3C9
:10D7E000C501B4010F94F41F87FD1CCF20E030E089
:10D7F00040EA51E4C501B4010F94B2270F942B28DD
:10D800001B01672B19F422242394312CB10190E0E1
:10D8100080E00F94F91F9B01AC0160E070E080E8AC
:10D820009FE30F94B2272B013C01AC019B01C50182
:10D83000B4010F945A204B015C01A30192016D8940
:10D840007E898F89988D0F945A206D8B7E8B8F8B5C
:10D85000988FA3019201698D7A8D8B8D9C8D0F9489
:10D860005A20698F7A8F8B8F9C8FA30192016D8DC7
:10D870007E8D8F8D98A10F945A206D8F7E8F8F8F04
:10D8800098A3A3019201C701B6010F945A2069A37E
:10D890007AA38BA39CA380E1EFE1FCE08E010F5FF4
:10D8A0001F4FD80101900D928A95E1F70E9410A3B5
:10D8B0002B013C0128EC420E511C611C711C0DA374
:10D8C0001EA381E0281A310809F460C00E9410A349
:10D8D0008B019C01041915092609370937FD59C028
:10D8E0002B013C0128EC420E511C611C711C80E094
:10D8F0000E943A562D893E894F89588D69817A81D7
:10D900008B819C810F94B82669837A838B839C8357
:10D91000298D3A8D4B8D5C8D6D817E818F819885AF
:10D920000F94B8266D837E838F8398872D8D3E8DCF
:10D930004F8D58A169857A858B859C850F94B82673
:10D9400069877A878B879C8729A13AA14BA15CA123
:10D950006D857E858F8598890F94B8266D877E8723
:10D960008F87988B750164018E010F5E1F4F9E019A
:10D97000235F3F4FAE01475F5F4FBE016B5F7F4F3D
:10D980008DA19EA10E940DF581119BCF75016401AF
:10D990003CCE0E941EBEAECF8F929F92AF92BF929E
:10D9A000CF92DF92EF92FF92CF93DF93809041026C
:10D9B00090904202A0904302B0904402FC01C080CB
:10D9C000D180E280F38020E030E0A901C701B601F8
:10D9D0000F94F41F882341F0C0924102D09242027A
:10D9E000E0924302F0924402C0916702D091680233
:10D9F00084E690E09093680280936702C090610291
:10DA0000D0906202E0906302F090640280E090E0C7
:10DA1000A0E8BFE38093610290936202A093630247
:10DA2000B09364020E94196A80924102909242026D
:10DA3000A0924302B0924402D0936802C09367025E
:10DA4000C0926102D0926202E0926302F09264029C
:10DA5000DF91CF91FF90EF90DF90CF90BF90AF908C
:10DA60009F908F9008950F931F93CF93DF9300D0D3
:10DA70001F92CDB7DEB79C010EE617E090E1EFE113
:10DA8000FCE0D80101900D929A95E1F7F90120810F
:10DA9000318142815381F80160857185828593854A
:10DAA0000F94B826F801608771878287938780E09A
:10DAB00090E0A0EAB0E489839A83AB83BC83CE0173
:10DAC00001960E94CC6C0F900F900F900F90DF91F9
:10DAD000CF911F910F9108952F923F924F925F9295
:10DAE0006F927F928F929F92AF92BF92CF92DF926E
:10DAF000EF92FF921F93CF93DF93CDB7DEB72C97B2
:10DB00000FB6F894DEBF0FBECDBF7A011901DC015C
:10DB10002D913D914D915C912D833E834F8358878C
:10DB2000FB01408051806280738080901F0C909038
:10DB3000200CA090210CB090220CA50194016D81C5
:10DB40007E818F8198850F94F41F81110EC011E0A2
:10DB5000A30192016091230C7091240C8091250CFB
:10DB60009091260C0F94F41F811110E0D1012D919A
:10DB70003D914D915C9129873A874B875C87F701EE
:10DB8000C080D180E280F38020910B0230910C02A2
:10DB900040910D0250910E02C701B6010F94F41F7F
:10DBA000882309F44EC0C0920B02D0920C02E0927E
:10DBB0000D02F0920E0280912B0C90912C0CA091F2
:10DBC0002D0CB0912E0C4091230C5091240C60919F
:10DBD000250C7091260C80926E0790926F07A09290
:10DBE0007007B09271074093720750937307609368
:10DBF000740770937507C0927607D0927707E0920A
:10DC00007807F092790780937A0790937B07A09327
:10DC10007C07B0937D0720E030E040E05FE3609157
:10DC20005D0C70915E0C80915F0C9091600C0F9474
:10DC30005A2069837A838B839C83CE0101960E944C
:10DC4000CC6C2D813E814F81588520936E07309397
:10DC50006F0740937007509371074092720750927C
:10DC600073076092740770927507D1012D913D91F1
:10DC70004D915C9160917A0770917B0780917C0750
:10DC800090917D070F94B82660937A0770937B0775
:10DC900080937C0790937D0711112FC020E030E026
:10DCA000A90169857A858B859C850F94F41F811164
:10DCB00033C060E070E088EC92E469837A838B8300
:10DCC0009C83CE0101960E94CC6C2C960FB6F894E2
:10DCD000DEBF0FBECDBFDF91CF911F91FF90EF90C0
:10DCE000DF90CF90BF90AF909F908F907F906F907C
:10DCF0005F904F903F902F9008952AEF3EE74AE2C1
:10DD00005FE36091610C7091620C8091630C909163
:10DD1000640C0F945A20D1CF60E070E080EA91E467
:10DD2000CCCF0F931F93CF93DF9300D000D01F92DF
:10DD30001F92CDB7DEB78B01FC0123A5211102C0D4
:10DD40000F94F2131D821E821F82188620E030E09D
:10DD500040E05FE36091270C7091280C8091290CC2
:10DD600090912A0C0F94B82669837A838B839C83C5
:10DD70009E012B5F3F4FAE014F5F5F4F63E27CE040
:10DD80008FE19CE00E946C6D1D821E821F821886AE
:10DD900020E030E040E05FE3F80160857185828536
:10DDA00093850F94B82669837A838B839C83B8010B
:10DDB0006C5F7F4F9E012B5F3F4FAE014F5F5F4F08
:10DDC000C8010E946C6D28960FB6F894DEBF0FBE96
:10DDD000CDBFDF91CF911F910F9108959B01AC01B1
:10DDE000485F5F4FBC016C5F7F4F0C946C6D2F924E
:10DDF0003F924F925F926F927F928F929F92AF92DB
:10DE0000BF92CF92DF92EF92FF920F931F93CF9327
:10DE1000DF93CDB7DEB7A6970FB6F894DEBF0FBE7F
:10DE2000CDBF8C011B015A87498740901F0C509031
:10DE3000200C6090210C7090220C8090230C90900C
:10DE4000240CA090250CB090260CDB018D919D91A7
:10DE50000D90BC91A02D8B8B9C8BAD8BBE8B9C01B0
:10DE6000AD01C301B2010F94B7266B017C01D10152
:10DE700014968D919D910D90BC91A02D8F8B988FB4
:10DE8000A98FBA8F9C01AD01C501B4010F94B726CB
:10DE90006B8F7C8F8D8F9E8FA985BA858D919D917B
:10DEA0000D90BC91A02D8B879C87AD87BE879C0170
:10DEB000AD01C301B2010F94B7266F8F78A389A378
:10DEC0009AA3A985BA8514968D919D910D90BC91C8
:10DED000A02D8F87988BA98BBA8B9C01AD01C501B2
:10DEE000B4010F94B7266BA37CA38DA39EA3A701B7
:10DEF0009601C701B6010F945A206B017C012B8D4E
:10DF00003C8D4D8D5E8DCA01B9010F945A209B0145
:10DF1000AC01C701B6010F94B8264B015C012B89F7
:10DF20003C894D895E896B857C858D859E850F94A6
:10DF3000B7262B013C012F89388D498D5A8D6F856D
:10DF4000788989899A890F94B7266B017C01A3018E
:10DF50009201C301B2010F945A202B013C01A70189
:10DF60009601C701B6010F945A209B01AC01C30171
:10DF7000B2010F94B8260F9466296B017C012F8D96
:10DF800038A149A15AA1CA01B9010F945A202B0105
:10DF90003C012BA13CA14DA15EA1CA01B9010F9486
:10DFA0005A209B01AC01C301B2010F94B8269B011A
:10DFB000AC01C501B4010F9418291816B4F520E07E
:10DFC00030E0A901C701B6010F94182987FF2AC0C4
:10DFD000C701B601905820E030E040EA50E40F94C9
:10DFE0001829181614F5A10169857A85C8010E94BF
:10DFF000F76EA6960FB6F894DEBF0FBECDBFDF91C9
:10E00000CF911F910F91FF90EF90DF90CF90BF9035
:10E01000AF909F908F907F906F905F904F903F90C8
:10E020002F900895C701B601D6CF20E030E040E040
:10E0300050E4C501B4010F941829181624F4B10155
:10E04000C8010E94916E19821A821B821C82BE0135
:10E050006F5F7F4FC1010E94EE6E2DEC3CEC4CECEB
:10E060005CE3C701B6010F945A209B01AC01F80193
:10E0700060817181828193810F945A206D837E83A8
:10E080008F839887D8019B968C919B978823C9F0A2
:10E090002AE939E949E95FE314966D917D918D9103
:10E0A0009C9117970F945A2069837A838B839C8362
:10E0B000BE016F5F7F4F8EE697E00E94EE6EF80123
:10E0C00013A6BE016B5F7F4F89859A850E94EE6E15
:10E0D00090CF3F924F925F926F927F928F929F92DA
:10E0E000AF92BF92CF92DF92EF92FF920F931F9366
:10E0F000CF93DF93CDB7DEB76C970FB6F894DEBF42
:10E100000FBECDBFDB010C91142F100F153008F09E
:10E1100067C11196DC90C22ECD0CB4E0BC1508F49A
:10E120005FC1ED2DF0E0E750FB4F8080912CB12CCA
:10E13000A12C002E04C0B694A794979487940A94B7
:10E14000D2F780FE4DC1EC2DF0E0E750FB4F808010
:10E15000912CB12CA12C012E04C0B694A7949794B5
:10E1600087940A94D2F780FE3BC1322E642F7C0143
:10E170004090C9055090CA056090CB057090CC05C1
:10E180008091D1059091D205A091D305B091D4058D
:10E19000898F9A8FAB8FBC8F660F770B072E000C81
:10E1A000880B990B0F94FB1F4B015C01602F000F34
:10E1B000770B880B990B0F94FB1F298D3A8D4B8D94
:10E1C0005C8D0F945A20A30192010F94B826A501EB
:10E1D00094010F94B8266D877E878F87988B612F67
:10E1E000110F770B880B990B0F94FB1F298D3A8D1C
:10E1F0004B8D5C8D0F945A20A30192010F94B82689
:10E20000A50194010F94B72669837A838B839C833D
:10E210004090CD055090CE056090CF057090D00510
:10E220008091D5059091D605A091D705B091D805DC
:10E23000898F9A8FAB8FBC8F632D660F770B072E5C
:10E24000000C880B990B0F94FB1F4B015C016D2D8B
:10E25000DD0C770B880B990B0F94FB1F298D3A8DE2
:10E260004B8D5C8D0F945A20A30192010F94B82618
:10E27000A50194010F94B826698B7A8B8B8B9C8BAC
:10E280006C2DCC0C770B880B990B0F94FB1F298DF1
:10E290003A8D4B8D5C8D0F945A20A30192010F94FF
:10E2A000B826A50194010F94B7266D837E838F83D2
:10E2B0009887F70180859185A285B38589879A879C
:10E2C000AB87BC878D8B9E8BAF8BB88F45E351E0BE
:10E2D00061E070E0CE0141960E94DCBD45E351E073
:10E2E00061E070E0CE0105960E94DCBD4AE351E09A
:10E2F00061E070E0CE010D960E94DCBD4AE351E082
:10E3000061E070E0CE0101960E94DCBD89889A88A8
:10E31000AB88BC8827E137EB41ED58EBC501B40170
:10E320000F94182987FD5CC023E030E04BE953E4EB
:10E33000C501B4010F94F41F18160CF451C08D845C
:10E340009E84AF84B88827E137EB41ED58EBC501D7
:10E35000B4010F94182987FD43C023E030E84DE94C
:10E3600053E4C501B4010F94F41F1816CCF18D804D
:10E370009E80AF80B88427E137EB41ED58EBC501B3
:10E38000B4010F94182987FD2BC023E030E04BE93E
:10E3900053E4C501B4010F94F41F18160CF18980E1
:10E3A0009A80AB80BC8027E137EB41ED58EBC5018B
:10E3B000B4010F94182987FD13C023E030E84DE91C
:10E3C00053E4C501B4010F94F41F18164CF0AE01CC
:10E3D0004F5F5F4FBE01635F7F4FC7010E94F76EC3
:10E3E0006C960FB6F894DEBF0FBECDBFDF91CF9114
:10E3F0001F910F91FF90EF90DF90CF90BF90AF9063
:10E400009F908F907F906F905F904F903F90089576
:10E410002F923F924F925F926F927F928F929F9234
:10E42000AF92BF92CF92DF92EF92FF920F931F9322
:10E43000CF93DF93CDB7DEB7CC58D1090FB6F894A0
:10E44000DEBF0FBECDBF85E19BE00E94323587E085
:10E450000E94ED4A81116EC084E50E942A1E882325
:10E4600029F00E941D2481110E944CB680E090E0AA
:10E47000A0E8BFE389839A83AB83BC838D839E83AB
:10E48000AF83B8878DEC9CECACE4BEE389879A87B8
:10E49000AB87BC8780E090E0A0E2B1E48D879E87E7
:10E4A000AF87B88B8CE390E09A8B898B8DEC90E0F2
:10E4B0009C8B8B8B8DEC9CECACECBEE38D8B9E8BA4
:10E4C000AF8BB88F80E090E0A0EEBFE3898F9A8F8A
:10E4D000AB8FBC8F1BA61CA64AE959E969E97EE30C
:10E4E0008FE40E945A246D8F7E8F8F8F98A360E0F7
:10E4F00083E40E94082489A360E08BE40E9408243E
:10E500008AA382E40E942A1E882381F10E941D248E
:10E51000009761F19C01285231092536310520F11F
:10E520006CE870E087EE9AE00E94083E82EE9AE086
:10E530000E943235C457DF4F0FB6F894DEBF0FBECE
:10E54000CDBFDF91CF911F910F91FF90EF90DF90A2
:10E55000CF90BF90AF909F908F907F906F905F9083
:10E560004F903F902F9008959A8B898B8CE40E9456
:10E570002A1E8823E1F00E9430246B017C01C986A9
:10E58000DA86EB86FC8620E030E0A9010F9418299A
:10E5900087FD0AC020E030E040E050E4C701B6014A
:10E5A0000F94F41F18161CF48AEB9AE0C1CF81E592
:10E5B0000E94DC1D882331F18091020590910305B2
:10E5C000892BE9F00E9430246B017C01CD82DE8230
:10E5D000EF82F8862DEC3CEC4CE45DE30F941829B7
:10E5E00087FD0AC020E030E040E751E4C701B601F2
:10E5F0000F94F41F181634F489E89AE099CF8EE549
:10E600009AE096CF83E50E942A1E8823E9F00E94B3
:10E6100030246B017C01CD8ADE8AEF8AF88E2DECE6
:10E620003CEC4CEC5DE30F94182987FD0AC020E018
:10E6300030E040E050E4C701B6010F94F41F181613
:10E640001CF487E39AE074CF80E50E94DC1D8823E8
:10E6500041F18091020590910305892B19F48FEF08
:10E6600099E066CF8BA58F5F8BA70E9430246B014A
:10E670007C01CD86DE86EF86F88A20E030E0A901B5
:10E680000F94182987FD0AC020E030E048EC51E4DF
:10E69000C701B6010F94F41F18161CF487ED99E01A
:10E6A00047CF86E40E942A1E8823E9F00E94302486
:10E6B0006B017C01C98EDA8EEB8EFC8E20E030E09F
:10E6C00040E85FE30F94182987FD0AC020E030E09E
:10E6D00040E850E4C701B6010F94F41F18161CF46B
:10E6E0008EEA99E025CFC98CDA8CEB8CFC8C8D8876
:10E6F0009E88AF88B88CA7019601C701B6010F9418
:10E700005A209B01AC0160E070E084E490E40F9437
:10E71000B22729813A814B815C810F945A202B01C9
:10E720003C01A5019401C501B4010F945A20A70131
:10E7300096010F945A202CEE31E548EB5DE30F94DF
:10E74000B2279B01AC01C301B2010F945A20698327
:10E750007A838B839C8388E40E942A1E882379F025
:10E760000E941D24009759F09C01255A31092F3031
:10E77000314018F080E899E0DBCE9C8B8B8B85E5EF
:10E780000E94DC1D8823C9F00E9410A36115710549
:10E790008105910511F00F947A1B809102059091EB
:10E7A0000305892B91F00E9430246093FE0470933E
:10E7B000FF04809300059093010582E50E94DC1D13
:10E7C000811108C08CE499E0B3CE60E070E088E489
:10E7D00092E4EBCF8091020590910305892B61F0C3
:10E7E0000E941D24AD969FAF8EAFAD9718161906E7
:10E7F0004CF088E199E09CCE8AE190E0AD969FAF25
:10E800008EAFAD9789E50E942A1E882381F10E9470
:10E8100030242091CB083091CC084091CD08509104
:10E82000CE080F94B7266B017C0188E50E942A1E52
:10E83000882331F10E9430242091C7083091C80804
:10E840004091C9085091CA080F94B7266BA37CA3C6
:10E850008DA39EA3CFA2D8A6E9A6FAA6CE01839641
:10E860000E949B1D811115C08EEE98E061CEC09074
:10E87000230CD090240CE090250CF090260CD5CFE2
:10E8800060911F0C7091200C8091210C9091220CB2
:10E89000DDCF84E40E94DC1D91E089270E94D463CF
:10E8A00080E090E0A0EAB0E48DA79EA7AFA7B8AB48
:10E8B00060E0CE018D960E94E75F9091F007CD5702
:10E8C000DF4F9883C358D0401092F0070E94951BE9
:10E8D0008DEC98E00E94323589899A898A319105B8
:10E8E0000CF044C08B899C890E94B21E61E080E0DC
:10E8F0000E94ECB8811142C06FEF82EE98E00E9456
:10E90000783C8CA5811104C0CE0101960F94F213BE
:10E9100080E090E0A0EAB0E48093760790937707D8
:10E92000A0937807B09379071DA61EA61FA618AA64
:10E93000BE01635D7F4F8EE697E00E94EE6ECD577D
:10E94000DF4F5881C358D0405093F0070E94951B69
:10E950008AA18111EFCD10927B1110927A110E9441
:10E96000A4BA90E080E00E94B21EE4CD0E94F021A3
:10E9700081E00E9475B78111B5CFBECF10922B0CEC
:10E9800010922C0C10922D0C10922E0C8BE29CE00D
:10E990000E94B55D8BA5882309F452C020E030E0C9
:10E9A00040E751E46091610C7091620C8091630CBE
:10E9B0009091640C0F94B2276DA77EA78FA798AB98
:10E9C00080E1EFE1FCE0AEE6B7E001900D928A95C0
:10E9D000E1F72D853E854F85588960917A077091C2
:10E9E0007B0780917C0790917D070F94B8266093F8
:10E9F0007A0770937B0780937C0790937D07CE0105
:10EA00008D960E94CC6C2D853E854F8558896091EE
:10EA10007A0770917B0780917C0790917D070F9416
:10EA2000B72660937A0770937B0780937C07909357
:10EA30007D078CA5811104C0CE0101960F94F213BD
:10EA4000E9EFF4E085E0DF011D928A95E9F780E1C6
:10EA5000EFE1FCE0AEE6B7E001900D928A95E1F7B8
:10EA600089859A85AB85BC858093760790937707D7
:10EA7000A0937807B09379071DA61EA61FA618AA13
:10EA8000BE01635D7F4F8EE697E00E94EE6EBE0191
:10EA9000635E7F4F8EE697E00E94EE6E89A1882329
:10EAA00009F41CC420911F0C3091200C4091210CC2
:10EAB0005091220CE5962CAF3DAF4EAF5FAFE5977E
:10EAC0008091230C9091240CA091250CB091260CE0
:10EAD000E1968CAF9DAFAEAFBFAFE197312C212C4B
:10EAE0009FEFA4969FAFA497AFEFA896AFAFA8975C
:10EAF000BFEFC158DF4FB883CF57D040EFE4C058C5
:10EB0000DF4FE883C058D040F3ECCF57DF4FF88396
:10EB1000C158D04027E4CE57DF4F2883C258D04099
:10EB200081E090E0A0E0B0E0022C04C0880F991FC3
:10EB3000AA1FBB1F0A94D2F7CC57DF4F8883998353
:10EB4000AA83BB83C458D040A9EFB4E0E796BFAF17
:10EB5000AEAFE79710E000E09101032C000C440BEE
:10EB6000550BC857DF4F288339834A835B83C858C6
:10EB7000D040C457DF4F2882CC58D040E796AEAD86
:10EB8000BFADE7978D91E796BFAFAEAFE79790E047
:10EB9000B0E0A0E0CC57DF4F288139814A815B810A
:10EBA000C458D04082239323A423B523892B8A2BD6
:10EBB0008B2B09F024C1C857DF4F688179818A8186
:10EBC0009B81C858D0400F94FB1F2091D1053091F4
:10EBD000D2054091D3055091D4050F945A2020912D
:10EBE000C9053091CA054091CB055091CC050F94D1
:10EBF000B826EB966CAF7DAF8EAF9FAFEB97B801A9
:10EC0000012E000C880B990B0F94FB1F2091D5054A
:10EC10003091D6054091D7055091D8050F945A20D0
:10EC20002091CD053091CE054091CF055091D00572
:10EC30000F94B8266B017C01EB962CAD3DAD4EAD2B
:10EC40005FADEB97E5966CAD7DAD8EAD9FADE59775
:10EC50000F94B7262B013C01A7019601E1966CADFC
:10EC60007DAD8EAD9FADE1970F94B7264B015C0152
:10EC7000A3019201C301B2010F945A202B013C0160
:10EC8000A5019401C501B4010F945A209B01AC0168
:10EC9000C301B2010F94B8260F9466294B015C01A1
:10ECA000EB962CAD3DAD4EAD5FADEB976BA17CA16E
:10ECB0008DA19EA10F94B7262B013C01A7019601BF
:10ECC0006FA178A589A59AA50F94B7266B017C0141
:10ECD000A3019201C301B2010F945A202B013C0100
:10ECE000A7019601C701B6010F945A209B01AC0100
:10ECF000C301B2010F94B8260F94662920E030E0DA
:10ED000040E751E40F94B227A50194010F94B8266F
:10ED10006B017C018090FE049090FF04A0900005A0
:10ED2000B090010520E030E040E85FE3C501B401A8
:10ED30000F9418291816F4F4C501B4010F9424286F
:10ED40004B015C0160E070E0CB01181419041A0457
:10ED50001B0434F40F942B1BA50194010F945A2625
:10ED60000F94FB1F9B01AC01B601C7010F94B8269D
:10ED70006B017C01C158DF4F2881CF57D040C0586C
:10ED8000DF4F3881C058D040CF57DF4F4881C1583E
:10ED9000D040CE57DF4F5881C258D040B601C7018E
:10EDA0000F94F41F87FF2BC0A4960FAFA497C457EE
:10EDB000DF4F3881CC58D040A8963FAFA897EC964B
:10EDC000CFAEEC97ED96DFAEED97EE96EFAEEE9709
:10EDD000EF96FFAEEF97C158DF4FC882CF57D040B4
:10EDE000C058DF4FD882C058D040CF57DF4FE8829D
:10EDF000C158D040CE57DF4FF882C258D0400F5F85
:10EE00001F4F0530110509F0B9CE4FEF241A340A0F
:10EE100055E02516310409F083CEA4968FADA49752
:10EE2000E82FF0E0E750FB4F208181E090E0A0E088
:10EE3000B0E0A8960FACA89704C0880F991FAA1F2E
:10EE4000BB1F0A94D2F7822B8083A8969FADA89708
:10EE50006A969FAF6A97A496AFADA4976B96AFAF33
:10EE60006B97EC968FADEC97ED969FADED97EE9688
:10EE7000AFADEE97EF96BFADEF976F968CAF9DAFAE
:10EE8000AEAFBFAF6F97A896BFADA897BF3F09F4CD
:10EE900009C2A496EFADA497EF3F09F403C26B2F0C
:10EEA000BB0F770B880B990B0F94FB1F2091D1059B
:10EEB0003091D2054091D3055091D4050F945A203A
:10EEC0002091C9053091CA054091CB055091CC05E0
:10EED0000F94B826162F072F382E292E862F902F05
:10EEE000A32DB22D65968CAF9DAFAEAFBFAF65972A
:10EEF000A496FFADA4976F2FFF0F770B880B990B8C
:10EF00000F94FB1F2091D5053091D6054091D70570
:10EF10005091D8050F945A202091CD053091CE05FF
:10EF20004091CF055091D0050F94B8266B017C011C
:10EF30006996CCAEDDAEEEAEFFAE6997CE018F5ACC
:10EF40009F4F0E949B1D882309F4B0C120E030E050
:10EF500040EA50E4612F702F832D922D0F94B82634
:10EF60004B015C01CB01D50121968CAF9DAFAEAFBB
:10EF7000BFAF21972596CCAEDDAEEEAEFFAE2597A6
:10EF8000A8962FADA8972111E3C1A4963FADA497F1
:10EF90003111B3C120E030E040EA50E4C701B601CE
:10EFA0000F94B8266B017C01A4964FADA49744231F
:10EFB00009F4C5C1A4968FADA49784300CF0BFC1ED
:10EFC00022ED422E23E5522E2BE7622E21E4722EF3
:10EFD00021968CAC9DACAEACBFAC219725968CAD88
:10EFE0009DADAEADBFAD2597A7968CAF9DAFAEAF33
:10EFF000BFAFA7979C01AD0169966CAD7DAD8EAD9D
:10F000009FAD69970F94B726AB966CAF7DAF8EAF6F
:10F010009FAFAB97A501940165966CAD7DAD8EADAC
:10F020009FAD65970F94B7262D966CAF7DAF8EAFD1
:10F030009FAF2D97AB962CAD3DAD4EAD5FADAB9771
:10F0400061962CAF3DAF4EAF5FAF6197A5019401C4
:10F0500060911F0C7091200C8091210C9091220CDA
:10F060000F94B7264B015C01A7962CAD3DAD4EAD7C
:10F070005FADA7976091230C7091240C8091250CB3
:10F080009091260C0F94B726A7966CAF7DAF8EAFEC
:10F090009FAFA797812F902FA32DB22D8DA79EA74D
:10F0A000AFA7B8ABC9AADAAAEBAAFCAAC984DA84CA
:10F0B000EB84FC84CDAADEAAEFAAF8AE2DEC3CECE2
:10F0C0004CEC5CE3C301B2010F945A2029813A81D0
:10F0D0004B815C810F945A2020912B0C30912C0C89
:10F0E00040912D0C50912E0C0F94B82669AF7AAF39
:10F0F0008BAF9CAFA5019401C501B4010F945A20B8
:10F100004B015C01A7962CAD3DAD4EAD5FADA79711
:10F11000CA01B9010F945A209B01AC01C501B40189
:10F120000F94B82620E030E040E050E40F94182916
:10F130001816ACF420E030E040E05FE3C701B60110
:10F140000F94B82629966CAF7DAF8EAF9FAF2997ED
:10F15000BE01635C7F4FCE0101960E94916E89854E
:10F160009A85AB85BC8529968CAF9DAFAEAFBFAFFE
:10F170002997A3961CAE1DAE1EAE1FAEA397BE016F
:10F18000615A7F4FCE01CD960E94EE6E8CA58823EA
:10F19000C1F02AE939E949E95FE36D817E818F8118
:10F1A00098850F945A20A3966CAF7DAF8EAF9FAF1A
:10F1B000A397BE01615A7F4F8EE697E00E94EE6EE4
:10F1C0001CA6E090590CF0905A0C00915B0C109129
:10F1D0005C0CA090550CB090560CC090570CD09081
:10F1E000580C9501A601B701C8010F9418291816EB
:10F1F00014F4750186018090410290904202A09023
:10F200004302B09044022DEC3CEC4CEC5DE3B701C2
:10F21000C8010F945A206093410270934202809378
:10F2200043029093440240E0BE01675B7F4FCE01F2
:10F230008D960E945EC280E1EFE1FCE0AEE6B7E0B1
:10F2400001900D928A95E1F78092410290924202DC
:10F25000A0924302B092440220E04FEFBE01675AF1
:10F260007F4FCE0101960E94697020E041E0BE010F
:10F27000675A7F4FCE0101960E9469702FEF40E0E0
:10F28000BE01675A7F4FCE0101960E94697021E04E
:10F2900040E0BE01675A7F4FCE0101960E9469701F
:10F2A0000E94A45D80919C0C80939D0CAD964EAD08
:10F2B0005FADAD9741505109AD965FAF4EAFAD9781
:10F2C000452B09F419CB6A968FAD6A9787FD14CB4D
:10F2D0006B968FAD6B9787FFE1CB0ECB2BA13CA13B
:10F2E0004DA15EA1E5962CAF3DAF4EAF5FAFE59768
:10F2F0008FA198A5A9A5BAA5EBCB812F902FA32DFF
:10F30000B22D21968CAF9DAFAEAFBFAF219720E05D
:10F3100030E040EA50E4C701B6010F94B7262596C5
:10F320006CAF7DAF8EAF9FAF2597A4965FADA497CE
:10F3300054300CF42FCE182D092D3A2C2B2C92ED95
:10F34000492E93E5592E9BEF692E90E4792E40CEFD
:10F35000A8969FADA89794300CF452C0A496AFAD78
:10F36000A497A4300CF120E030E040EA50E4612F93
:10F37000702F832D922D0F94B72621966CAF7DAF01
:10F380008EAF9FAF219720E030E040EA50E4C70104
:10F39000B6010F94B7266B017C01A496EFADA4973C
:10F3A000E4300CF40DCECBCF812F902FA32DB22DB6
:10F3B00021968CAF9DAFAEAFBFAF219720E030E07C
:10F3C00040EA50E4C701B6010F94B82625966CAF09
:10F3D0007DAF8EAF9FAF2597A496BFADA497B11117
:10F3E000D2CF20E030E040EA50E4612F702F832D2F
:10F3F000922D0F94B726162F072F382E292E9FCF28
:10F40000A496FFADA497F1110DC020E030E040E2DA
:10F4100051E4B401C5010F94B726162F072F382EDB
:10F42000292ECECDA4962FADA49724309CF020E0B9
:10F4300030E040E251E4B401C5010F94B7262196B3
:10F440006CAF7DAF8EAF9FAF2197182D092D3A2C51
:10F450002B2CB6CD182D092D3A2C2B2C82ED482EB5
:10F4600083E5582E8BEF682E81E4782EB1CD2F9254
:10F470003F924F925F926F927F928F929F92AF9244
:10F48000BF92CF92DF92EF92FF920F931F93CF9391
:10F49000DF93CDB7DEB7EA970FB6F894DEBF0FBEA5
:10F4A000CDBF8091300C888B87E50E94DC1D8823BE
:10F4B00009F423C120E030E0A9016091D1057091E9
:10F4C000D2058091D3059091D4050F94F41F81113A
:10F4D00008C00E94D94A82E19CE00E94323510E0C7
:10F4E0001FC18AE50E942A1E882339F10E94302418
:10F4F0002091CF083091D0084091D1085091D20886
:10F500000F94B7266B017C0120E030E040E251EC23
:10F51000C701B6010F94182987FD0AC020E030E02A
:10F5200040E251E4C701B6010F94F41F181674F4B9
:10F530000E94D94A85E09CE0D0CFC090270CD090A3
:10F54000280CE090290CF0902A0CDECF40E050E02F
:10F5500060EC7FE788E50E945A242091C70830912B
:10F56000C8084091C9085091CA080F94B7262B01CA
:10F570003C0140E050E060EC7FE789E50E945A24BE
:10F580002091CB083091CC084091CD085091CE0805
:10F590000F94B7264B015C016FEF89E40E94EC23C6
:10F5A000182F6FEF8AE40E94EC23082FA301920129
:10F5B000C301B2010F94AA2981116EC0A501940163
:10F5C000C501B4010F94AA29811166C08BA19CA129
:10F5D000ADA1BEA18FA798ABA9ABBAAB2091C905CD
:10F5E0003091CA054091CB055091CC05C301B201C1
:10F5F0000F94B7262B013C0120E030E040E05FE3B0
:10F600006FA578A989A99AA90F945A209B01AC01EA
:10F61000C301B2010F94B8262FA538A949A95AA948
:10F620000F94B2270F942428162F4FA058A469A432
:10F630007AA42091CD053091CE054091CF0550910F
:10F64000D005C501B4010F94B7264B015C0120E041
:10F6500030E040E05FE3C301B2010F945A209B0108
:10F66000AC01C501B4010F94B826A30192010F9417
:10F67000B2270F942428062F812F012E000C990BFE
:10F6800097FD33C005979CF5802F002E000C990B39
:10F6900097FD2FC005977CF5153008F020CF053079
:10F6A00008F01DCF80E00E94D46395E01902F001BC
:10F6B0001124E00FF11D07FDFA95EE0FFF1FEE0F6D
:10F6C000FF1FE957F84FC082D182E282F382602F98
:10F6D000812F0F94630F88890E94D46388898823BF
:10F6E00009F4FDCE0E94752FFACE10E0CDCF14E0C4
:10F6F000CBCF00E0D1CF04E0CFCF8AE40E94DC1D65
:10F70000182F811127C070E060E086E50E94212457
:10F710009A838983059708F180EE9BE00E94323539
:10F72000812FEA960FB6F894DEBF0FBECDBFDF91F2
:10F73000CF911F910F91FF90EF90DF90CF90BF90EE
:10F74000AF909F908F907F906F905F904F903F9081
:10F750002F9008950E94B269C2CE60E084E40E94B6
:10F7600008248F8740E050E0BA018AE50E945A24BD
:10F770006BA77CA78DA79EA740E050E86BE376E4DB
:10F7800083E50E945A2420E030E040E752E40F94E1
:10F79000B22760933D0270933E0280933F029093A4
:10F7A0004002E0903012F0903112D7018D909D9080
:10F7B000AD90BC9020E030E0A901C501B4010F94E8
:10F7C000B8266FAB78AF89AF9AAF20E030E040E267
:10F7D00051E40F94F41F87FF06C01FAA18AEB0E2D1
:10F7E000B9AFE1E4EAAF20E030E84DE953E4C50108
:10F7F000B4010F94B8266FA7672E8BAB9CAB20E0AB
:10F8000030E041E953E40F941829181634F41FA688
:10F81000612CF1E9FBAB23E42CABD70114968D905E
:10F820009D90AD90BC90179720E030E0A901C501F4
:10F83000B4010F94B826D62EE72EF82E092F20E01B
:10F8400030E040EA51E40F94F41F87FF05C0D12C4B
:10F85000E12CF0EAFF2E01E420E030E04BE953E434
:10F86000C501B4010F94B826B62EC72E8DAB9EAB42
:10F8700020E030E04CE853E40F941829181634F4D3
:10F88000B12CC12CBCE8BDABE3E4EEAB88E40E9434
:10F89000DC1D882309F410C20E9430240F94242810
:10F8A0001B0177FF02C06F5F7F4F7595679571955C
:10F8B000619571096A567F4F072E000C880B990BD2
:10F8C0000F94FB1F762E872E982EA92E2D2D3E2DC0
:10F8D0004F2D502F0F94182918161CF4D72C740193
:10F8E0000A2D2FA938AD49AD5AAD672D782D892D38
:10F8F0009A2D0F941829181624F07FA888AC99AC7B
:10F90000AAAC872D982DA92DBA2D8B8B9C8BAD8BF6
:10F91000BE8B8D2D9E2DAF2DB02F8F8B988FA98FE5
:10F92000BA8FB101330C880B990B0F94FB1F1B018D
:10F930002C01AC019B016D2D7E2D8F2D902F0F94EE
:10F94000B826D62EE72EF82E092F2B2D3C2D4DA9AB
:10F950005EA90F94F41F87FF04C0BD2CCE2CFDAA16
:10F960000EABA2019101672D782D892D9A2D0F9450
:10F97000B826D62EE72EF82E092F2FA5362D4BA907
:10F980005CA90F94F41F87FF04C0DFA66E2CFBAAAE
:10F990000CAB8FA5962DABA9BCA98B8F9C8FAD8F7F
:10F9A000BE8F8B2D9C2DADA9BEA98F8F98A3A9A327
:10F9B000BAA3BE01695E7F4FCE0143960E94152D0A
:10F9C000882309F4AAC1BE01615E7F4FCE014B9628
:10F9D0000E94152DE82E882309F49FC12F89388DA8
:10F9E000498D5A8D6F8D78A189A19AA10F94B72660
:10F9F00020E030E040E85EE30F945A204B015C01C8
:10FA00002B893C894D895E896B8D7C8D8D8D9E8D7A
:10FA10000F94B72620E030E040E85EE30F945A20D0
:10FA20006BA37CA38DA39EA38FA298A6A9A6BAA61A
:10FA300089819A811816190674F48EEA9BE00E9457
:10FA400032358F85882321F084EA9BE00E9432358D
:10FA50008AE00E94F9340E94A45D0E94711C80E03B
:10FA60000E94D46380917F07811103C081E00E94CE
:10FA700037602091D1053091D2054091D305509146
:10FA8000D4056BA17CA18DA19EA10F94F41F8111BF
:10FA900030C02091D5053091D6054091D7055091C1
:10FAA000D8056FA178A589A59AA50F94F41F811197
:10FAB00020C02091C9053091CA054091CB055091D5
:10FAC000CC056B897C898D899E890F94F41F8111E7
:10FAD00010C02091CD053091CE054091CF055091B9
:10FAE000D0056F89788D898D9A8D0F94F41F8823A6
:10FAF000A9F00E94B26988E0FE01B396A1EDB5E0DD
:10FB000001900D928A95E1F788E0FE017396A9ECC9
:10FB1000B5E001900D928A95E1F7188A60E085E4DE
:10FB20000E940824882309F4FBC0F1E0FFA71B868C
:10FB30001C861D861E861A8A9E2C44E7C42E4BE026
:10FB4000D42E52E8A52E5BE0B52E1A8915300CF0A4
:10FB5000F7C06B857C858D859E859B01AC010F94DC
:10FB6000AA298111EDC0992009F4DDC031E03BAB39
:10FB700035E0232E91E09926F12EFF0CFF0CF10EBB
:10FB8000F394898B19896A89121509F4D5C0062E58
:10FB9000000C770B880B990B0F94FB1F2FA138A536
:10FBA00049A55AA50F945A202F89388D498D5A8D11
:10FBB0000F94B8262B013C01612F110F770B880B96
:10FBC000990B0F94FB1F2BA13CA14DA15EA10F949B
:10FBD0005A202B893C894D895E890F94B8266B8306
:10FBE0007C838D839E834F82588669867A8689813D
:10FBF0009A81892B79F06F2D80E99BE00E94DE3D90
:10FC000069E170E08EE89BE00E94083E8BE89BE093
:10FC10000E9432351F9299E19F931F92FF92DF92CB
:10FC2000CF92BF92AF921F920F94701029814FA56F
:10FC3000BE01695F7F4FCE0103960F9434112B01F3
:10FC40003C014B865C866D867E860FB6F894DEBFDF
:10FC50000FBECDBFAC019B010F94AA29811169C0D1
:10FC600089883A8825E0382D320380011124030D5C
:10FC7000111D37FC1A95000F111F000F111F095796
:10FC8000184FA30192016BA57CA58DA59EA50F948D
:10FC9000B826D8016D937D938D939C931397632D14
:10FCA000882D0F94630F188A81E00E943A56F394CE
:10FCB0008989BBA98B0F65CF4D2D5E2D6F2D702FC0
:10FCC00086E40E945A241B012C014FA958AD69AD4E
:10FCD0007AAD8CE40E945A246B8B7C8B8D8B9E8B2F
:10FCE0002F8A388E498E5A8E4B2D5C2D6DA97EA998
:10FCF00082E40E945A246B017C014FA5562D6BA90A
:10FD00007CA982E50E945A246B8F7C8F8D8F9E8FF9
:10FD1000CF8ED8A2E9A2FAA24CCE84EC9BE0FECC16
:10FD200022E02FA704CF8FEF8BAB22242A9484E00C
:10FD300021CF88890E94D4638A898F5F8A8B05CFFF
:10FD40000E94ECF10E94A460882359F088890E94E7
:10FD5000D46380E090E0A0ECBFE78B879C87AD8701
:10FD6000BE876B857C858D859E859B01AC010F943C
:10FD7000AA29811159C08F85811126C082E0F82EF1
:10FD800002E094E0C92E12E0DC2CD11A21E041E01F
:10FD9000612F802F0E94092221E04FEF612F8F2DCC
:10FDA0000E9409222FEF41E06D2D802F0E94092231
:10FDB0002FEF4FEF6D2D8F2D0E940922115020F74C
:10FDC0000150F3940F3FF9F60E944F3D0E94371EF9
:10FDD0008F85811124C087E29CE00E94211D4B0188
:10FDE0005C018FE19CE00E94C71E9B01AC01C50134
:10FDF000B4010F945A209B01AC016091270C7091C3
:10FE0000280C8091290C90912A0C0F94B7266093AE
:10FE1000270C7093280C8093290C90932A0C8F85C3
:10FE20008111E888E092300C0E94581C8091300CBF
:10FE300081110E94DA290E944E620E94752F6B8503
:10FE40007C858D859E8511E09B01AC010F94AA29CC
:10FE5000811166CC44CB8F929F92AF92BF92CF928A
:10FE6000DF92EF92FF920F931F93CF93DF9300D017
:10FE70001F92CDB7DEB75C016B017A01122F002310
:10FE8000E1F10E94DD4A8DE998E00E94323561E09F
:10FE9000812F0E94FE369090130583E08093130516
:10FEA00081E080931E0C0E94F53C82E080938911D2
:10FEB00040E36DE878E089E798E00E94FA3C40E092
:10FEC0006EE170E182E798E00E94FA3C61E08DE625
:10FED00098E00E94DC3C8FE798E00E94C521809169
:10FEE0001E0C882341F060E0812F0E94FE3681E0E5
:10FEF0000E943A56F4CF9092130520E030E0A90119
:10FF0000F50160817181828193810F94F41F8823B0
:10FF100071F080E090E0A0ECB0E489839A83AB8339
:10FF2000BC83BE016F5F7F4FC5010E94146320E058
:10FF300030E0A901F60160817181828193810F9483
:10FF4000F41F882351F18090690C90906A0CA09066
:10FF50006B0CB0906C0C80E090E0A0E7B1E4809373
:10FF6000690C90936A0CA0936B0CB0936C0C80E0BE
:10FF700090E0A0EAB1E489839A83AB83BC83BE019D
:10FF80006F5F7F4FC6010E9414638092690C90924C
:10FF90006A0CA0926B0CB0926C0C20E030E0A901CE
:10FFA000F70160817181828193810F94182918165D
:10FFB00074F480E090E0A0E4B0E489839A83AB839A
:10FFC000BC83BE016F5F7F4FC7010E9414638091A5
:10FFD000E5042EE130E1882311F02EE438E04CE511
:10FFE00058E066E678E081E00E941D3D0E94F53C05
:10FFF00081E00F900F900F900F90DF91CF911F91A4
:020000021000EC
:100000000F91FF90EF90DF90CF90BF90AF909F90B7
:100010008F900895CF93C82F8091DD0B83FD14C07E
:100020008091FA08811110C080915F029091600266
:100030009C01215031094091E5115091E611421780
:10004000530714F40E94B21ECC2329F061E080E033
:10005000CF910C94ECB88091FA0891E089278093B5
:100060003C0280913C02882389F08091E3119091B9
:10007000E4112091E5113091E611821B930B97FF5B
:1000800003C0919581959109029744F410923C0226
:100090008091DD0B83FF06C0C1E01AC080E00E94A2
:1000A0003A56DFCFC091FA08C11112C080915F02A9
:1000B0009091600201972091E5113091E611281787
:1000C000390754F70E94DD4A80E398E00E943235F8
:1000D0008C2FCF910895AF92BF92CF92DF92EF9283
:1000E000FF920F931F93CF93DF93CDB7DEB7649743
:1000F0000FB6F894DEBF0FBECDBF0E94DC4B87FD6C
:10010000AFC08AE50E942A1E882309F4BAC040E0E5
:1001100050E0BA018AE50E945A247B018C012091AB
:10012000270C3091280C4091290C50912A0C60E04A
:1001300070E088EC93E40F94B7265B016C019701A3
:10014000A8010F941829181614F07501860120E0F3
:1001500030E0A901B701C8010F941829181624F43A
:10016000E12CF12C00E010E0B701C8010F94242825
:10017000072E000C880B990B0F94FB1F698B7A8B51
:100180008B8B9C8B20E030E0A9010F94F41F882317
:1001900021F0CE0141960E94336D80E090E0A0EA0C
:1001A000B1E48D879E87AF87B88B19861A861B8628
:1001B0001C868CE40E94DC1D882309F467C00E9421
:1001C00030246B017C0120E030E0A901C701B601B9
:1001D0000F94182987FF04C0F7FAF094F7F8F09409
:1001E000CD82DE82EF82F8862091E5113091E61112
:1001F0002430310574F08091E3119091E411821B59
:10020000930B97FF03C091958195910901E00497A5
:100210000CF400E080E00E940A80882359F022E07C
:10022000AE01435F5F4FBE016B5F7F4FCE0109960A
:100230000E942B7F69897A898B899C898B019C011B
:10024000305809831A832B833C8320E030E0A901D6
:100250000F94F41F882321F0CE0101960E94336D84
:1002600064960FB6F894DEBF0FBECDBFDF91CF917D
:100270001F910F91FF90EF90DF90CF90BF90AF90C4
:100280000895E12CF12C00E211E449CFC090C4059F
:10029000D090C505E090C605F090C70594CF7F9239
:1002A0008F929F92AF92BF92CF92DF92EF92FF9286
:1002B0000F931F93CF93DF9300D000D01F921F9214
:1002C000CDB7DEB76C015B014A01722E7801009157
:1002D00011060E94BE1E8091E5119091E6118E15C7
:1002E0009F051CF4C7010E94B21E80E00E940A8094
:1002F000882331F0272DA401B501C6010E942B7F70
:100300001E141F043CF4C7010E94B21E60E080E08E
:100310000E94ECB881E00E940A8080E090E0A0E7B3
:10032000B2E489839A83AB83BC8380E090E0A0E849
:10033000B0EC8D839E83AF83B887BE016F5F7F4F24
:10034000CE0105960E94146387E00E94F128811176
:1003500058C08091270C9091280CA091290CB09145
:100360002A0C4091ED045091EE046091EF047091DD
:10037000F004C090E904D090EA04E090EB04F0901F
:10038000EC04C0926E07D0926F07E0927007F09273
:1003900071074093720750937307609374077093CB
:1003A00075078093760790937707A0937807B093AB
:1003B000790780E090E0A8E4B2E489839A83AB8374
:1003C000BC83CE0101960E94CC6C8091F104909187
:1003D000F204A091F304B091F40480937607909313
:1003E0007707A0937807B093790780E090E0A0EAC0
:1003F000B0E489839A83AB83BC83CE0101960E94CB
:10040000CC6CC12CD12C80E7E82E82E4F82EC98276
:10041000DA82EB82FC8280E090E0A0E8B0E48D8399
:100420009E83AF83B887BE016F5F7F4FCE01059675
:100430000E94146320E030E0A9016091F5047091FE
:10044000F6048091F7049091F8040F94F41F87FF4D
:100450000BC0C982DA82EB82FC82BE016F5F7F4FE4
:1004600085EF94E00E9414638091F5049091F60466
:10047000A091F704B091F80480932B0C90932C0C6E
:10048000A0932D0CB0932E0C80937A0790937B074A
:10049000A0937C07B0937D078AE797E00E94B55D43
:1004A0008091C80581110F94A90E61E08CEB98E052
:1004B0000E94453C80911B11815080931B1142E5A5
:1004C00057E164EC78E085E00E94FAEF80911B111F
:1004D000882339F00E9425A780911B1181508093B9
:1004E0001B118091E804882351F01092E804809158
:1004F000E6048093F8088091E7048093F9080E944D
:100500006F3080911C11823011F40E9440350E949E
:10051000ECF128960FB6F894DEBF0FBECDBFDF9189
:10052000CF911F910F91FF90EF90DF90CF90BF90F0
:10053000AF909F908F907F900895CF92DF92EF922F
:10054000FF920F931F93CF93DF9300D01F92CDB7ED
:10055000DEB77C016B018A0161E081E498E00E94D2
:10056000453C42E557E168E478E085E00E94FAEF17
:1005700090911B1181E0890F80931B118091DD13F5
:1005800082FF06C08B7F8093DD139E5F90931B11CB
:100590000E940A3680E1EFE1FCE0A9EEB4E00190B0
:1005A0000D928A95E1F70E94A45D8091E804811183
:1005B0000FC081E08093E8048091F8088093E604FE
:1005C0001092F8088091F9088093E7041092F908D6
:1005D00020E030E0A901F70160817181828193817F
:1005E0000F94F41F8823F1F08091FA0881110CC058
:1005F00080915F029091600201972091E311309108
:10060000E4112817390774F080E090E0A0E7B2E425
:1006100089839A83AB83BC83BE016F5F7F4FC70121
:100620000E94146387E00E94F128811103C0B60183
:100630000E94686220E030E0A901F80160817181C8
:10064000828193810F94F41F882341F080E00E94FF
:100650000A80882319F0C8010E944463129A64E654
:1006600070E080E090E00E949E2581E00F900F9066
:100670000F900F90DF91CF911F910F91FF90EF900E
:10068000DF90CF900895CF92DF92EF92FF92CF93B9
:10069000DF936B017C01D42FC091130583E080931D
:1006A000130581E080931E0CC114D104E104F10410
:1006B00031F00E9410A3C60ED71EE81EF91E8091CD
:1006C0001E0C882389F0C114D104E104F10421F443
:1006D0008D2F0E943A56F3CF0E9410A36C197D090A
:1006E0008E099F0997FDF4CF10921E0CC09313053D
:1006F000DF91CF91FF90EF90DF90CF9008950F930F
:100700001F93CF93DF93C82F162F0E94DD4AC1118C
:1007100094C0C4E9D7E0CE010E94323561E0812F58
:100720000E94FE360E9410A3685370458F4F9F4F62
:1007300060930D0670930E0680930F06909310063B
:10074000109211060091130583E08093130530E0A9
:1007500020E04EE150E162E278E082E00E941D3D3F
:1007600082E298E00E94C52181E080931E0C809176
:100770001E0C882309F464C060E0812F0E94FE36BD
:1007800080911106882309F454C00E94DD4A88E054
:1007900098E00E94323530E020E042EF57E069EF08
:1007A00077E082E00E941D3D89EF97E00E94C5211D
:1007B00041E060E070E0CB010E94438330E020E044
:1007C00050E040E065EE77E085E00E941D3D85EE5B
:1007D00097E00E9495320E94BE1E80E00E940A802F
:1007E0000E94DD4ACE010E9432350E9410A3685358
:1007F00070458F4F9F4F60930D0670930E06809348
:100800000F06909310061092110630E020E04EE1A2
:1008100050E169ED77E082E00E941D3D88EC97E0B1
:100820000E94C52181E080931E0C61E0812F0E940F
:10083000FE3681E00E943A569ACFC9EAD7E06BCFE4
:1008400000931305DF91CF911F910F910895CF92DF
:10085000DF92EF92FF920F931F93CF93DF93CDB769
:10086000DEB7A0970FB6F894DEBF0FBECDBF0E94D3
:10087000DC4B87FDCCC085E40E94DC1D882309F495
:10088000D5C00E9430246B017C0120E030E0A9013A
:100890000F94182987FF04C0F7FAF094F7F8F09442
:1008A000F7FAF094F7F8F094CD8EDE8EEF8EF8A282
:1008B0008CE0E4ECF2E0DE01119601900D928A9555
:1008C000E1F78AE50E942A1E882351F040E050E0BB
:1008D000BA018AE50E945A2469877A878B879C87A8
:1008E00088E50E942A1E882351F040E050E0BA01BA
:1008F00088E50E945A2469837A838B839C8389E5E7
:100900000E942A1E882351F040E050E0BA0189E598
:100910000E945A246D837E838F83988785E50E9489
:10092000DC1D882309F489C00E9430246B017C01FE
:1009300020E030E0A901C701B6010F94182987FF14
:1009400004C0F7FAF094F7F8F094F7FAF094F7F897
:10095000F094C98EDA8EEB8EFC8E1D8A1E8A1F8A59
:10096000188E8CE40E94DC1D882309F46FC00E945D
:1009700030246B017C0120E030E0A901C701B60101
:100980000F94182987FF04C0F7FAF094F7F8F09451
:10099000C98ADA8AEB8AFC8A62E070E082E40E940B
:1009A0002124F82E80911B11811131C021E0AE016C
:1009B000475E5F4FBE016F5F7F4FCE014D960E9435
:1009C0009D82882321F16F2D81E00E947F8382E543
:1009D0000E942A1E882309F442C00E941D2440E080
:1009E00050E060EA71E44D875E876F87788B2091D5
:1009F0001B11222361F08C012F2DAE01435F5F4F4D
:100A0000BE016F5E7F4FCE0145960E944F81A0963A
:100A10000FB6F894DEBF0FBECDBFDF91CF911F910F
:100A20000F91FF90EF90DF90CF900895C12CD12CC3
:100A300080E8E82E80E4F82E33CFC090C005D09037
:100A4000C105E090C205F090C30572CFC090C40507
:100A5000D090C505E090C605F090C7058CCF90E01A
:100A600080E0BDCFCF92DF92EF92FF920F931F9362
:100A7000CF93DF93CDB7DEB76C970FB6F894DEBF98
:100A80000FBECDBF8CE40E94DC1D882309F4B0C0EA
:100A90000E9430246B017C0120E030E0A9010F941A
:100AA000182987FF04C0F7FAF094F7F8F094F7FAE2
:100AB000F094F7F8F094C98EDA8EEB8EFC8E8CE011
:100AC000E4ECF2E0DE01119601900D928A95E1F7D7
:100AD00088E50E942A1E8823A1F040E050E0BA0178
:100AE00088E50E945A242091C7083091C808409197
:100AF000C9085091CA080F94B72669837A838B83FB
:100B00009C8389E50E942A1E8823A1F040E050E0E2
:100B1000BA0189E50E945A242091C7083091C8087B
:100B20004091C9085091CA080F94B7266D837E83FF
:100B30008F8398878AE50E942A1E882351F040E01F
:100B400050E0BA018AE50E945A2469877A878B8728
:100B50009C871D861E861F86188A80911B11811115
:100B600038C020E0AE01435F5F4FBE016F5F7F4F33
:100B7000CE0149960E949D82882359F18091C80533
:100B800081110F94A90E60E080E00E947F83898D1F
:100B90009A8DAB8DBC8DB0588D8B9E8BAF8BB88FE3
:100BA000198A1A8A1B8A1C8A1D861E861F86188A25
:100BB00080911B11882369F010E000E020E0AE0175
:100BC0004B5E5F4FBE016F5E7F4FCE010D960E9460
:100BD0004F816C960FB6F894DEBF0FBECDBFDF918C
:100BE000CF911F910F91FF90EF90DF90CF900895DC
:100BF000C12CD12C80E8E82E80E4F82E58CF2F921B
:100C00003F924F925F926F927F928F929F92AF929C
:100C1000BF92CF92DF92EF92FF920F931F93CF93E9
:100C2000DF93CDB7DEB7E5970FB6F894DEBF0FBE02
:100C3000CDBF8DAB209113052CAB21E02093130584
:100C4000809131058D3409F401C6843511F40C947A
:100C50000E9B873409F091C180912F05909130054A
:100C60008B31910509F4DDC108F079C1843091051B
:100C700008F030C12091E3068230910508F48EC15E
:100C8000213009F091C111E0029709F010E00E94B3
:100C9000712419821A821B821C821D821E821F826D
:100CA000188682E50E942A1E882309F490C10E94BA
:100CB00030246B017C0120E030E0A9010F94F41F87
:100CC000882309F4EAC040901F0C5090200C6090DB
:100CD000210C7090220C8091230C9091240CA091F7
:100CE000250CB091260C8CA79DA7AEA7BFA780901E
:100CF0006E0790906F07A0907007B0907107809179
:100D0000720790917307A0917407B091750788AB33
:100D100099ABAAABBBABA5019401C301B2010F947F
:100D2000F41F81110DC028A939A94AA95BA96CA596
:100D30007DA58EA59FA50F94F41F882309F4ADC04F
:100D4000A3019201C501B4010F94B72620E030E061
:100D500040E05FE30F945A2068A779A78AA79BA772
:100D60002CA53DA54EA55FA568A979A98AA99BA92F
:100D70000F94B72620E030E040E05FE30F945A2064
:100D80002B013C0120E030E0A901C701B6010F941E
:100D9000F41F881F8827881F181709F40FC180E0E7
:100DA00090E0A0E8BFEB8CA79DA7AEA7BFA728A5A2
:100DB00039A54AA55BA5CA01B9010F945A204B0178
:100DC0005C01A3019201C301B2010F945A209B015F
:100DD000AC01C501B4010F94B8260F9466294B01EC
:100DE0005C01AC019B01C701B6010F94B72668AB4B
:100DF00079AB8AAB9BABA5019401C701B6010F94F7
:100E0000B8269B01AC0168A979A98AA99BA90F946E
:100E10005A206B017C0120E030E0A9010F941829D1
:100E200087FDD1C0C701B6010F9466296B017C0113
:100E3000C301B2019058A50194010F94B2272CA5CB
:100E40003DA54EA55FA50F945A20A70196010F94CA
:100E50005A2028A539A54AA55BA50F94B826698311
:100E60007A838B839C83A501940168A579A58AA5C3
:100E70009BA50F94B2272CA53DA54EA55FA50F9469
:100E80005A20A70196010F945A20A30192010F94B2
:100E9000B8266D837E838F83988720E030E0A90198
:100EA00069817A818B819C810F94F41F8111A3C089
:100EB00020E030E0A9016D817E818F8198850F94BB
:100EC000F41F811198C00E94D94A80EC9EE00E94D4
:100ED00032356AC08531910509F466C08A319105C1
:100EE00009F49CC0049709F048C080E50E942A1EBE
:100EF000C12CD12C7601882321F00E94AA236B01FA
:100F00007C0183E50E942A1E882361F00E94302420
:100F100020E030E04AE754E40F945A200F942B2845
:100F20006B017C010E94A45D80911D11811105C09F
:100F300060E086ED9EE00E94783C0E9410A3C60E01
:100F4000D71EE81EF91E0E9410A36C197D098E0998
:100F50009F0997FF29C080E00E943A56F4CF8A3259
:100F6000910509F4E8C260F48D31910509F411C2CC
:100F700008F470C04E9709F464C20F94F71014C0BF
:100F80008B35910509F4BAC38C35910509F4BAC3C0
:100F90008A35910591F71092EB0706C0213021F4B4
:100FA0000E9471240E94196A3DA9311102C00F9458
:100FB000A4108CA9809313050C94D49380E090E046
:100FC000A0E8BFE3F0CEC12CD12C760131CF89E46B
:100FD0000E942A1E882331F00E94302469837A837C
:100FE0008B839C838AE40E942A1E882309F455CFB0
:100FF0000E9430244ECF412FBE016F5F7F4F8EE69F
:1010000097E00E945EC20E9410A360936E117093DD
:101010006F118093701190937111C6CF0E94087266
:10102000C3CF87E00E94ED4A8111BECF8CE0E0ED96
:10103000F2E0DE01119601900D928A95E1F770E0E1
:1010400060E080E50E94CA23BE016F5F7F4F0E946F
:101050006862AACF87E00E94F128811106C060E093
:101060008FE40E94082481119FCF0E94A45D1092FA
:1010700046026091300C8CE40E940824E82E80E047
:101080000E94D4630E9410A360936E1170936F113D
:1010900080937011909371110E94711C81E0809374
:1010A000A0060E94492A8AE50E94DC1DF82E8823AA
:1010B00069F081E00E94F128182F82E00E94F12857
:1010C00011110C94319B11E0811101C010E088E5F1
:1010D0000E94DC1D81110C94239B111141C189E5F3
:1010E0000E94DC1D082F811307C0012FF11204C0DC
:1010F00011E001E0FF24F39482E50E942A1E882378
:1011000009F431C10E9430246CA37DA38EA39FA358
:1011100020E030E0A9010F94F41F882361F0111141
:1011200005C0011103C0FF2009F40CC160E0CE012D
:1011300084960E94E75F112309F47FC0002309F41D
:1011400079C010921F0C1092200C1092210C10925A
:10115000220C1092230C1092240C1092250C109249
:10116000260C0E94DA298AE698E10E941B1D4B0199
:101170005C018EE698E10E941B1D2B013C01AC0135
:101180009B01C501B4010F94182918160CF0F0C08A
:10119000A5019401C301B2010F94B2279B01AC01D8
:1011A0000F945A2020E030E040E85FE30F94B82627
:1011B0000F94662920E030E048E452E40F945A206E
:1011C00068A379A38AA39BA320E030E040EC5FE30F
:1011D000C301B2010F945A20905869837A838B839C
:1011E0009C8320E030E040EC5FE3C501B4010F9444
:1011F0005A2090586C8F7D8F8E8F9F8FAE01405EEE
:101200005F4FBE016F5F7F4FCE014C960E94A65F7D
:101210000E941E5210921F0C1092200C1092210C52
:101220001092220C1092230C1092240C1092250C78
:101230001092260C80E00E94AD60002319F081E03E
:101240000E94AD60FF2009F47DC083E00E94ED4A5A
:10125000811178C00E94DA292091FD073091FE07A4
:101260004091FF075091000860E070E086E193E450
:101270000F94B7262B013C01209101083091020800
:10128000409103085091040860E070E086E193E427
:101290000F94B7264B015C018091270C9091280C8C
:1012A000A091290CB0912A0C809376079093770730
:1012B000A0937807B0937907009130121091311202
:1012C000D8012D913D914D915C91C301B2010F94D4
:1012D000B72660936E0770936F07809370079093A3
:1012E0007107F8012481358146815781C501B40118
:1012F0000F94B726609372077093730780937407F7
:10130000909375078EE697E00E949B1D8823A9F1B4
:101310001C8E1D8E1E8E1F8E88E0EEE6F7E0DE012D
:10132000119601900D928A95E1F7AE01445E5F4FF0
:10133000BE016B5F7F4FCE0101960E94A65F82E0E7
:101340000E94AD600E94DA2980919F068093A006DA
:101350008E2D0E94D4630E94581C0E94752F24CEAB
:10136000012F10E0C9CE60E070E080E890E4CCCEC0
:10137000A3019201C501B4010FCF60E081EF9EE0AF
:101380000E94783C0E94DD4A8FED9EE00E9432353B
:10139000D9CF14E00E9410A360936E1170936F1167
:1013A00080937011909371118091300C811127C03E
:1013B0008EE40E94DC1D882321F082E09FE00E94E1
:1013C000639B87E00E94ED4A81111FC00E94377A1B
:1013D0008823D9F0115001F130E020E042E557E1D7
:1013E0006DE27FE085E00E941D3D61E080E29FE0CC
:1013F0000E94453C88E09FE00E94639BCBCF60E069
:101400008FE40E940824882399F20E94F53C8BEC1B
:101410009FE00E94639BC8CD61E08EEB9FE00E943D
:10142000453C89E49FE00E94639B61E08DE397E186
:101430000E94453C40E070E060E08AE39FE00E944B
:1014400061510091301210913112D8012D913D91CE
:101450004D915C9160911F0C7091200C8091210C3A
:101460009091220C0F94B826AB01BC0188E50E9434
:101470005A2469837A838B839C83F8012481358184
:10148000468157816091230C7091240C8091250C2A
:101490009091260C0F94B826AB01BC0189E50E94FF
:1014A0005A246D837E838F839887BE016B5F7F4F45
:1014B000CE0101960E94152D882309F475CD80E098
:1014C0000E94D4630E94711C61E085E40E9408249C
:1014D000182F21E0482FBE016B5F7F4FCE01019690
:1014E0000F9434116B017C01AC019B010F94AA296C
:1014F000811119C049815A816B817C818DEE9FE0F9
:101500000E94E63D4D815E816F81788588EE9FE087
:101510000E94E63DB701A60183EE9FE00E94E63DF2
:101520008AE00E94F9340E94581C11110E944E62F8
:101530000E94752F39CD8091E306813009F034CDBA
:1015400089E40E942A1E082FF12C882319F00E949A
:101550001D24F82E8AE40E942A1EE82E882379F0A2
:101560000E941D24182F002309F4C0C0F4E0FF15C9
:1015700008F0B9C085EF9FE00E94323515CD10E02C
:101580000111F4CF80E1EFE1FCE0AEE6B7E00190BD
:101590000D928A95E1F7002319F16F2DFF0C770B5F
:1015A000880B990B0F94FB1F2091D1053091D20528
:1015B0004091D3055091D4050F945A202091C9052C
:1015C0003091CA054091CB055091CC050F94B826B7
:1015D00060936E0770936F07809370079093710705
:1015E000EE2019F1612F110F770B880B990B0F94D7
:1015F000FB1F2091D5053091D6054091D70550911C
:10160000D8050F945A202091CD053091CE054091F8
:10161000CF055091D0050F94B82660937207709350
:101620007307809374079093750760E080E50E94CC
:1016300008248823C1F10023D1F0E0913012F09109
:101640003112208131814281538160916E07709106
:101650006F0780917007909171070F94B726609380
:101660006E0770936F078093700790937107EE2059
:10167000D1F0E0913012F091311224813581468110
:1016800057816091720770917307809174079091F0
:1016900075070F94B7266093720770937307809352
:1016A00074079093750740E050E0BA0186E40E9409
:1016B0005A246B017C0120E030E0A9010F94182925
:1016C0001816C4F420E030E040E752E4C701B60148
:1016D0000F94B22769837A838B839C83CE01019612
:1016E0000E94CC6C61CCEE2009F44CCF153008F48C
:1016F00049CF40CF60E070E0CB01ECCF8FE080932A
:10170000EB0752CC80912E05882381F1893009F0B6
:101710004BCC1CEDA12E12E0B12E0FE1C02E0CE03F
:10172000D02EE12C00E010E0D5018D915D010E94EA
:101730002A1EF82E882361F0133011F4082FFE2C96
:101740000E943024F6016083718382839383EF2C9F
:101750001F5FF4E0CF0ED11C143031F7EE2009F4F6
:1017600057C00E94DA290E94752F1ECCBCEDCB2EEB
:10177000B2E0DB2EF12CE12C00E010E0D6018D91DF
:101780006D010E942A1E382E8823D9F10E94302430
:101790004B015C01133059F0F701E953F74F2081F9
:1017A0003181428153810F94B7264B015C01F701CF
:1017B000E15EF34F2081318142815381C501B40143
:1017C0000F94B7262B013C012DEB37E346E855EB90
:1017D0000F94182987FD0AC02DEB37E346E855E33F
:1017E000C301B2010F94F41F18165CF41330C1F456
:1017F00080922B0C90922C0CA0922D0CB0922E0C5F
:10180000032D1F5FB4E0EB0EF11C143009F0B6CFCE
:10181000002309F4A8CF8BE29CE00E94B55DA3CF22
:10182000F701EF50F84F5F01A301920160817181D0
:10183000828193810F94B826D5016D937D938D930A
:101840009C931397812F0E94381CDBCF80912F052A
:10185000909130058837910511F40C94A29508F009
:1018600067C28D34910509F4D9C608F0EFC08A31FA
:10187000910509F40EC608F092C08431910509F46F
:1018800054C508F06FC08131910509F415C508F001
:1018900042C0029708F071CB80E50E942A1EC12C3D
:1018A000D12C7601882321F00E94AA236B017C01B0
:1018B00083E50E942A1E882361F00E94302420E0E4
:1018C00030E04AE754E40F945A200F942B286B0120
:1018D0007C010E94A45D8091360590913705892B8B
:1018E00009F4E5C40F94051180912F0590913005FE
:1018F00066E170E1892B11F46EE070E130E020E0E8
:101900004EE150E182E00E941D3D40E0C701B6017A
:101910000E94438349CB429709F02FCB83E50E9475
:101920002A1E882311F40C94DA940E9410A3609369
:101930006E1170936F1180937011909371110E94CA
:10194000302420E030E04AE754E40F945A200F940A
:101950002B286093140270931502809316029093C3
:10196000170222CB8731910509F414C570F4853133
:10197000910509F40BC5469709F0FFCA8091DD1364
:1019800082FD12CB0E9437AF0FCB8831910509F44D
:1019900016C5499709F0F1CA0E94328505CB8032FD
:1019A000910509F4FAC5C0F58D31910509F4DEC53C
:1019B00070F48B31910509F47FC54C9709F0DDCAAD
:1019C00080913605909137050E9429B4EDCA8E3179
:1019D000910509F4D2C54F9709F0CFCA0E94582A41
:1019E0006C8F7D8F8E8F9F8FBE016F5F7F4FCE017B
:1019F0004C960E94E620CE0101960E94B4F10E940E
:101A0000DD4ABE016F5F7F4F82E990E10E944F5334
:101A10008AE00E94F934C8CA8934910509F4EAC5FC
:101A200050F48132910509F4E1C5C09709F0A5CAC7
:101A30000E942264B9CA8B34910509F4EBC58C3439
:101A4000910509F09ACA0E940A36AECA8B369105F2
:101A500009F4C3C608F0F9C08435910509F45ECFD6
:101A600030F58135910509F485C790F48E349105E0
:101A700009F083CA70E060E083E50E9421248E347F
:101A8000910509F0D0C50E9432510E94ECF18CCA38
:101A90008235910509F486C78335910509F06DCA31
:101AA0008091EB078F7E80628093EB077DCA88363A
:101AB000910509F43CC608F099C08535910509F4F3
:101AC000BCC78C35910509F058CA0E94DC4B87FDD4
:101AD0006BCA8091320584FD09C08091340587FD71
:101AE00005C080913505837009F4D4C7ECEDCE2E86
:101AF000E2E0DE2EF1E3EF2EFCE0FF2E10E0D60157
:101B00008D916D010E942A1E882309F465C013304F
:101B100009F0B8C70E9430244B015C0120E030E09E
:101B200040EA51E40F94F41F87FF4EC0A5019401D1
:101B30006091510C7091520C8091530C9091540C07
:101B40000F94B2272B013C01AC019B016091E0088E
:101B50007091E1088091E2089091E3080F945A2077
:101B60006093E0087093E1088093E2089093E308A3
:101B7000A30192016091610C7091620C8091630CE1
:101B80009091640C0F945A206093610C7093620CD6
:101B90008093630C9093640C6091F0087091F1084D
:101BA0008091F2089091F3080F94F91FA30192011C
:101BB0000F945A200F942B286093F0087093F1082B
:101BC0008093F2089093F3088092510C9092520CFB
:101BD000A092530CB092540C1F5FF4E0EF0EF11C76
:101BE000143009F08CCF0E94C225DEC989369105D8
:101BF00009F4C8C58A36910509F0BFC960E080E5DF
:101C00000E94EC23F82EE1E0E81708F4CDC981E446
